:020000040800F2
:103000000080002099EB00084DC800086DC800083A
:1030100000000000000000000000000000000000B0
:10302000000000000000000000000000D3FB0008CA
:103030000000000000000000D5FB00083D03002058
:103040003BEB00086DEB00086FEB000871EB00082C
:1030500073EB000875EB000877EB000879EB0008CC
:103060007BEB0008450300207DEB00087FEB0008A8
:10307000ED03002081EB000883EB000885EB0008DE
:1030800087EB000899C80008A9C80008B9C800085B
:10309000C9C80008D9C80008E9C8000889EB0008B9
:1030A0008BEB00088DEB00088FEB00084904002033
:1030B00091EB000893EB000895EB000897EB0008F4
:1030C00001000000000000000A00000000000000F5
:1030D0006400000000000000E803000000000000A1
:1030E0001027000000000000A08601000000000082
:1030F00040420F0000000000809698000000000091
:1031000000E1F5050000000000CA9A3B0000000045
:1031100000E40B540200000000E8764817000000AD
:103120000010A5D4E800000000A0724E18090000AD
:1031300000407A10F35A00000080C6A47E8D030080
:103140000000C16FF286230000008A5D78456301AC
:10315000000064A7B3B6E00D0000E8890423C78A25
:10316000014902480860704708ED00E0003000089F
:1031700000B587B0544800683821084000902028E6
:1031800000D982E00098810001A040588746C046DF
:103190008B3200088B3200088B3200088B3200081B
:1031A0008B3200088B3200088B3200088B3200080B
:1031B000153200088B3200088B3200088B32000871
:1031C0008B3200088B3200088B3200088B320008EB
:1031D000313200088B3200088B3200088B32000835
:1031E0008B3200088B3200088B3200088B320008CB
:1031F0001D3200088B3200088B3200088B32000829
:103200008B3200088B3200088B3200088B320008AA
:103210002732000830492F48086045E02E497D20BC
:103220000002086040E02C490120C00308603BE038
:10323000264801680322114003910068702108406C
:103240000009401C02900398032805D102992148E7
:103250000AF006FA059004E002991D480AF000FA07
:103260000590059A194801687F231B021940090A35
:10327000514305910068400F401C04900598049943
:103280000AF0EEF9144908600EE0144800680721BE
:10329000C9020840C10A01208840019001990C48E8
:1032A0000AF0DEF90C490860074800680F2109029E
:1032B000084081090A4840580690069A064908685D
:1032C000D040086007B000BD081002400C1002405A
:1032D0000024F40000127A0074060020001002405E
:0432E000E4320008CC
:1032E40000000000000000000000000000000000DA
:1032F40000000000000000000000000000000000CA
:1033040001000000020000000300000004000000AF
:10331400060000000700000008000000090000008B
:103324000000000000000000000000000000000099
:10333400010000000200000003000000040000007F
:1033440000B581B06946002008700A490868012266
:10335400120210430860022000F00EF8002803D087
:1033640069460120087001E009F04AFA68460078CD
:0833740001B000BD0020024081
:10337C0000B583B0029001A90020087017480078AE
:10338C00002824D0164800680090144801787D204D
:10339C00C0000AF05FF9014600980AF05BF90CF0E6
:1033AC00EDFE00280FD10298032808D802990022BC
:1033BC00D0430CF0D3FE02980A49086002E001A940
:1033CC000120087002E001A90120087002E001A9A7
:1033DC000120087001A8007803B000BD3A0300205A
:0833EC007406002054060020C5
:1033F4000348027803490868801808607047C0468B
:083404003A03002044070020F8
:0C340C00014800687047C04644070020DB
:1034180000B583B00290FFF7F5FF01900298009085
:103428000098401C002804D00748017800984018EC
:103438000090FFF7E7FF0199401A0099884200D2EF
:0C344800F7E703B000BDC0463A030020C7
:1034540081B000900449086802229043009A104306
:0C346400086001B07047C0463000014015
:10347000024908680122904308607047300001400B
:1034800081B0009004490868032252029043009AD8
:0C3490001043086001B0704700000140CC
:10349C0000B58BB0099008A9002008700790069021
:1034AC0004900998002803D10AA90120087093E11F
:1034BC0009983C21405C0128FFD10998006900283B
:1034CC0005D009980069012149058842FFD1099866
:1034DC00806D002808D1099804F0CAFD09990020D4
:1034EC00C865099954228854099800680CF0ACFC02
:1034FC00002812D10998006800F082F9B8480068D9
:10350C00B8490AF0A7F84000801C049004980028E1
:10351C0003D00498401E0490F8E7099800680CF05A
:10352C0093FC00280BD10999886D102210438865F3
:10353C00099AD16D01200143D16508A90870099839
:10354C0000680BF026FB05900998806DC0060028DA
:10355C0000D536E10598002800D032E10998806D3D
:10356C0002210843012109028843099988650998B9
:10357C0000680CF073FC00284ED109980068C068F4
:10358C001821884309998A6810430968C86009980A
:10359C004168032292071140C06C0143069808430E
:1035AC00069009983C21405C01280FD10999486884
:1035BC000322920710400A6C10434A6C1043896C2A
:1035CC0008430699084301210843069009980068AE
:1035DC0000698549084006990843099909680861FA
:1035EC000998406803218907884215D009984068DA
:1035FC000121890788420FD0099840680121C90729
:10360C00884209D0794908680F2293049843099A93
:10361C0052681A40801808600998017E8903427E1E
:10362C00D2031143827E52031143026B531E9A4103
:10363C0012038918C26811430291C07C000600284D
:10364C0006D5099800690121C9078843019002E059
:10365C0001204005019002990198014309982C2200
:10366C00805C40000143079808430790099820218B
:10367C00405C012813D10998807E002805D1079859
:10368C00012109040843079009E00999886D20225B
:10369C00104388650999C86D01221043C8650998C3
:1036AC00406A002809D00998416A0722920111400A
:1036BC00806A014307980843079009980068C0681E
:1036CC004B4908400799084309990968C86009984B
:1036DC000068006947490840069908430999096838
:1036EC000861099908684A6B00210BF05BFA09998B
:1036FC0008688A6B40490BF055FA09980069002854
:10370C0007D109980168886A0F22D2431043886256
:10371C0033E0099800690121490588422DD1002028
:10372C000390039807280DD80998006E0399890017
:10373C00C8400F2108400F2800D103E00398401C1B
:10374C000390EEE70398012807D109980168886A6D
:10375C000F22D243104388620FE009980068806AF8
:10376C000999C8698000021F1C2002400F20C04329
:10377C0090400A6E10430968886209980068C06816
:10378C001E490840079988420BD109990020C86549
:10379C000998806D012108430221884309998865A5
:1037AC000EE00998806D1021084302218843099985
:1037BC008865099AD16D01200143D16508A908706B
:1037CC0007E00999886D10221043886508A901202B
:1037DC00087008980AA908700AA800780BB000BDF8
:1037EC0074060020400D030002FCFF1F0827014057
:1037FC001902FEFF02FCFFDF04FFFF07E7FF3F8318
:10380C0081B00090009880680121090708430349A2
:10381C0008400099886001B07047C046E8FFFF7F00
:10382C0000B585B0039000200190039800680CF05F
:10383C0015FB00285BD10398006880682F4908426B
:10384C000CD00399886D102210438865039AD16DB2
:10385C0001200143D16504A908704BE0039800686E
:10386C0000F01AFE26480BF064FA000200280DD571
:10387C0024480068244909F0EDFE401C0190019891
:10388C00002803D00198401E0190F8E70398407E71
:10389C0001282CD0FFF7B4FD029003980068006853
:1038AC00C007002823D1039800680CF0D7FA002831
:1038BC0003D10398006800F0EFFDFFF7A1FD02991A
:1038CC00401A032812D3039800680068C007002828
:1038DC000CD10399886D102210438865039AD16D21
:1038EC0001200143D16504A9087003E0D5E704A9C0
:1038FC000020087004A8007805B000BD17000080F7
:0C390C000827014074060020400D030055
:1039180081B000900098806803490840001D009914
:0C392800886001B07047C046E8FFFF7FD8
:1039340000B585B0039002910192039800680BF0E2
:103944002CF9002860D103985421405C012803D14C
:1039540004A9022008705DE00399542201208854D0
:1039640003980068C068C00700280FD10398006856
:103974000CF078FA002803D00398006800F056F899
:1039840003980168C86801221043C8600398FFF7D0
:103994004BFF0146684601700078002833D1039834
:1039A400806D0121090208431C4908400399886578
:1039B40003990020C8650398016D1948C8620398EB
:1039C400016D184808630398016D1748486303980C
:1039D40001681C200860039954220020885403982D
:1039E400016848681022104348600399086D09680B
:1039F4004031029A019B0BF05AFA69460870039809
:103A04000068FFF787FF02E069460220087000980B
:103A140004A9087004A8007805B000BDFEF1FFFFFA
:0C3A240029FF0008D1EC0008E7EC0008C6
:103A300081B000900098806803490840801C00997C
:0C3A4000886001B07047C046E8FFFF7FBF
:103A4C0000B59DB01B901A9119A900200870179011
:103A5C001B9800690121C907884204D01B98006992
:103A6C00E649884200D1FFE71B985421405C0128AD
:103A7C0003D11CA902200870BCE11B99542201201F
:103A8C0088541B9800680BF084F8002800D0A2E141
:103A9C001A984068022800D15BE11B98006901214B
:103AAC00C907884204D01B980069D449884206D1C2
:103ABC001B9800681A99096800F0AEF9F1E01B98A0
:103ACC00016E1A9843681F2213400F229A409143AB
:103ADC00169100684003002807D11A9800681F212E
:103AEC0089060840800E1590C2E01A980078C0072D
:103AFC00002802D000201490B8E01A9800788007B3
:103B0C00002802D501201390AEE01A9800784007E7
:103B1C00002802D502201290A4E01A980078000721
:103B2C00002802D5032011909AE01A980078C0065C
:103B3C00002802D50420109090E01A980078800696
:103B4C00002802D505200F9086E01A9800784006D0
:103B5C00002802D506200E907CE01A98007800060A
:103B6C00002802D507200D9072E01A984078C00703
:103B7C00002802D008200C9068E01A984078800742
:103B8C00002802D509200B905EE01A984078400777
:103B9C00002802D50A200A9054E01A9840780007B1
:103BAC00002802D50B2009904AE01A984078C006EC
:103BBC00002802D50C20089040E01A984078800626
:103BCC00002802D50D20079036E01A984078400660
:103BDC00002802D50E2006902CE01A98407800069A
:103BEC00002802D50F20059022E01A988078C00793
:103BFC00002802D01020049018E01A9880788007D2
:103C0C00002802D5112003900EE01A9801680120BB
:103C1C00820411401220002301939142029001D0A2
:103C2C0001980290029803900398049004980590D0
:103C3C0005980690069807900798089008980990A0
:103C4C0009980A900A980B900B980C900C980D9070
:103C5C000D980E900E980F900F9810901098119040
:103C6C001198129012981390139814901498159010
:103C7C00169815991A9A52681F231A4091400843B6
:103C8C001B9908661A9840688008401C1B99C969E2
:103C9C00884206D81B9800681A9A516812680BF073
:103CAC0031F81B9800681A9A1168926800F0C2F8F3
:103CBC001A98C078000600284AD551480BF039F8FC
:103CCC0018901A9800684F4988421DD118A880781E
:103CDC000006002818D418990120C0050143484853
:103CEC000CF0DAF94A4800684A4909F0B3FC01467D
:103CFC000C2048430C3017901798002803D01798C5
:103D0C00401E1790F8E723E01A9800683E49884255
:103D1C000CD118A8C078C007002807D11899012029
:103D2C000006014336480CF0B7F911E01A98006808
:103D3C00364988420CD118A880784006002807D450
:103D4C0018990120800501432D480CF0A5F9FFE7D7
:103D5C0040E01B9800690121C907884204D01B98D8
:103D6C0000692649884205D11B9800681A99096890
:103D7C0000F074F81A98C078000600282AD520485C
:103D8C000AF0D7FF18901A9800681E49884207D18C
:103D9C0018990120C005814319480CF07DF919E0F0
:103DAC001A9800681849884207D118990120000612
:103DBC00814313480CF070F90CE01A980068134911
:103DCC00884207D118990120800581430C480CF0DA
:103DDC0063F9FFE707E01B99886D20221043886583
:103DEC0019A9012008701B99542200208854199895
:103DFC001CA908701CA800781DB000BD0400008030
:103E0C0008270140001000B0004000B8002000B4AA
:083E1C0074060020400D0300B4
:103E240082B001900091009A034802400199886A87
:0C3E34001043886202B07047FFFF0700D7
:103E400083B00290019100920298406901990A02A0
:103E5000904300991140034A114008430299486178
:083E600003B0704700FFFF07EB
:103E680082B0019000910098C2430448024301992E
:103E7800886A1040886202B07047C0460000F8FFA8
:103E880000B5B3B0319030912FA900200870309858
:103E98004068032189058842FFD131983C21405C64
:103EA800012800D1FFE731985421405C012803D153
:103EB80032A9022008708DE23199542201208854D9
:103EC800319800680AF067FE002800D054E2309864
:103ED8000068E64988423ED1309840682C9001211C
:103EE800C905884212D02C9803218905884214D12B
:103EF80031980068309989687F22D204914303225F
:103F080092058A18D94900F06FFA0CE031980068D8
:103F1800D649D74A00F068FA05E031980068D349D5
:103F2800002200F061FA3199886D01221204904351
:103F38008865319800680AF007FF3098007B0128EF
:103F480004D1319800680AF006FF03E03198006850
:103F58000AF00AFF10E2309840682B900121C90549
:103F6800884200D1C5E12B9803218905884200D0F9
:103F7800C7E130980068BF49884200D0D9E030983E
:103F880080684003002807D1309880681F2189067F
:103F98000840800E2A90C2E03098007AC0070028B6
:103FA80002D000202990B8E03098007A80070028D5
:103FB80002D501202890AEE03098007A400700280A
:103FC80002D502202790A4E03098007A0007002844
:103FD80002D5032026909AE03098007AC00600287F
:103FE80002D50420259090E03098007A80060028B9
:103FF80002D50520249086E03098007A40060028F3
:1040080002D5062023907CE03098007A000600282C
:1040180002D50720229072E03098407AC007002825
:1040280002D00820219068E03098407A8007002864
:1040380002D5092020905EE03098407A4007002899
:1040480002D50A201F9054E03098407A00070028D3
:1040580002D50B201E904AE03098407AC00600280E
:1040680002D50C201D9040E03098407A8006002848
:1040780002D50D201C9036E03098407A4006002882
:1040880002D50E201B902CE03098407A00060028BC
:1040980002D50F201A9022E03098807AC0070028B5
:1040A80002D01020199018E03098807A80070028F4
:1040B80002D5112018900EE0309881680120820402
:1040C80011401220002316939142179001D01698A0
:1040D8001790179818901898199019981A901A9874
:1040E8001B901B981C901C981D901D981E901E9844
:1040F8001F901F9820902098219021982290229814
:1041080023902398249024982590259826902698E3
:104118002790279828902898299029982A902A98B3
:104128000123834031980168A02288581843885099
:10413800DEE0309880684003002807D13098806816
:104148001F2189060840800E1590C8E03098007A33
:10415800C007002802D000201490BEE03098007AF2
:104168008007002802D501201390B4E03098007A27
:104178004007002802D502201290AAE03098007A61
:104188000007002802D503201190A0E03098007A9B
:10419800C006002802D50420109096E03098007AD6
:1041A8008006002802D505200F908CE03098007A10
:1041B8004006002802D506200E9082E03098007A4A
:1041C8000006002802D507200D9078E03098407A44
:1041D800C007002802D008200C906EE03098407A82
:1041E8008007002802D509200B9064E03098407AB7
:1041F8004007002802D50A200A905AE03098407AF1
:104208000007002802D50B20099050E03098407A2A
:10421800C006002802D50C20089046E03098407A65
:104228008006002802D50D2007903CE03098407A9F
:104238004006002802D50E20069032E03098407AD9
:104248000006002802D50F20059028E03098807AD3
:10425800C007002802D0102004901EE03098807A11
:104268008007002808D51120039014E00000C07CC6
:10427800FFFF8700FFFF1700309881680120820444
:1042880011401220002301939142029001D001981D
:10429800029002980390039804900498059005985A
:1042A800069006980790079808900898099009982A
:1042B8000A900A980B900B980C900C980D900D98FA
:1042C8000E900E980F900F981090109811901198CA
:1042D800129012981390139814901498159015989A
:1042E8000123834031980168A422885818438850D4
:1042F8000EE03198006830990968394A00F074F87E
:1043080006E03198006830990968002200F06CF8DE
:10431800309800683349884217D13199886D012255
:10432800520490438865319800680BF0C5FE3098B8
:10433800007B012804D1319800680BF0C5FE03E02A
:10434800319800680BF0CAFE16E03199886D012299
:10435800920490438865319800680BF0C9FE309844
:10436800007B012804D1319800680BF0C9FE03E0F6
:10437800319800680BF0CEFE3098006817498842E3
:1043880013D13098006931990968C9681822114019
:10439800890888402E903098406931990968C96821
:1043A8001140890888402D9005E0309800692E90CA
:1043B800309840692D9031980068309909682E9A94
:1043C8002D9B00F039F831995422002088542F98F9
:1043D80032A9087032A8007833B000BD0000C07C54
:0843E800FFFF8700FFFF170033
:1043F00084B003900291019202980F49884203D140
:1044000003980C30009008E00398029901225205AD
:104410001140C90C4018A030009000980068029A22
:10442000D143064B194308400199114008430099B4
:10443000086004B07047C0460000C07C00003883AC
:1044400085B004900391029201930498039A03218A
:104450000B0511461940090D01235B051A40520D49
:10446000891889004018203000900098006805499C
:10447000084002990904019A114308430099086011
:0844800005B0704700F000F0E8
:1044880081B0009000988068034908401030009976
:0C449800886001B07047C046E8FFFF7F5D
:1044A40081B000900098806803490840401C00993E
:0C44B400886001B07047C046E8FFFF7F41
:1044C00000B585B003900020019003985421405C12
:1044D000012803D104A90220087061E00399542245
:1044E0000120885403980BF0C7FC02A908700398B8
:1044F00000680BF01DFE002846D10398806D022154
:1045000008430122110288430399886503980068D3
:10451000C06803231840009003980168C868984356
:10452000C860039801688868D207104388600398C0
:1045300000680BF005FE002817D00198401C019080
:104540000198194988420FD30398806D10210843C0
:1045500002218843039988650399542200208854D6
:1045600004A9012008701BE0E1E7009A03980168A4
:10457000C8681043C8600398806D01210843022178
:1045800088430399886504E00399886D10221043DD
:1045900088650399542200208854029804A9087061
:0C45A00004A8007805B000BD00F2020085
:1045AC0070B582B0024601A80270009100214056FD
:1045BC00002815D4002401A908570322D34318401E
:1045CC00164A805809578C07E50EFF24AC40A043CF
:1045DC00009CA401E4B2AC4020431940885019E07F
:1045EC0001A908780F24204008380322D34318402F
:1045FC00094A8058002549578D07EE0EFF25B54016
:10460C00A843009DAD01EDB2B540284321400839C7
:10461C001940885002B070BD1CED00E000E400E0D1
:10462C0081B001466846017000214056002807D42D
:10463C00684601781F20014001208840014908602C
:08464C0001B0704700E100E03D
:1046540081B00146684601700021405600280BD401
:10466400684601781F200140012088400349086002
:10467400BFF34F8FBFF36F8F01B0704780E100E04D
:10468400BFF34F8F034904480860BFF34F8F00BF47
:0C469400FDE7C0460CED00E00400FA0554
:1046A00000B583B001900198401E000E002802D092
:1046B0000120029010E00198401E09490860002086
:1046C0000090C0430321FFF771FF0098054908607F
:1046D000054A072111600290029803B000BDC04650
:0C46E00014E000E018E000E010E000E052
:1046EC0000B583B001900198002803D102A90120E4
:1046FC00087050E00198407F002805D101990020F6
:10470C000877019803F046FD01990220487701983B
:10471C00007900280CD10198016821484861019862
:10472C0000688068182188430199096888600AE04C
:10473C0001988168C2680AF071F9002803D002A9B7
:10474C000120087027E001984079002805D10198D4
:10475C0001680020C043086103E0019908690968F9
:10476C0008610198006880686021884301994A6952
:10477C00104309688860019800688068802188432C
:10478C0001998A691043096888600199012048776A
:10479C0002A90020087002A8007803B000BDC04632
:0447AC00B71DC10470
:1047B00010B588B0069005910492002001900598EC
:1047C00000690128FFD1059800680428FFD10698E8
:1047D0004079012803D107A902200870DFE006997B
:1047E0000120487106990220087105980068042884
:1047F00065D10498002823D1FEF708FE01900698A1
:104800000068406B0004002811D5FEF7FFFD0199F8
:10481000401A02280AD30699086908221043086141
:1048200006990320087107A90870B8E0E7E701209E
:10483000FEF7F2FD059880690699096808641FE093
:1048400006980068406BC00F002811D0FEF7DEFD0F
:104850000199401A02280AD30699086908221043D0
:10486000086106990320087107A9087097E0E7E737
:104870000120FEF7D1FD0598806906990968486412
:1048800006980068806C049B10210B40464A9A40B1
:104890009043059AD2699A401043069A1268906430
:1048A00006980068C06C049A0A40FF219140884332
:1048B0000599096A9140084306990968C8640598F2
:1048C0000069012819D106980068806B039004984C
:1048D000102210401F2181400398884303900598BF
:1048E000406902900299049810408140039808435F
:1048F0000390039806990968886306980068C06B5E
:1049000003900498102210400721814003988843A7
:104910000390059908688B681843C968084302909A
:10492000029904981040814003980843039003982B
:1049300006990968C86304991140012084038C40DA
:1049400006990B681968A1431960069909680968F6
:10495000039104991140154B8B400399994303919E
:10496000059949680291029B049911408B40039973
:10497000194303910399069B1B6819600499114020
:10498000C0238B4006990A68116899431160069903
:10499000087106990020487107A90020087007A82F
:1049A000007808B010BDC046FF030000FE0F0000F5
:1049B00000B585B003900398002803D104A9012015
:1049C000087066E00398019000683449401814218B
:1049D00008F046FE01998000086403992522022010
:1049E00088540398016808682D4A104008600398AD
:1049F00002908268C1680A4301690A4341690A4317
:104A000081690A43C1690A43016A0A430168086867
:104A100010430860039800F045F80398806801216E
:104A20008903884202D103990020486003994868AD
:104A30003F221040496C08600399C86C896C48603B
:104A40000398406800280FD00398406804280BD8CA
:104A5000039800F049F80398016D0020086003995D
:104A6000886D496D486006E0039900200865039948
:104A700048650399886503990020C8630399252236
:104A800001208854039924220020885404A900207E
:104A9000087004A8007805B000BDC046F8FFFDBF4F
:044AA0000F80FFFF85
:104AA40000B583B002900299086C032290430B4A2C
:104AB40080184864029800780838142108F0CEFD64
:104AC400019002990648886401991F200140012041
:104AD40088400299C86403B000BDC0460008024083
:044AE4008008024004
:104AE80082B00190019840683F21084000900098EA
:104AF80080000849401801990865019906484865E9
:104B08000098411E032001400120884001998865D2
:0C4B180002B07047FC0802404009024057
:104B240084B003900291019200930399C86C896C3C
:104B340048600398006D002803D00399886D496D7F
:104B440048600398006C1C210840012282400F49F0
:104B5400086810430860009803990968486003983E
:104B64008068102808D10198039909688860029820
:104B740003990968C86007E0029803990968886086
:104B8400019803990968C86004B0704704000240A2
:104B940082B000900098002803D101A90120087078
:104BA40048E000982521405C02280AD0009904209E
:104BB400C863009924220020885401A901200870A8
:104BC40038E00098016808680E2290430860009855
:104BD400416C086801221302984308600098016838
:104BE4000868904308600098006C1C2108408240CB
:104BF40012490868104308600099C86C896C4860C1
:104C04000098006D00280AD00098016D0868012200
:104C14001202904308600099886D496D48600099BC
:104C2400252201208854009924220020885401A9B7
:104C34000020087001A8007802B070470400024008
:104C440000B587B0059004A801700392059825214A
:104C5400405C02280AD005990420C86305992422DF
:104C64000020885406A901200870B7E00598006860
:104C740000688006002806D5059A01200102D16348
:104C840006A90870AAE004A80078002807D10598AE
:104C9400016C1C20014002208840029006E0059827
:104CA400016C1C200140042088400290FEF7ACFBFC
:104CB40001904C480068029908423FD14948006875
:104CC4000599096C1C221140C8400007002817D51B
:104CD4000598016C1C200140012003468B40424A88
:104CE4001168194311600599C863059925228854F0
:104CF400059924220020885406A9012008706DE03B
:104D04000398401C002818D0FEF77EFB0199401A36
:104D14000399884202D8039800280ED105992020CF
:104D2400C86305992522012088540599242200206E
:104D3400885406A90120087050E0BAE70598006D70
:104D4400002816D00598406D00680599896D0842C1
:104D54000FD00598016D08680122130218430860FA
:104D64000599886D496D48600599C86B9202104396
:104D7400C8630598806C00680599C96C084209D01D
:104D84000599C86C896C48600599C86B0122520268
:104D94001043C86304A80078002812D10598006C59
:104DA4001C210840022282400F4908681043086011
:104DB400059924220020885405992522012088542D
:104DC40009E00598006C1C21084004228240064931
:104DD40008681043086006A90020087006A8007837
:0C4DE40007B000BD0000024004000240C7
:104DF00010B588B006900591039302921C48007884
:104E0000012803D107A9022008702DE018490120CC
:104E100008701749002048607D20C00000F034F879
:104E2000014601A801700078002817D106980128D2
:104E300005D10598039B029A00F074F803E00598E9
:104E4000029900F019F87D20C00000F01DF801A9BA
:104E50000870069A074908689043086004490020D2
:104E60000870019807A9087007A8007808B010BD5D
:104E7000241300201420024008B4024B9C4608BCB6
:084E80006047C046CD0500208B
:104E880000B585B00390FEF7BDFA0399401801906C
:104E98000120000402901D4800680299084209D0C8
:104EA800FEF7B0FA0199884203D304A903200870D9
:104EB80028E0F0E715490868154A1040029015489F
:104EC80008600298002806D002981349486004A98F
:104ED8000120087016E0FEF795FA03994018019032
:104EE8000A4800684003002809D5FEF78BFA0199A3
:104EF800884203D304A90320087003E0F0E704A95B
:104F08000020087004A8007805B000BD10200240F9
:0C4F1800FAC30000FBC3000024130020BB
:104F240084B003900193009207490868012210435A
:104F34000860009803990860BFF36F8F0198039984
:0C4F4400486004B07047C04614200240D2
:104F500081B06946002008700A480068C00F002828
:104F60000CD00949094808600948086005480068EC
:104F7000C00F002802D069460120087068460078FA
:104F800001B0704714200240082002402301674509
:044F9000AB89EFCD2D
:104F940081B068460122027007480168D2071143B4
:104FA40001600068C00F002802D069460020087024
:0C4FB4006846007801B0704714200240ED
:104FC00000B585B0039002912E480078012803D1E6
:104FD00004A90220087051E02A49012008702949DB
:104FE000002048607D20C000FFF74EFF014601A869
:104FF0000170007800283BD1039904204860039891
:10500000006804280AD10398406800F03FF87D202A
:10501000C000FFF739FF01A9087029E002990020BC
:10502000C04308600398806800900098039A9168D4
:10503000D2688918884216D203984068009900F017
:1050400033F87D20C000FFF71FFF014601A8017063
:105050000078002803D000980299086003E00098C7
:10506000401C0090E1E7084908680222904308606C
:10507000044900200870019804A9087004A8007869
:0C50800005B000BD2413002014200240E5
:10508C0081B00090009804490A6810430122120470
:0C509C001043086001B07047142002406F
:1050A80083B002900191074908683F22D2009043DB
:1050B8000090009A0198C0001043034A104308600A
:0C50C80003B070471420024002000100F9
:1050D4008AB0099008910020079008980068079901
:1050E400C840002800D130E108980068079A0121DF
:1050F4009140084006900698002800D121E10898C4
:10510400406803210840012805D00898406803211D
:10511400084002282AD10998806805900798400021
:10512400032181400598884305900898C168079831
:1051340040008140059808430590059809998860C6
:105144000998406805900798012181400598884393
:10515400059008984068102108400109079881408B
:10516400059808430590059809994860089840688F
:1051740003210840032814D00998C06805900798B3
:105184004000032181400598884305900898816870
:1051940007984000814005980843059005980999AF
:1051A400C860089840680321084002281ED1099865
:1051B4000799C90889004018006A059007984007B4
:1051C400C00E0F2181400598884305900898016915
:1051D40007984007C00E814005980843059005983C
:1051E4000999079AD20892008918086209980068F8
:1051F400059007984100032002468A40059991438F
:105204000591089949680140079840008140059834
:1052140008430590059809990860089880798007E3
:10522400002800D18DE0079803218843484940585D
:10523400059007988007C00E0F2181400598884388
:105244000590099805210907884202D1002004909D
:105254001DE009983F49884202D10120039014E0DF
:1052640009983D49884202D1022002900BE0099935
:105274003A4A0320052300939142019001D00098FB
:105284000190019802900298039003980490049965
:1052940007988007C00E814005980843059005983B
:1052A4000799032291432A4A88502D4800680590A3
:1052B400069905988843059008988079C0070028C6
:1052C40003D0069905980843059005982449086079
:1052D4002448006805900699059888430590089825
:1052E40080798007002803D506990598084305901E
:1052F40005981C4908601C480068059006990598A3
:105304008843059008988079C006002803D506993B
:1053140005980843059005981349086013480068E8
:105324000590069905988843059008988079800629
:10533400002803D5069905980843059005980B495C
:1053440008600798401C0790C7E60AB07047C0463B
:10535400601802400004005000080050000C005087
:1053640080180240841802400018024004180240C9
:105374008BB00A9009910020089009980899C840B8
:10538400002800D198E00998089A0121914008402A
:1053940007900798002800D18AE0089803218843E1
:1053A40046494058069008988007C00E0F21814056
:1053B400069808400690069805900A980521090762
:1053C400884202D1002004901DE00A983C4988429A
:1053D40002D10120039014E00A983A49884202D18C
:1053E400022002900BE00A99374A03200523009318
:1053F4009142019001D00098019001980290029886
:1054040003900398049005980499089A9207D20E81
:105414009140884221D1079A2C490868904308603A
:10542400079A2B49086890430860079A2949086835
:1054340090430860079A28490868904308600898D0
:105444008007C10E0F2088400690069B0899032010
:1054540081431A4A88589843885008984000032288
:10546400134683400A990868184308600899480756
:10547400C00E0F2383400A98C90889004118086A9E
:105484009843086208984000134683400A99886844
:10549400984388600898012383400A994868984390
:1054A40048600898400082400A99C8689043C860E0
:1054B4000898401C089060E70BB0704760180240E1
:1054C4000004005000080050000C005080180240F6
:0C54D40084180240001802400418024036
:1054E00000B583B001901749086803225202904327
:1054F000019A10430860019801214902884219D19C
:105500001148016806204843104908F0A9F8401CDA
:1055100000900F480068400500280BD5009800282F
:1055200003D00098401E009003E002A903200870F9
:1055300003E0EEE702A90020087002A8007803B09B
:1055400000BDC046007000407406002040420F00BD
:045550001470004093
:1055540010B588B006900698002803D107A9012049
:105564000870CEE206980078C007002873D0FA4885
:105574000068382108400490F84800680321084076
:1055840003900498102802D10398032802D00498A9
:1055940008280DD1F24800688003002807D5069832
:1055A4004068002803D107A901200870A9E252E04D
:1055B4000698406801210904884206D1E849086830
:1055C40001221204104308601AE00698406805217D
:1055D400090488420AD1E249086801229304184365
:1055E4000860086812041043086009E0DC49086890
:1055F40001221304984308600868920490430860E9
:1056040006984068002813D0FDF7FEFE0590D448A4
:105614000068800300280AD4FDF7F6FE0599401AB5
:10562400652803D307A9032008706AE2EFE712E0B4
:10563400FDF7EAFE0590CA480068800300280AD5F1
:10564400FDF7E2FE0599401A652803D307A9032054
:10565400087056E2EFE7069800788007002800D427
:1056640090E0BD480068382108400490BB480068B9
:105674000321084003900498102802D103980228BB
:1056840002D00498002834D1B548006840050028A9
:1056940007D50698C068002803D107A9012008701F
:1056A4002FE2B04908687F2212029043069A526999
:1056B400120210430860049800280FD1A848026819
:1056C4000721C9028A43069B1B691A4302600068CA
:1056D4000840C10AA448C840A4490860A448006816
:1056E400FDF74AFE002803D007A90120087008E24C
:1056F40048E00698C06800282BD09949086807221A
:10570400D2029043069A1269104308600868012285
:10571400120210430860FDF777FE0590FD4800680B
:10572400400500280AD4FDF76FFE0599401A0328A6
:1057340003D307A903200870E3E1EFE7F6490868FB
:105744007F2212029043069A5269120210430860A3
:1057540018E0F04908680122120290430860FDF73E
:1057640053FE0590EB480068400500280AD5FDF774
:105774004BFE0599401A032803D307A90320087098
:10578400BFE1EFE7069800780007002848D5DF4816
:1057940000683821084018280DD1E04800688007C7
:1057A400002807D506988069002803D107A901209D
:1057B4000870A6E134E006988069002818D0D7491B
:1057C4000868012210430860FDF71EFE0590D348C7
:1057D4000068800700280AD4FDF716FE0599401AD0
:1057E400032803D307A9032008708AE1EFE717E031
:1057F400CA490868012290430860FDF705FE059038
:10580400C6480068800700280AD5FDF7FDFD059904
:10581400401A032803D307A90320087071E1EFE7B6
:10582400069800784007002800D4ADE002A90020C3
:105834000870B64800683821084020280DD1BA48BD
:1058440000688007002807D506988068002803D1DF
:1058540007A90120087054E196E0B1480068C0002F
:1058640000280CD4AE480268012109070A430260EB
:10587400006808400190019802A901200870A94815
:105884000068C005002818D4A6490868012212023D
:1058940010430860FDF7B8FD0590A2480068C005F4
:1058A40000280AD4FDF7B0FD0599401A032803D354
:1058B40007A90320087024E1EFE70698806801280F
:1058C40005D19949086801221043086016E006983A
:1058D4008068052809D194490868042210430860A7
:1058E400086801221043086008E08F490868012213
:1058F4009043086008680422904308600698806812
:10590400002814D0FDF780FD0590874800688007C3
:1059140000280BD4FDF778FD0599401A8349884285
:1059240003D307A903200870EBE0EEE722E0FDF7BC
:105934006BFD05907C480068800700281AD5FDF7A8
:1059440063FD0599401A7949884203D307A90320C6
:105954000870D6E0EEE7C046081002400C10024082
:1059640000100240041002400024F40074060020D9
:105974005406002002A80078012805D16849086867
:1059840001221207904308600698C069002800D1DC
:10599400B4E05E48006838210840102870D00698AA
:1059A400C069022849D15B49086801221206904364
:1059B4000860FDF729FD059056480068800100281D
:1059C4000AD5FDF721FD0599401A032803D307A939
:1059D4000320087095E0EFE74D490868554A1040E8
:1059E400069B1A6A5C6A22439C6A24022243DC6A8C
:1059F40022431C6B22435B6B1A4310430860454BE4
:105A0400186801221406204318600868120710431E
:105A14000860FDF7F9FC05903E4800688001002805
:105A24000AD4FDF7F1FC0599401A032803D307A90A
:105A34000320087065E0EFE721E036490868012299
:105A440012069043086032490868032290430860B4
:105A54000868374A10400860FDF7D6FC05902D48C9
:105A64000068800100280AD5FDF7CEFC0599401A8C
:105A7400032803D307A90320087042E0EFE73DE0C1
:105A84000698C069012803D107A90120087038E0ED
:105A94001F48006803900398032108400699096A87
:105AA400884227D10398702108400699496A8842A0
:105AB40020D103987F21090208400699896A0902C6
:105AC400884217D103981F21490408400699C96ADE
:105AD40088420FD103980721490608400699096BAB
:105AE400884207D103980721490708400699496B62
:105AF400884203D007A90120087002E007A900200A
:105B0400087007A8007808B010BDC046081002400D
:105B14000C100240001002400410024060100240C9
:105B24003C100240007000405C10024089130000E9
:085B3400FFFFFEEE8C80C111A1
:105B3C0000B585B0039002910398002803D104A905
:105B4C0001200870E9E002987649096807221140A3
:105B5C0088421CD97349086807229043029A104363
:105B6C000860FDF74DFC01906E4800680721084065
:105B7C00029988420BD0FDF743FC0199401A7149F8
:105B8C00884203D304A903200870C6E0ECE703980D
:105B9C0000788007002813D5039800784007002868
:105BAC0005D56149086807221203104308605E4955
:105BBC0008680F2212029043039A926810430860FF
:105BCC0003980078C007002860D00398406801282B
:105BDC0009D1584800688003002803D404A9012087
:105BEC0008709AE032E003984068022809D15148C5
:105BFC0000688001002803D404A9012008708CE0FF
:105C0C0024E003984068002809D14A480068400500
:105C1C00002803D404A9012008707EE016E0039844
:105C2C004068032809D1424800688007002803D443
:105C3C0004A90120087070E008E03C480068800767
:105C4C00002803D404A90120087066E036490868CE
:105C5C0007229043039A526810430860FDF7D0FB6B
:105C6C000190314800683821084003994968C900FF
:105C7C0088420BD0FDF7C4FB0199401A3149884288
:105C8C0003D304A90320087047E0EAE702982549EA
:105C9C0009680722114088421CD222490868072251
:105CAC009043029A10430860FDF7AAFB01901D482F
:105CBC00006807210840029988420BD0FDF7A0FB31
:105CCC000199401A1F49884203D304A90320087084
:105CDC0023E0ECE7039800784007002808D5124928
:105CEC000868072212039043039AD2681043086095
:105CFC0000F02AF80C4909680F22120211408A0997
:105D0C000D4989581F221140C8400C4908600C48A5
:105D1C000068FDF72DFB04A9087004A8007805B0F5
:105D2C0000BDC04600200240081002405C1002403A
:105D3C006010024000100240E4320008740600209B
:085D4C00540600208913000039
:105D540000B587B03A4800688006400F00280ED18D
:105D64003B4800680721C9020840C10A0120884055
:105D740002900299354807F071FC01905CE03048CC
:105D8400006838210840082802D12F48019053E0C8
:105D94002B48006838210840102837D12948016869
:105DA4000322114005910068702108400009401C3D
:105DB400039005980090022810D0009803280DD174
:105DC4000399214807F04AFC01461E4800687F22D7
:105DD40012021040000A484306900CE003991B4845
:105DE40007F03CFC0146174800687F22120210406D
:105DF400000A4843069013480068400F401C049072
:105E04000698049907F02AFC019015E00C480068F4
:105E140038210840202803D10120C00301900BE061
:105E24000748006838210840182803D17D20000263
:105E3400019001E000200190019807B000BDC04628
:105E4400081002400C10024000127A000024F400F2
:045E540000100240F8
:0C5E5800014800687047C0467406002036
:105E640000B581B0FFF7F6FF009000F00DF8014691
:105E74000098090B8A00034989581F221140C84021
:085E840001B000BD2433000849
:105E8C0002480068072109030840704708100240C7
:105E9C00034908680122D204104308607047C046C9
:045EAC0000100240A0
:105EB00000B581B00C4800680090009803210902E9
:105EC00008400A49086068464078C007002801D0A9
:105ED00009F07BF8684640788007002801D509F072
:105EE00075F801B000BDC0461C10024020100240F1
:105EF00000B587B0069003A90020087002A90870B9
:105F0000069880788007002800D487E001A9002047
:105F10000870A6480068C00000280CD4A348026896
:105F2000012109070A4302600068084000900098B8
:105F300001A9012008709E4908680122120210433D
:105F40000860FDF763FA049099480068C0050028CE
:105F50000AD4FDF75BFA0499401A032803D303A976
:105F60000320087000E0EFE703A80078002848D17C
:105F70009048006803210902084005900598002810
:105F800014D005980699096B88420FD08949086892
:105F90000322120290430590086801221204104364
:105FA00008600868904308600598086005A80078B4
:105FB000C007002813D0FDF729FA04907D48006837
:105FC000800700280BD4FDF721FA0499401A7A497A
:105FD000884203D303A90320087000E0EEE703A87A
:105FE0000078002809D173490868032212029043FF
:105FF000069A126B1043086002E0039802A9087029
:1060000002E0039802A9087001A80078012805D1D0
:1060100066490868012212079043086006980078D4
:10602000C007002807D06549086803229043069AF4
:10603000526810430860069800788007002807D54A
:106040005E4908680C229043069A926810430860E3
:1060500006980078C006002808D558490868032229
:1060600092029043069AD2681043086006984078DE
:106070008007002808D551490868032292049043FC
:10608000069A9269104308600698407840070028F5
:1060900008D54A490868032212059043069AD26936
:1060A00010430860069800788006002808D5434908
:1060B0000868032212039043069A1269104308608D
:1060C000069840784006002814D53C490868032209
:1060D00092079043069A126A104308600698006A75
:1060E00001218907884205D1354908680122120437
:1060F00010430860069880780007002807D52F49CC
:10610000086840229043069A526A10430860069835
:1061100080788006002812D5284A10680121890558
:106120008843069B9B6A184310600698806A8842E1
:1061300005D1234908680122120610430860069819
:1061400080784006002812D51C4A106801210906F3
:106150008843069BDB6A184310600698C06A884231
:1061600005D11749086801221206104308600698F5
:1061700040780007002814D51049086803229203CC
:106180009043069A526910430860069840690121BD
:106190008903884205D10A49086801221204104384
:1061A000086002A8007807B000BDC0463C1002405D
:1061B000007000405C10024089130000541002403F
:0461C0000C1002407D
:1061C40083B00290019102980068009002983349CC
:1061D400884208D0029801218907884203D0029896
:1061E4002F49884208D10098702188430090019873
:1061F400416800980843009002982849884218D0C2
:10620400029801218907884213D0029824498842C0
:106214000FD00298234988420BD002982249884221
:1062240007D002982149884203D002982049884225
:1062340009D1009803210902884300900198C1689C
:106244000098084300900098802188430199496987
:1062540008430090009802990860019880680299A8
:10626400C862019800680299886202980B498842C2
:106274000BD002980C49884207D002980B498842F7
:1062840003D002980A49884203D10198006902990F
:10629400086302990120486103B07047002C014053
:1062A4000004004000200040004001400044014040
:0462B400004801405D
:1062B80083B0019001983D21405C012803D002A9D8
:1062C8000120087036E001993D2202208854019887
:1062D80000681A4988420FD001980068012189078F
:1062E800884209D0019800681549884204D001986D
:1062F80000681449884214D10198006880681249DE
:1063080008400090009806280AD000980121090446
:10631800884205D001980168086801221043086086
:1063280005E001980168086801221043086002A985
:106338000020087002A8007803B07047002C0140C4
:0C6348000004004000400140070001007C
:1063540083B0019001983D21405C012803D002A93B
:10636400012008703CE001993D22022088540198E4
:106374000168C86801221043C860019800681A497E
:1063840088420FD00198006801218907884209D00A
:10639400019800681549884204D00198006814499E
:1063A400884214D10198006880681249084000901E
:1063B400009806280AD0009801210904884205D0D3
:1063C40001980168086801221043086005E00198FB
:1063D4000168086801221043086002A900200870BF
:1063E40002A8007803B07047002C0140000400406C
:0863F400004001400700010018
:1063FC0081B0009000980168C86801229043C86081
:10640C0000980068006A0B4908420BD1009800689C
:10641C00006A0949084205D1009801680868012200
:10642C009043086000993D2201208854002001B05F
:0C643C007047C04611110000440400002D
:1064480000B581B0009000980068006902210840FA
:106458004008002822D000980068C068022108403F
:10646800400800281AD0009801680220C04308613B
:106478000099012008770098006880698007002843
:1064880003D0009809F012FF05E0009809F012FF08
:10649800009809F013FF0099002008770098006819
:1064A8000069042108408008002823D0009800686B
:1064B800C06804210840800800281BD000980168A3
:1064C8000420C043086100990220087700980068FA
:1064D80080698005800F002803D0009809F0E6FE47
:1064E80005E0009809F0E6FE009809F0E7FE00993B
:1064F8000020087700980068006908210840C00853
:10650800002822D000980068C06808210840C00808
:1065180000281AD0009801680820C0430861009933
:106528000420087700980068C0698007002803D015
:10653800009809F0BBFE05E0009809F0BBFE009842
:1065480009F0BCFE009900200877009800680069EF
:10655800102108400009002823D000980068C0686E
:1065680010210840000900281BD00098016810205D
:10657800C043086100990820087700980068C0693E
:106588008005800F002803D0009809F08FFE05E0F1
:10659800009809F08FFE009809F090FE00990020FD
:1065A8000877009800680069C00700280DD0009897
:1065B8000068C068C007002807D00098016801205B
:1065C800C0430861009806F093F9009800680069D4
:1065D800C0B2C00900280ED000980068C068C0B2D8
:1065E800C009002807D0009801688020C0430861CE
:1065F800009809F0C1FE00980068006901210902AD
:106608000840000A00280DD000980068C068C0B291
:10661800C009002806D0009801681B480861009846
:1066280009F0AEFE00980068006940210840800922
:1066380000280FD000980068C068402108408009F1
:10664800002807D0009801684020C04308610098DE
:1066580009F038FE009800680069202108404009C8
:1066680000280FD000980068C06820210840400921
:10667800002807D0009801682020C04308610098CE
:0C66880009F076FE01B000BDFFFEFFFF30
:1066940000B585B00390029103983C21405C012829
:1066A40003D104A9022008709CE003993C22012034
:1066B400885403993D220220885403980068806816
:1066C400019001984949084001900198FF2109026D
:1066D40088430190019803990968886002980068CA
:1066E400009000286CD00098102869D000982028C9
:1066F40066D00098302863D00098402853D0009882
:10670400502836D00098602840D0009870280BD0CC
:10671400009801210903884205D00098012149030A
:10672400884216D053E052E003980068029B9968AF
:106734005A68DB6808F096FC03980068806801904A
:1067440001987721084301900198039909688860AA
:106754003DE003980068029B99685A68DB6808F07A
:1067640081FC0398016888680122920310438860C1
:106774002DE003980068029A5168D26809F0A8FDD8
:1067840003980068502100F033F820E00398006873
:10679400029A5168D26809F0C3FD03980068602129
:1067A40000F026F813E003980068029A5168D26852
:1067B40009F08EFD03980068402100F019F806E006
:1067C400039800680299096800F012F8FFE703993A
:1067D4003D220120885403993C220020885404A9B6
:1067E4000020087004A8007805B000BD88FFCEFF23
:1067F40083B0029001910298806800900098074944
:10680400084000900198009908430721084300902C
:1068140000980299886003B07047C0468FFFCFFF8D
:1068240085B00390029103983C21405C012803D178
:1068340004A90220087058E003993C2201208854DE
:1068440003993D220220885403980068406801900F
:10685400039800688068009003980068254988427E
:1068640009D101980F2109058843019002984168D4
:10687400019808430190019870218843019002987F
:1068840001680198084301900198039909684860D8
:1068940003980068174988420FD0039800680121C3
:1068A4008907884209D0039800681349884204D0B4
:1068B40003980068114988420CD1009880218843CC
:1068C400009002988168009808430090009803990A
:1068D4000968886003993D220120885403993C2269
:1068E4000020885404A90020087004A8007805B08A
:1068F4007047C046002C01400004004000400140A5
:1069040010B592B011900CA900200870119800687D
:10691400FD49884200D1FFE7119988680A6910434C
:106924004A691043C96908431090119800680068C7
:10693400F6490840109908431199096808601198AC
:10694400006840680321090388431199CA68104309
:106954000968486011988069109011980068EA49A4
:10696400884204D01198016A109808431090119835
:1069740000688068E649084010990843119909683D
:10698400886011980068C06A0F21884311994A6A87
:1069940010430968C86211980068DE49884227D10B
:1069A400DD48006803210840099003281CD8099891
:1069B400810001A040588746CD690008DD690008C0
:1069C400D5690008E56900080EA9002008700EE0EA
:1069D4000EA9022008700AE00EA90420087006E03F
:1069E4000EA90820087002E00EA91020087085E0A6
:1069F40011980068EC4988423AD1EE4800680C21AD
:106A0400084008900C282FD80898810001A040580D
:106A14008746C0464D6A00086D6A00086D6A000822
:106A24006D6A00085D6A00086D6A00086D6A0008F6
:106A34006D6A0008556A00086D6A00086D6A0008EE
:106A44006D6A0008656A00080EA9002008700EE04F
:106A54000EA9022008700AE00EA90420087006E0BE
:106A64000EA90820087002E00EA91020087045E065
:106A740011980068CD49884203D10EA900200870FE
:106A84003CE011980068CA49884203D10EA900204D
:106A9400087033E011980068C24988422BD1C54878
:106AA4000068032189020840079000280FD0079846
:106AB40001218902884212D007980121C902884223
:106AC40009D007980321890288420CD00FE00EA94F
:106AD400002008700EE00EA9022008700AE00EA93A
:106AE4000420087006E00EA90820087002E00EA930
:106AF4001020087002E00EA9102008701198006898
:106B0400A849884277D10EA800780690082826D88C
:106B14000698810001A040588746C046456B00088E
:106B2400636B00084D6B0008636B0008536B00082F
:106B3400636B0008636B0008636B00085B6B000801
:106B4400FFF78EF90A900FE09B480A900CE0FFF7DC
:106B5400FFF80A9008E00120C0030A9004E0002036
:106B64000A900CA9012008700A98002842D00A98BB
:106B74001199496A4A009149895A06F06FFD0B90B0
:106B84000B9811994A6803215143884205D30B9805
:106B9400119949680903884203D90CA90120087096
:106BA40028E00A9811990491496A4A0083498A5A4B
:106BB40000230593194606F075FD049A059B040EFF
:106BC400090209190002526854080019594106F0D3
:106BD40069FD0D900D98000A032808D30D98000D47
:106BE400002804D10D9811990968C86002E00CA925
:106BF40001200870C5E01198C0690121C9038842C9
:106C040061D10EA800780390082826D80398810043
:106C140001A040588746C046416C00085F6C0008DC
:106C2400496C00085F6C00084F6C00085F6C00083A
:106C34005F6C00085F6C0008576C0008FFF710F9E0
:106C44000A900FE05C480A900CE0FFF781F80A9084
:106C540008E00120C0030A9004E000200A900CA977
:106C6400012008700A9800282CD00A9811990291E2
:106C7400496A4A005149895A06F0F0FC02994000D9
:106C840049684A08801806F0E9FC80B20D900D9816
:106C9400102814D30DA84088002810D10D990F2076
:106CA40081430FA801800D990E2211404A080F99C3
:106CB40011430180008811990968C86002E00CA999
:106CC400012008705DE00EA800780190082830D8F3
:106CD4000198810001A040588746C046056D000810
:106CE400376D0008216D0008376D0008276D000816
:106CF400376D0008376D0008376D00082F6D0008E8
:106D0400FFF7AEF80A9019E000800040F369FFCF66
:106D1400FFF4FF11003801405410024026480A9045
:106D24000CE0FFF715F80A9008E00120C0030A9070
:106D340004E000200A900CA9012008700A98002899
:106D44001FD00A9811990091496A4A001B49895A2F
:106D540006F084FC009949684A08801806F07EFC15
:106D640080B20D900D98102808D30DA840880028F3
:106D740004D10D9811990968C86002E00CA901209A
:106D8400087011996A220120885211996822885248
:106D9400119900200867119948670CA8007812B06F
:106DA40010BDC04600800040004400400048004040
:106DB400004C0040541002400024F40080080108F4
:106DC40000B585B0039003998C2200208850FCF70D
:106DD4001BFB0290039800680068000700280ED58A
:106DE4000398029B1B49009101214905002208F0E8
:106DF400EFF9002803D004A90320087025E00398C4
:106E040000680068400700280ED50398029B1149CA
:106E1400009101218905002208F0DAF9002803D045
:106E240004A90320087010E00399842220208850CC
:106E340003998822885003990020C8660399802208
:106E44000020885404A90020087004A8007805B024
:086E540000BDC046FFFFFF0175
:106E5C008CB00490039102A80280049884214058BD
:106E6C00202800D09EE00398002803D002A80088B8
:106E7C00002803D105A90120087096E004988068C9
:106E8C000121090388420CD104980069002808D11B
:106E9C0003A80078C007002803D005A901200870BA
:106EAC0083E004988021405C012803D105A90220CD
:106EBC0008707AE004998022012088540398049980
:106ECC000865029804995422885202980499562213
:106EDC00885204990020486704998C2288500499A0
:106EEC008422212088500498406E01214907884251
:106EFC002AD10498806801210903884207D104989B
:106F0C000069002803D104992D48486702E00499D0
:106F1C002A4848670499802200208854EFF3108097
:106F2C0007900798019001220B920B9880F3108820
:106F3C00049801688868D2051043886001980A900B
:106F4C000A9880F3108829E00498806801210903CD
:106F5C00884207D104980069002803D10499164887
:106F6C00486702E00499134848670499802200207E
:106F7C008854EFF310800690069800900120099039
:106F8C00099880F3108804980168086880221043DF
:106F9C00086000980890089880F3108805A90020D4
:106FAC00087002E005A90220087005A800780CB052
:106FBC007047C0463FF30008997000089103010820
:046FCC00D16F000879
:106FD0008BB00490049884214058212857D10498FC
:106FE0006A21405A02A9088002A8008800284ED0D1
:106FF00004985621405A00282AD1EFF310800690B9
:107000000698019001220A920A9880F31088049849
:1070100001688868D20590438860019809900998B2
:1070200080F31088EFF31080059005980090012000
:107030000890089880F31088049801680868402236
:107040001043086000980790079880F310881EE0AE
:1070500004980068C0690006002813D50498006DE4
:107060000390039800880B490840049909688862D6
:107070000499086D801C086504995622885A401EA0
:107080008852FFE70298401E02A90880ACE70BB0C7
:087090007047C046FF0100003B
:107098008AB00390039884214058212842D103984C
:1070A8005621405A00282AD1EFF310800590059800
:1070B800019001200990099880F3108803980168CD
:1070C800086880229043086001980890089880F327
:1070D8001088EFF310800490049800900120079026
:1070E800079880F3108803980168086840221043C5
:1070F800086000980690069880F3108812E00398BC
:10710800006D0290029800880749084003990968B1
:1071180088620399086D801C086503995622885A6D
:0C712800401E88520AB07047FF010000B2
:1071340000B589B00490039102A8028004988821C4
:107144004058202856D10398002803D002A800886C
:10715400002803D105A9012008704EE00498806836
:107164000121090388420CD104980069002808D140
:1071740003A80078C007002803D005A901200870DF
:107184003BE004988021405C012803D105A902203A
:10719400087032E004998022012088540499002068
:1071A400C86604980068174988421AD00498006891
:1071B40040680002002814D5EFF31080069006986A
:1071C400019001220892089880F3108804980168BD
:1071D400086892061043086001980790079880F3A6
:1071E40010880498039902AA128800F00DF805A9E2
:1071F400087002E005A90220087005A8007809B00B
:0872040000BDC04600800040FF
:10720C0093B00690059104A80280059806998865AC
:10721C00049806995C228852049806995E2288523A
:10722C0006990020086706988068012109038842A6
:10723C000DD106980069002804D106996022644893
:10724C00885203E006996022FF20885229E00698B4
:10725C00806800280DD106980069002804D1069991
:10726C006022FF20885203E0069960227F2088521A
:10727C0017E0069880680121090788420DD106980D
:10728C000069002804D1069960227F20885203E00F
:10729C00069960223F20885203E006996022002064
:1072AC00885206998C220020885006998822222028
:1072BC008850EFF310800A900A98039001221292E2
:1072CC00129880F3108806980168886810438860CB
:1072DC0003981190119880F310880698406E012144
:1072EC004907884246D104A8008806996822895A21
:1072FC0088423FDB0698806801210903884207D148
:10730C0006980069002803D106993548086702E001
:10731C000699324808670699802200208854EFF3BA
:10732C00108009900998029001221092109880F315
:10733C0010880698016808681202104308600298C9
:10734C000F900F9880F31088EFF310800890089836
:10735C00019001220E920E9880F310880698016815
:10736C00886812071043886001980D900D9880F37F
:10737C0010882AE00698806801210903884207D109
:10738C0006980069002803D106991348086702E0A3
:10739C000699104808670699802200208854EFF35C
:1073AC00108007900798009001200C900C9880F3A7
:1073BC001088069801680868092252011043086079
:1073CC0000980B900B9880F31088002013B0704736
:1073DC00FF010000F3F40008CDF3000881760008EB
:0473EC00F173000831
:1073F00000B59FB00F900F986021405A0DA90880EA
:107400000F980068C06909900F980068006808909C
:107410000F980068806807900F98882140582228AC
:1074200000D020E10F986821405A0BA908800BA8D2
:10743000018800200029019005D009A800782021AA
:107440000840400901900198C007002800D1CDE014
:107450000F980068406A0CA908800F98806D0E9004
:107460000C980D9908400E9908800F99886D801C22
:1074700088650F995E22885A401E88520F980068CE
:10748000C069099009A800784007002846D009A8DB
:107490000078C00700280DD008A84078C007002851
:1074A00008D00F980068012303620F998C22885836
:1074B0001843885009A80078800700280ED507A82F
:1074C0000078C007002809D00F98016802200862E0
:1074D0000F998C22885804231843885009A80078F3
:1074E000400700280ED507A80078C007002809D05B
:1074F0000F980168042008620F998C228858022393
:10750000184388500F988C214058002806D00F98B7
:1075100008F09AFF0F998C22002088500F985E2166
:10752000405A002861D1EFF310801490149806900F
:1075300001221E921E9880F310880F980168086837
:1075400012029043086006981D901D9880F31088E1
:10755000EFF3108013901398059001201C901C9855
:1075600080F310880F9801688868444A104088604A
:1075700005981B901B9880F310880F998822202073
:1075800088500F99002008670F98C06E012829D1F4
:107590000F990020C866EFF31080129012980490A3
:1075A00001201A901A9880F310880F9801680868D3
:1075B00010229043086004981990199880F310885D
:1075C0000F980068C069102108400009012803D104
:1075D0000F980168102008620F985C21415A08F04A
:1075E00037FF02E00F9808F03DFF20E70F985E217B
:1075F000415A0AA801800088002833D00AA80088D0
:107600000F996822895A88422CDAEFF31080119082
:107610001198039001221892189880F310880F98FF
:10762000016888681207904388600398179017983C
:1076300080F310880F9910480867EFF310801090BE
:107640001098029001201690169880F310880F98D9
:107650000168086820221043086002981590159868
:1076600080F3108805E00F980168886908221043AC
:1076700088611FB000BDC046CDF30008FEFFFFEFDC
:1076800000B59DB00D900D986021405A0CA908805E
:107690000D980068C06908900D9800680068079010
:1076A0000D980068806806900D988821405822281F
:1076B00000D01EE10D986821405A0AA908800AA846
:1076C000018800200029009005D008A8007820211A
:1076D0000840400900900098C007002800D1CBE086
:1076E0000D980068406A0BA908800B980C99084017
:1076F0000D99896D08700D99886D401C88650D99EC
:107700005E22885A401E88520D980068C069089011
:1077100008A800784007002846D008A80078C007CD
:1077200000280DD007A84078C007002808D00D9881
:107730000068012303620D998C22885818438850F1
:1077400008A80078800700280ED506A80078C00792
:10775000002809D00D980168022008620D998C223A
:10776000885804231843885008A800784007002848
:107770000ED506A80078C007002809D00D9801682A
:10778000042008620D998C228858022318438850DF
:107790000D988C214058002806D00D9808F054FE12
:1077A0000D998C22002088500D985E21405A0028A7
:1077B00061D1EFF3108012901298059001221C9273
:1077C0001C9880F310880D98016808681202904395
:1077D000086005981B901B9880F31088EFF31080C9
:1077E00011901198049001201A901A9880F3108833
:1077F0000D9801688868444A104088600498199080
:10780000199880F310880D998822202088500D99AE
:10781000002008670D98C06E012829D10D9900201D
:10782000C866EFF310801090109803900120189014
:10783000189880F310880D9801680868102290430A
:10784000086003981790179880F310880D980068C7
:10785000C069102108400009012803D10D98016872
:10786000102008620D985C21415A08F0F1FD02E0F9
:107870000D9808F0F7FD22E70D985E21415A09A8FE
:1078800001800088002833D009A800880D9968225B
:10789000895A88422CDAEFF310800F900F980290EB
:1078A00001221692169880F310880D980168886856
:1078B00012079043886002981590159880F31088FD
:1078C0000D9910480867EFF310800E900E98019004
:1078D00001201490149880F310880D9801680868AE
:1078E00020221043086001981390139880F31088A9
:1078F00005E00D98016888690822104388611DB071
:0C79000000BDC046F3F40008FEFFFFEFDE
:10790C0000B587B005900491039202930598002866
:10791C0003D106A90120087052E005988421405833
:10792C00002806D10599802200208854059805F07E
:10793C00F7FA059984222420885005980168086874
:10794C000122904308600598FEF7D6FF012803D169
:10795C0006A90120087033E00598806A002802D03F
:10796C00059807F096FB0598016888680122930337
:10797C0018438860059800688068D103884304998F
:10798C00084305990968886003984005019002989E
:10799C0001040198084301900598006800680A49A1
:1079AC000840019908430599096808600598016821
:1079BC000868104308600598FFF7FEF906A90870DF
:0C79CC0006A8007807B000BDFFFF00FC1B
:1079D80070B58AB009900998406E002807D10999B6
:1079E8006A220120885209996822885232E008A93F
:1079F80001910820087007A9087009980068806834
:107A0800072252061040400E06AA029210700998EA
:107A180000688068420F05A80270097802780E484D
:107A28000490805C48430D490391895C05F014FE7D
:107A3800019B029A039904460498099D6A26AC534F
:107A48001B781278805C5843895C05F005FE09991B
:107A5800682288520AB070BD5F11010867110108D9
:107A680070B5FFB0FFB098B0FFAB283305930B4655
:107A780005990693034606980B63C8628A6209A8AB
:107A88000861012080024861002088610A6B0A624F
:107A9800C861059AD06A0178FFA84C300170D16A94
:107AA800491CD1620078002800D17EE1FFA84C3043
:107AB8000078252800D06CE1059900204860012055
:107AC800C8600598C06A0178FFA84C30017000783A
:107AD800233804900D2845D80498810001A0405807
:107AE8008746C0465B7B00086D7B00086D7B0008FD
:107AF8006D7B00086D7B00086D7B00086D7B0008BE
:107B08006D7B0008497B00086D7B0008257B000819
:107B18006D7B00086D7B0008377B00080599486875
:107B2800012210434860C86A401CC8621DE00599DC
:107B38004868022210434860C86A401CC86214E0C2
:107B480005994868042210434860C86A401CC86206
:107B58000BE005994868082210434860C86A401C31
:107B6800C86202E005990020C8600598C06800282E
:107B7800A7D10599002008600598C06A0178FFA878
:107B88004C3001700078302804DBFFA84C300078B6
:107B98003A2800DB0FE00599C86A401CC8620868EB
:107BA8000A224243FFA84C30007880183038086019
:107BB80001200028E0D1059800218160C06A017881
:107BC800FFA84C30017000782E2822D10599C86A88
:107BD800401CC8620598C06A0178FFA84C30017043
:107BE8000078302804DBFFA84C3000783A2800DB06
:107BF8000FE00599C86A401CC86288680A22424397
:107C0800FFA84C30007880183038886001200028A0
:107C1800E0D10598C06A0078FFA94C310870FFA828
:107C28004C3000786C2804D0FFA84C3000786828C5
:107C380009D10598C16A491CC162C06A0078FFA9C8
:107C48004C31087000E002E001200028E7D1FFA8CD
:107C58004C3000780390252800D18FE003985828ED
:107C680048D0039863280FD0039864281CD0039841
:107C7800702871D0039873284FD00398752826D0A0
:107C88000398782836D07FE00598836A19680A1D1A
:107C98001A600968C160C16808A801700178FFA866
:107CA800383008F015FC6FE0059A936A1868011DD2
:107CB80019600068D060D1689368106852680192B2
:107CC8000090FFA838300A2207F022FD5CE0059AF0
:107CD800936A1868011D19600068D060D1689368BC
:107CE8001068526801920090FFA838300A2200F00C
:107CF80075F849E0059A936A1868011D19600068CB
:107D0800D060D16893681068526801920090FFA80B
:107D18003830102200F062F836E00598826A106860
:107D2800011D11600068079007980178FFA84C3082
:107D380001700799491C07910078002800D10AE0D2
:107D4800FFA84C300178FFA8383008F0C1FB05982F
:107D5800C0690028E8D517E00598836A19680A1DE4
:107D68001A600968C160C168002001900823009367
:107D7800FFA83830102200F031F805E0FFA83830AD
:107D8800252108F0A5FBFFE70599C86A401CC862D1
:107D980006E0FFA84C300178FFA8383008F098FBBF
:107DA8000598C069002800D473E60598C0690128C1
:107DB8000EDB05988069002805D00599086B8A694B
:107DC80009A906F049FD05998A69C8698018C8613A
:0C7DD8000598C0697FB07FB018B070BD86
:107DE40010B590B0139C129C0F900E910D920C93B1
:107DF4000E98099001200A90089009980D998842DC
:107E040008D309980D9905F029FC09900898401C9D
:107E14000890F2E70C980899884201D90C980890C8
:107E240013A80078C007002834D11298002831D054
:107E340013A800788007002806D50C98002803D1E1
:107E440007A93020087002E007A9202008701299C1
:107E54000020002906900BD00899129A01200023D3
:107E640004939142059001D30498059005980690D7
:107E74000698C00700280DD01298401E12900F9843
:107E840007A9097808F026FB0F98C068002800D5D8
:107E940000E0DCE70F98C06800285DD40C98022845
:107EA40003D30C98401E0C9009E00E980A9905F033
:107EB400D5FB0B900B980D99884200D204E00D98E5
:107EC4000A9948430A90E9E70E980A9905F0C6FB17
:107ED4000B900B980A9941430E98401A0E900F98F4
:107EE4000B9A1E49895C08F0F5FA0F98C0680028BF
:107EF40000D507E00D990A9805F0B0FB0A900A989E
:107F04000028E1D113A80078C007002824D01298D3
:107F1400002821D012990020002903900BD0089941
:107F2400129A0120002301939142029001D30198F7
:107F34000290029803900398C00700280CD012986E
:107F4400401E12900F98202108F0C4FA0F98C068C0
:107F5400002800D500E0DDE710B010BD6F11010866
:107F640010B586B0002101910591049103913A481E
:107F740002903A4A0260012293074360031D816024
:107F8400C160540504610824446101764176827617
:107F94000624C4611977416281622C23C2541303FD
:107FA40003634263022282633C228154C164FBF76F
:107FB40073FA002801D002F0E1FF012003900020B1
:107FC400049027480590244803A9FBF73DFD0028A9
:107FD40001D002F0D3FF2348039004200490002032
:107FE40005901D4803A9FBF72FFD002801D002F0DE
:107FF400C5FF1D48039008200490174803A9FBF708
:1080040023FD002801D002F0B9FF184803900C208A
:108014000490114803A9FBF717FD002801D002F0D2
:10802400ADFF13480390102004900B4803A9FBF7FD
:108034000BFD002801D002F0A1FF0E48039014208C
:108044000490054803A9FBF7FFFC002801D002F0C7
:1080540095FF06B010BDC0469807002000240140DB
:1080640004FFFF0702000004040000080800000CDD
:088074008000001C4000001810
:10807C0010B59AB019900020189017901690159082
:10808C00149007A8342105F095FB199800682D4928
:10809C00884255D101208003079000200F9007A83B
:1080AC00FDF720FF002801D002F064FF264802688B
:1080BC00012109050A4302600068084006900698F1
:1080CC002248026801210A430260006808400590BA
:1080DC000598CF2014900320039015900020029057
:1080EC00169005200190000714A9FCF7EDFF019BE9
:1080FC00029A039916480490164C046043608260FF
:10810C00C2608022026101221302436192028261E9
:10811C002022C26109030162FCF744FC002801D053
:10812C0002F028FF19980A490165199888620C20F9
:10813C0000900022114608F011F8009806F024FE79
:10814C001AB010BD0024014040100240341002400F
:08815C00901000200800024011
:1081640000B581B00B4800900B49016001210171F9
:108174004171072282601022C260002202614261C2
:1081840082610162FCF7B0FA002801D002F0F6FE29
:0C81940001B000BD0013002000300240CC
:1081A00082B00190019800680749884209D10748C8
:1081B0000268012109030A43026000680840009038
:1081C000009802B07047C0460030024038100240AC
:1081D00000B589B06846242105F0F2FA104811492B
:1081E000016006F0EDFD002801D002F0C9FE00227A
:1081F0000092019202920392049209486946FCF7A8
:10820000D7FA002801D002F0BBFE054869461022CB
:10821000FCF7CEFA002801D002F0B2FE09B000BD92
:0882200040130020007400402F
:1082280000B58BB00A90002009900890079006903E
:1082380005900A9800681749884228D116480268AC
:10824800012149070A430260006808400490049825
:108258001248026801210A4302600068084003903E
:10826800039830200590032000900690002001908C
:1082780007900520000705A9FCF728FF0099019A37
:108288001120029007F06CFF029806F07FFD0BB0FA
:1082980000BDC046007400403C100240341002404B
:1082A80000B583B01748026801210A4302600068DC
:1082B8000840029002981448019014490160002176
:1082C80041600122930383604023C36080230361DC
:1082D80053024361D2028261C16103210903016231
:1082E800FCF762FB002801D002F046FE092000904E
:1082F8000121002207F034FF009806F047FD03B083
:1083080000BDC04638100240341000201C00024056
:0883180000487047EE07000069
:1083200085B00390029101920398019940180D497C
:10833000884202D30120049010E0002000900098B1
:108340000199884208D20398009A805C0299885467
:108350000098401C0090F2E700200490049805B0BB
:088360007047C046010002084D
:1083680000B589B0FCF7F0FD00284DD12E4A116800
:108378000120430299431160022104912B49097895
:108388004908891E0691079004A803A9FCF714FE62
:10839800002827D1264802900020019002982549FC
:1083A80088421ED802990198C300234AD018D2588F
:1083B80043680120FCF718FD002806D10298083010
:1083C80002900198401C01900AE0174908680122B0
:1083D800520210430860FCF7D9FD032008901FE003
:1083E800DCE70AE0104908680122520210430860DD
:1083F800FCF7CCFD0220089012E00B490868012226
:1084080052021043086002E00120089008E0FCF7DF
:10841800BDFD002802D00420089001E0002008904B
:10842800089809B000BDC04600200240E075FF1F53
:0C84380000F0010837F0010848070020A0
:1084440000B583B00190644964483822FFF766FFA1
:10845400002802D001200290BAE05F480090009901
:108464000A784878000280188A78C97809028A183C
:1084740001990A83C8820098017940790002401862
:108484000199488300988179C079000240180199C4
:1084940088830098017A407A000240180199C883C1
:1084A4000098817AC07A00024018019908850098E2
:1084B400017B407B00024018019948870098817C29
:1084C400C07C00024018019988870098017D407D96
:1084D400000240180199C8870098817DC07D000280
:1084E40040180199422288520098017E407E000281
:1084F40040180199442288520098817EC07E00026F
:1085040040180199462288520098017F407F00025A
:1085140040180199482288520098817FC07F000248
:10852400401801994A2288520098817BC07B00023E
:10853400401801994C2288520098017C407C00022A
:10854400401801994E228852009908462030202272
:10855400895C407800024118214801800088002885
:1085640003D00199502201208852009801463031ED
:108574003022825C4878000280188A78C97809021F
:108584008A1801994A810881009908462C302C22C6
:10859400895C407800024018382802D002200290FA
:1085A40016E0009908462E302E22895C407800029D
:1085B4004018002802D00320029009E000982421EA
:1085C400405C652802D00420029001E00020029063
:1085D400029803B000BDC0464807002000F001081F
:0485E400EA15002074
:1085E80070B584B0029001A801705C490091029AAC
:1085F800138B1904D48A009A1470240A54701B0A25
:10860800D370090C91700299498B009A1171090A6B
:1086180051710299898B009A9171090AD171029955
:10862800C98B009A1172090A51720299098D009A30
:108638009172090AD1720299498F009A1173090A35
:1086480051730299898F009A9174090AD174029919
:10865800C98F009A1175090A517502994222895ADF
:10866800009A9175090AD17502994422895A009A8B
:108678001176090A517602994622895A009A91760A
:10868800090AD17602994822895A009A1177090A6B
:10869800517702994A22895A009A9177090AD17723
:1086A80002995622895A009B1A46203220241955CD
:1086B800090A517002994C22895A009A9173090A41
:1086C800D17302994E22895A009A1174090A517479
:1086D800009B1A46283228241D5D517809024D193D
:1086E8009678D1780902891909044919491C19553C
:1086F8000B0ED3700B0C9370090A5170009B1A462D
:108708002C322C243821195500215170009B1A460F
:108718002E322E2419555170009A24236521D154E4
:10872800007800280ED002994A8910040B89009C11
:1087380021463031302563551B0A4B70120ACA7026
:10874800000C8870FFF70CFE002802D0012003906F
:1087580001E000200390039804B070BD4807002092
:1087680070B584B01D48029002981D4924220192D8
:1087780005F01AF8019A029B1946283128241D5D34
:108788004878000245198E78C878000280190004DC
:108798004019401C1855030ECB70030C8B70000A4F
:1087A8004870029B19462C312C243820185500207B
:1087B8004870029B19462E312E241855487002998C
:1087C80065208854FFF7CCFD002802D002200390D2
:1087D80001E000200390039804B070BD4807002012
:0487E800D0E80008CD
:1087EC0000B583B00A4801A90122FFF793FD0028C8
:1087FC0002D00120029008E001A80078652802D080
:10880C000120029001E000200290029803B000BD0C
:04881C0024F001083B
:1088200000B589B0FCF794FB00284DD12E4A1168A1
:108830000120430299431160022104912B490978D8
:108840004908491E0691079004A803A9FCF7B8FB44
:10885000002827D12648029000200190029825493F
:1088600088421ED802990198C300234AD018D258D2
:1088700043680120FCF7BCFA002806D102980830B2
:1088800002900198401C01900AE0174908680122F3
:10889000520210430860FCF77DFB032008901FE0A4
:1088A000DCE70AE010490868012252021043086020
:1088B000FCF770FB0220089012E00B4908680122C7
:1088C00052021043086002E00120089008E0FCF723
:1088D00061FB002802D00420089001E000200890ED
:1088E000089809B000BDC04600200240E075FF1F97
:0C88F00000F8010811F8010880070020C2
:1088FC0000B583B015480190019900200090487094
:10890C0008700199C87088700199487108710199B3
:10891C00C87188710199487208720199C87288727D
:10892C000199487308730199C87388730199487445
:10893C000874FFF76FFF002802D00220029001E0BC
:10894C0000200290029803B000BDC04680070020B2
:10895C0000B583B00190314931481822FFF7DAFC99
:10896C00002802D00120029054E02C48009000987E
:10897C0001784078000240180199012212028852B5
:10898C0000988178C0780002401801998122520029
:10899C0088520098017940790002401801994122CF
:1089AC009200885200988179C07900024018019990
:1089BC001122120188520098017A407A0002401864
:1089CC0001998322520088520098817AC07A000261
:1089DC00401801992122D20088520098017B407BDB
:1089EC000002401801998522520088520098817B20
:1089FC00C07B0002401801994322920088520098D3
:108A0C00017C407C00024018019987225200885258
:108A1C0000200290029803B000BDC04680070020E1
:048A2C0000F8010845
:108A300000B583B001902B480090019801210902F4
:108A4000405A00990870000A487001988121490035
:108A5000405A00998870000AC87001984121890025
:108A6000405A00990871000A4871019811210901C2
:108A7000405A00998871000AC87101988321490001
:108A8000405A00990872000A487201982121C900D1
:108A9000405A00998872000AC872019885214900DD
:108AA000405A00990873000A4873019843218900CD
:108AB000405A00998873000AC873019887214900B9
:108AC000405A00990874000A4874FFF7A9FE00286C
:108AD00002D00220029001E000200290029803B030
:088AE00000BDC0468007002024
:108AE80070B592B00020119010900F900E900D90DC
:108AF8005448026804210A430260006808400C9048
:108B08000C985048026820210A4302600068084017
:108B18000B900B984B48026801210A4302600068D9
:108B280008400A900A984748026802210A430260EE
:108B380000680840099009984248026808210A43D9
:108B480002600068084008900898012205925103C5
:108B58003D48029007F084FB02980599890300229A
:108B6800049207F07DFB049A384801901F2631468D
:108B780007F076FB049A364806900224214607F04F
:108B88006FFB02980499059A03235B030D930E92D9
:108B98000F9110910DA90791FCF798FA0298049A81
:108BA800059B0799DD030D950E920F92FCF78EFA3F
:108BB8000198049A059B07990D960E930F921092AF
:108BC800FCF784FA0198049B059A0799FF26360258
:108BD8000D960E930F92FCF779FA049807990922DB
:108BE80012020D920E900F90052000070390FCF7DB
:108BF8006DFA0298049B059A0799C0260D960E9364
:108C08000F92FCF763FA0398049B059A07990D9550
:108C18000E930F92FCF75AFA049A059B0698079947
:108C28000D940E930F921092FCF750FA049B059A3C
:108C3800069807990C240D940E930F92FCF746FAA8
:108C480012B070BD341002400008005000040050FB
:048C5800000C0050BC
:108C5C0000B583B0029001910B490020009005F003
:108C6C0013FE0098029905F00FFE0098074905F0D5
:108C7C000BFE0098019905F007FE0098044905F0D9
:108C8C0003FE03B000BDC0467F11010845EB000890
:048C9C00930B01082D
:108CA00000B583B0029001910B490020009005F0BF
:108CB000F1FD0098029905F0EDFD0098074905F0D7
:108CC000E9FD0098019905F0E5FD0098044905F0DB
:108CD000E1FD03B000BDC0468711010845EB000867
:048CE000930B0108E9
:108CE40000B583B0029001910B490020009005F07B
:108CF400CFFD0098029905F0CBFD0098074905F0D7
:108D0400C7FD0098019905F0C3FD0098044905F0DA
:108D1400BFFD03B000BDC0468F11010845EB00083C
:048D2400930B0108A4
:108D280000B59BB000201A903F4802680121C9068F
:108D38000A43026000680840199019983B4908687E
:108D48003122104308603A4908680F22D2031043C1
:108D58000860384901200860002017901690FAF73B
:108D6800EDFA06F0B4FDFFF7BBFEFFF799FAFFF73F
:108D7800F5F804F099F8FFF7F1F9FFF725FA03F091
:108D8800ABFF00F0A3FC03F087FF03F031FF03F013
:108D980007FF03F0DDFE03F0A5FE03F043FF00F03C
:108DA8009DFC2548FDF784FA002803D02348244970
:108DB800FFF794FF2349002006F071FD1F48224960
:108DC800FFF748FF21480068214908402149401819
:108DD8001290112854D81298810001A04058874653
:108DE800758E0008898E0008898E0008898E000813
:108DF800898E0008898E0008898E0008898E0008EF
:108E0800898E0008898E00086B8E0008898E0008FC
:108E1800898E0008898E0008898E0008898E0008CE
:108E28007F8E0008618E00083C10024008580140FF
:108E38000C580140FC13002084110020AF0E0108DB
:108E4800B40E0108C90E0108CE0E010800580140F1
:108E5800FF0F0000AAFBFFFFFB48FC49FFF7FAFEE3
:108E680012E0F948FA49FFF7F5FE0DE0F648F9492E
:108E7800FFF7F0FE08E0F448F749FFF7EBFE03E0E0
:108E8800F148F649FFF7E6FEFE480068030CFE4984
:108E9800FB4A0020119006F002FD06F015FD02467F
:108EA8001198FA4906F0FBFCFFF732FA02461198CE
:108EB800F74906F0F4FC1198F649962206F0EFFC03
:108EC800FCF744FF02461198F34906F0E8FCFCF76A
:108ED8003DFFF24988420AD8E9481090F049FFF767
:108EE800FDFE1098EF49FFF7F9FE07F047F900F08B
:108EF8000DFC00F03DFCFFF775FC002807D0E048AA
:108F0800E949FFF7C9FEFFF72BFCFFF7F3FCE74839
:108F1800FFF794FA002803D0D948E549FFF7DEFEA9
:108F2800E248FFF717FD002803D0D548E149FFF7CD
:108F3800D5FEDE480F9001210B02C25A521CC252C4
:108F4800DD4A11604621425A4A21415A5143DB4ABF
:108F58001160C18F6E204843642104F07DFB0146F7
:108F68000F9840228152C08BD549022206F0F4FCAA
:108F78000F98408B65280ED1CC48C18A008B00041D
:108F88004118D0480190D0480090D048D04B0022DA
:108F980007F0D2FA20E0C548408B6F280ED1C348AD
:108FA800C18A008B00044118C6480190C648009049
:108FB800C648C74B012207F0BFFA0DE0BB48C18A7B
:108FC800008B00044118BF480190BF480090BF487B
:108FD800BF4B022207F0B0FABE4805F035FE002864
:108FE80018D1BC48FBF768FA00280ED1B94807F039
:108FF800ADF8159015983F2108430090B649B74A37
:109008009F4B002006F04BFC03E09D48B449FFF756
:1090180065FE03E09A48B349FFF760FEB2480C903A
:1090280000210E9105F0EBFE01460C9814911021D9
:1090380005F0E5FE01460E981391149BAB49904A42
:109048000D9206F02CFC0D9A0E98139BA84906F079
:1090580026FC012000F0CAFB9E48A6490622FAF722
:1090680065FC002803D08648A349FFF737FEA349CB
:1090780008680422904308609B480B9000210A91DD
:1090880007F086F80B981021099107F081F80A9BE0
:109098000B9819461A4607F0C5F809990A9B0B98C8
:1090A8001A4607F0BFF800F027FC95499548086074
:1090B800954A96491160964908609649086096490C
:1090C80008609649086096499648086000F034FFA1
:1090D8007E4807F0F3FA002810D07C4803F0AAF97C
:1090E800022807D190480068002802D0774807F086
:1090F800EDFA03E076498822222088506B485421F3
:10910800405A8A490988884206D168495222012072
:1091180088526C49088005E0644952220020885230
:109128006849088082480068002800D196E15F48B5
:10913800008C002800D190E164482621405C00287A
:1091480000D08AE15948008C089001283AD0089844
:10915800022852D00898032800D1FBE00898052877
:1091680044D008980A2800D111E10898142800D1A1
:1091780010E108981E2800D110E108987D21890087
:10918800884200D121E108986A49884200D142E129
:1091980008986949884200D12BE1089867498842B4
:1091A80000D13CE108986649884200D118E1089846
:1091B8006449884200D1F4E008986349884200D1A4
:1091C80020E130E139480021FFF70AFA002803D0EE
:1091D8002B485E49FFF782FD3448FFF72FF9002836
:1091E80003D027483249FFF779FD33E1244858492D
:1091F800FFF730FD01F0E8FE2CE12C48408B652894
:109208000ED12A48C18A008B000441182D480190CC
:109218002D4800902D482E4B002207F08DF92DE0A7
:109228002248408B6F281BD12048C18A008B00043C
:10923800411824480190244800902448244B0122D6
:1092480007F07AF91AE0C046AF0E0108950B01083D
:10925800B70B0108D90B0108FB0B010859EB0008F3
:10926800F348C18A008B00044118F5480190F5487D
:109278000090F548F54B022207F05EF9EAE0C04697
:10928800AF0E010800580140971101081D0C010894
:10929800B3110108530C0108DF0E0108FF8FD0033A
:1092A800E711010898080108FF110108C8140020F7
:1092B800F00E0108AB080108B41300206406002072
:1092C80000040050EC150020B8060020C00C002057
:1092D800A40F0020980700201D0F01082B12010879
:1092E800DA0801083E0F0108401300204F0F01085B
:1092F8007C0F0108DE150020750C010808000240EB
:10930800441400203903002048140020599E000806
:1093180040140020841400207414002098140020A5
:109328004C140020D59E00087C060020EA15002079
:10933800FC130020504F0000F9750000C5760000AE
:109348006E9D0000E3C4000058EC0000230E0108E5
:10935800D50A0108FFF704FA002803D0B348C64924
:10936800FFF7BCFCFFF7C6FAB148FFF767F800281B
:1093780003D0AE48AF49FFF7B1FCAD48FFF7EAFAB2
:10938800002803D0A948AC49FFF7A8FC62E002F026
:1093980035FC5FE0002000F029FA5BE002F0CAFB30
:1093A80058E0A3480121FFF71BF9002803D09F4884
:1093B800B049FFF793FC9E48FFF740F8002803D018
:1093C8009A489C49FFF78AFC44E0A1490A680020B2
:1093D8009060096848619649EA22885202F088FD3F
:1093E8009E4800689B49884202D19C49A048086071
:1093F80030E09A4800689749884202D197499B48CB
:10940800086027E0954800689249884202D193494C
:10941800954808601EE092498E4808601AE0904915
:109428009048086016E0954802680121C943116117
:10943800026800215162FCF789FF002803D07B48AD
:109448008F49FFF74BFC78490020086077488D4921
:10945800FFF722FC76490020088402E074490020C6
:10946800088400F02BFEF9F7CDFF1890189817998B
:10947800884200D12AE618981790784800688047F3
:1094880000F05CFE804907910868400008600520EC
:1094980000070121890305F07DFD02460798016850
:1094A800114301600068002802D0189800F062FE9D
:1094B800189801F04BF8189801F03EFC1898169986
:1094C800401A724988420FD3189816905748704925
:1094D800FFF7C0FB59480068002805D05448FFF73B
:1094E800A3FA5649002008605148808D069000284C
:1094F80006D00698012804D0069802282FD091E0BB
:1095080090E064480068012811D10920059005F011
:1095180048FC0598694A6A491160454AEA230021CE
:10952800D15205F033FC4C496648086016E05B48A8
:109538000068012803D148495F4808600EE0584890
:109548000068012803D144495A48086006E0554894
:109558000068012802D140495548086062E04D483A
:109568000068012803D04C480068012823D14F48DF
:10957800006800281ED10920049005F012FC049808
:109588004E4A4F4911602A4AEA230021D15205F078
:10959800FDFB40480068012802D12F49494808606E
:1095A8003D480068012802D12B49474808603F49D7
:1095B8000120086036E03948006801280AD13B4894
:1095C8000068002805D124493B4808603749012034
:1095D800086027E03248006801280AD1334800684B
:1095E800002805D11C49334808603049012008602B
:1095F80018E02C48006801280AD12C480068002887
:1096080005D115492A48086028490120086009E061
:1096180025480268189825490391096890470399D5
:109628000020086052E5C046FC130020AF0E010878
:10963800C8140020F00E0108AB080108B41300207C
:10964800EC150020B8060020C00C0020A40F002054
:1096580040130020390300207414002098140020BF
:109668004C140020D59E000889BC000895BD000850
:1096780079BE000887130108EC0A0108D011002000
:10968800AB130108BF10010858060020C1D401001F
:10969800A90F0108FC070020D8130020C8130020D8
:1096A800CC130020C4130020AC140020D4130020D5
:1096B800C1AE000861AE000825AE00082C140020D9
:1096C80001000020EDAD000821AF000808B4024BEE
:0C96D8009C4608BC6047C04639030020D7
:1096E40000B581B0094800908B21490004F066F868
:1096F4000099C92008800120488000208880C88003
:109704000884F622885201B000BDC046C814002067
:1097140000B587B01648039001220192114606F065
:10972400A1FD019A03980221029106F09BFD019A82
:1097340003980421049106F095FD7D200690C00055
:10974400F9F768FE019903980022059206F08AFD54
:1097540002990398059A06F085FD03980499059AE1
:1097640006F080FD06988000F9F754FE07B000BDAE
:04977400000400509D
:1097780000B583B015480068029015480190029919
:10978800019A1448302305F049FB002804D01248F8
:109798001549FFF7A3FAFEE70F481049FFF75AFAF1
:1097A8000C487D21CA000021FBF748FA002804D0A4
:1097B80009480C49FFF792FAFEE707480849FFF7FE
:1097C80049FA01980149086003B000BD08ED00E0BE
:1097D8000008002034100020AF0E0108F10801082D
:0C97E80033120108D10C0108930C010899
:1097F40010B588B00790F9F707FE069006982E4931
:109804000968401A7D218900884202D807980028F7
:109814004FD02A48FCF7F0FD2948808D002802D05B
:1098240006982549086026490491002005908885FA
:109834000920019005F0B7FA0198049A0599214C82
:10984400214B2360EA23D15205F0A2FA05991F4A5D
:109854001F4810601F4A20481060204A20481060AA
:109864002048036801220292D2431A6102685162BD
:10987400FCF76EFD02981C490B6802021A60096825
:10988400400208600C20039002F0A6F9039805F04A
:109894007FFA04990598154A1060154A1060154A14
:1098A4001060154A106089225200885245229200A5
:1098B400885208B010BDC046EC1300201C120020D2
:1098C400C81400202C14002001000020841400205F
:1098D40099B1000874140020E9B000084414002071
:1098E40055B20008B412002098070020C8130020C5
:0C98F400C4130020FC070020CC1300204F
:1099000000B583B001200102FA4805F047FB0128A9
:1099100040D101204102F74805F040FB012839D130
:1099200001208102F34805F039FB012832D10120E2
:10993000C102F04805F032FB002815D1EE48EF498E
:10994000FFF78CF9EE49EF480860EF49EF480860EF
:10995000EF484860EF48C8608860EF490120087010
:10996000EE490820488514E0E348ED49FFF776F911
:10997000E349EC480860E449E4480860EA48486084
:10998000E448C8608860E44901200870E349002089
:1099900048859EE101200102D64805F0FFFA002823
:1099A0003FD101204102D34805F0F8FA012838D10F
:1099B00001208102CF4805F0F1FA012831D10120C0
:1099C000C102CC4805F0EAFA002815D1CA48D749A7
:1099D000FFF744F9CA49D6480860CB49D548086022
:1099E000D5484860CB48C8608860CB4901200870E2
:1099F000CA490920488513E0F548D049FFF72EF9F8
:109A0000F549CF480860F649CA480860CD48486023
:109A1000C048C8608860F74901200870F649488549
:109A200057E101200102E94805F0B8FA012840D1C8
:109A300001204102E54805F0B1FA002839D10120A2
:109A40008102E24805F0AAFA012832D10120C102C0
:109A5000DE4805F0A3FA002815D1DD48F949FFF7E3
:109A6000FDF8DD49F8480860DD49F4480860F7482A
:109A70004860EC48C8608860DE4900200870DE4914
:109A80000A20488514E0D248EA49FFF7E7F8D249AE
:109A9000E9480860D249E9480860E9484860E14877
:109AA000C8608860D34900200870D34902204885E7
:109AB0000FE101200102C54805F070FA002840D1ED
:109AC00001204102C14805F069FA002839D101207E
:109AD0008102BE4805F062FA012832D10120C1029C
:109AE000BA4805F05BFA002815D1B948CE49FFF70E
:109AF000B5F8B949CD480860B949C8480860CC48AC
:109B00004860C848C8608860BA4900200870BA49EF
:109B10000B20488514E0AE48BE49FFF79FF8AE49D8
:109B2000BD480860AE49BD480860BD484860BD48B2
:109B3000C8608860AF4900200870AF49032048859D
:109B4000C7E001200102A14805F028FA012842D10E
:109B5000012041029D4805F021FA01283BD1012056
:109B600081029A4805F01AFA002834D10120C10276
:109B7000964805F013FA002816D19548A449FFF736
:109B80006DF895499E480860954996480860964842
:109B90004860964888609648C860964901200870D9
:109BA00095490C20488515E089489849FFF756F8F3
:109BB00089498A4808608A498A4808608A48486012
:109BC0008A4888608A48C8608A49012008708A49A2
:109BD000042048857DE0012001027C4805F0DEF983
:109BE000002842D101204102784805F0D7F9012828
:109BF0003BD101208102754805F0D0F9002834D10D
:109C00000120C102714805F0C9F9002816D1704839
:109C10007D49FFF723F87049794808607049714819
:109C2000086071484860714888607148C86071492F
:109C30000020087070490D20488515E0644871497E
:109C4000FFF70CF864496548086065496548086095
:109C500065484860654888606548C8606549002077
:109C6000087065490520488533E00120C102574846
:109C700005F094F9002816D155486049FEF7EEFF2B
:109C800055495F480860564956480860564848603C
:109C9000564888605648C8605649012008705649A1
:109CA0000C20488515E04A484A49FEF7D7FF4A4943
:109CB0004A4808604A494B4808604B4848604B484E
:109CC00088604B48C8604B49012008704A4904200D
:109CD0004885012001033D4805F060F9002833D193
:109CE0005B49012008604449488D10221043488593
:109CF0002DE0C04600040050AF0E0108070D01081A
:109D0000AC14002095B20008741300205DB3000865
:109D10009DB30008390300203B030020C814002035
:109D200024090108F5B30008BDB40008310D01088D
:109D300035B50008FDB500083DB600084F0901081B
:109D400095B600085DB70008414900200860012071
:109D500041031E4805F022F9002808D13D490120A1
:109D600008602549488D20221043488502E0394982
:109D70000020086001200190010214480290FBF7C6
:109D8000F9FA019902984902FBF7F4FA019902984D
:109D90008902FBF7EFFA01990298C902FBF7EAFA88
:109DA000019902980903FBF7E5FA01990298490322
:109DB000FBF7E0FA019902988903FBF7DBFA0199B6
:109DC0000298C903FBF7D6FA03B000BD00040050A7
:109DD000AF0E0108DE0F0108AC14002029BA0008FC
:109DE00074130020BDB8000801B900085DB900086F
:109DF000B9B900083B030020C81400206312010811
:109E0000D5B70008FB090108D90D0108D0090108E0
:109E1000AF0D0108A509010895B60008FDB50008B9
:109E20005DB7000839030020850D010835B500082D
:109E30003DB600087A090108F5B300085DB30008D3
:109E4000BDB400085B0D010895B200089DB3000881
:089E5000D01300200C140020C7
:109E580000B583B0F9F7D6FA0290184800680028D0
:109E680013D1029816490968401A164988420CD33A
:109E7800154801220192114606F0F2F901980F499E
:109E8800086002980E49086015E00C480068002830
:109E980011D002980A490968401A33280BD30A4896
:109EA80001210022009206F0DBF9009803490860BE
:109EB80002980349086003B000BDC046A4140020FE
:0C9EC800A0140020B703000000040050AC
:109ED40080B512490A6800209060096848611049F9
:109EE400EA2288520F491048086010480068002888
:109EF40013D10F480068002808D109491120020134
:109F0400885A401C88520B490120086008490120E6
:109F14000860F9F779FA0849086080BD4013002009
:109F2400C81400202C14002039030020C81300207A
:0C9F3400C4130020B41300205C060020C1
:109F400010B586B0F9F762FA014652480160006820
:109F500051490968401A022800D299E04D4800682A
:109F60004D4908604D4801684D480490428F8A1859
:109F7000E8214252415E4B2080004843494903F0AA
:109F800047FB0146049896390591D822845E4649DC
:109F90000B681B1B0B60059C0B681B190B60096889
:109FA000CB179B0CC918890B8152EA21405A002813
:109FB0006BD03E480068002809D13C490120086068
:109FC0003949002008603649D822885260E0344878
:109FD000EA21405A02282AD13148D821405E3C214A
:109FE000C943884222DC3248006800281ED109207B
:109FF000029004F0DAFE02982E4A1368002199605C
:10A0000012685161264A0392EA23D1522A4A2B4907
:10A01000116004F0BFFE039A2549012008608721E2
:10A020004B00D15A491CD152254908602CE01C48EC
:10A03000EA21405A032827D11948D821405E3D28FB
:10A0400022DB1B48006800281ED10920009004F084
:10A05000ACFE0098174A136800219960126851619C
:10A060000F4A0192EA23D152134A1449116004F0B5
:10A0700091FE019A0E490120086087214B00D15AB8
:10A08000491CD1520E49086002E0084900200860CE
:10A0900006B010BDC0140020C4140020B813002066
:10A0A000C8140020FF0F0000B8140020BC140020CA
:10A0B000CC130020401300202C1400203903002072
:04A0C000B4130020B5
:10A0C40000B581B0F9F7A0F9009000981749096824
:10A0D400401A002828D000981449086002F086FC31
:10A0E400082002F0F3FC002806D011481349FEF7BB
:10A0F400B3FD01F021FD17E0082006F01BFB00284A
:10A1040006D00B480C49FEF7A7FD01F079FD0BE0E2
:10A11400042002F0DBFC002806D005480549FEF7C0
:10A124009BFD0020FFF764FB01B000BD3C14002040
:10A13400AF0E0108AF120108260A0108030E010838
:10A1440080B508480068804707480068804707488A
:10A1540000688047064800688047064800688047D2
:10A1640080BDC04644140020481400204014002040
:08A17400841400207414002083
:10A17C0000B5A1B020902098CF490968401A4E280C
:10A18C0000D297E12098CC490860CC481F90CC486D
:10A19C001E901E9ACB49CC4B0020199005F07DFBEC
:10A1AC0019981F9A1E9BC949189105F076FB1998AE
:10A1BC00C7491A91D8228A5EC64905F06EFB1899D8
:10A1CC0019981F9A1E9B05F068FB1A991998FC2286
:10A1DC008A5EC14905F061FB189919981F9A1E9B5C
:10A1EC0005F05BFB1A991998EC228A5EBB4905F0C5
:10A1FC0054FB189919981F9A1E9B05F04EFB1A993F
:10A20C001998CC228A5AB64905F047FB1899199827
:10A21C001F9A1E9B05F041FB1A991998D2228A5A53
:10A22C00B04905F03AFB189919981F9A1E9B05F036
:10A23C0034FB1A98CA21415AAB481B90AB4A1C926A
:10A24C0000291D9001D01C981D9019981D9AA849A1
:10A25C0005F023FB189919981F9A1E9B05F01DFBFE
:10A26C001A991B98C822895A0029179001D01C985A
:10A27C0017901998179A9F4905F00FFB1899199880
:10A28C001F9A1E9B05F009FB19989B4916910968AA
:10A29C00CA6A9A4905F001FB189919981F9A1E9BD6
:10A2AC0005F0FBFA1699199809680A6B944905F0A0
:10A2BC00F4FA189919981F9A1E9B05F0EEFA1A9841
:10A2CC00EA21405A002802D19148159016E08048A6
:10A2DC00EA21405A012802D18C4814900CE07C48A9
:10A2EC00EA21415A8748884A12920229139001D0D8
:10A2FC00129813901398149014981590159A8549E8
:10A30C000020109005F0C9FA10981F9A1E9B6F49F7
:10A31C000F9105F0C2FA6E481190E221405E0D904B
:10A32C000A210C9103F06EF90C9902460D980E92CD
:10A33C005143401A06F04EFA0E9A0346109876498D
:10A34C0005F0ABFA0F9910981F9A1E9B05F0A5FA11
:10A35C001198F621405AC00700280CD06F490A9179
:10A36C00704A00200B9005F098FA0A990B986C4AE9
:10A37C0005F093FA04E06949694A002005F08DFA6A
:10A38C001F9A1E9B5149002005F087FA5048F62170
:10A39C00405A800700280CD560490891614A00207A
:10A3AC00099005F07AFA089909985F4A05F075FA50
:10A3BC0004E05A495C4A002005F06FFA1F9A1E9B74
:10A3CC004249002005F069FA4148F621405A4007FD
:10A3DC0000280CD551490691524A0020079005F0EF
:10A3EC005CFA06990798514A05F057FA04E04B4974
:10A3FC004E4A002005F051FA1F9A1E9B334900204B
:10A40C0005F04BFA3248F621405A000700280CD5CB
:10A41C0042490491434A0020059005F03EFA049904
:10A42C000598434A05F039FA04E03C49404A0020BB
:10A43C0005F033FA1F9A1E9B2449002005F02DFAD3
:10A44C002348F621405A800600280CD53349029146
:10A45C00344A0020039005F020FA029903982A4A06
:10A46C0005F01BFA04E02D49274A002005F015FAE7
:10A47C001F9A1E9B1549002005F00FFA2D4802214A
:10A48C0004F086FD01280CD1244900912B4A0020B0
:10A49C00019005F002FA00990198294A05F0FDF99E
:10A4AC0004E01E49244A002005F0F7F92549002054
:10A4BC0005F0F3F921B000BD94140020C712010877
:10A4CC002B1201082B100108AF0E0108CF12010846
:10A4DC00C8140020D7120108E3120108301001083B
:10A4EC00410A01084C0A0108190E0108EF12010873
:10A4FC00391001084210010840130020570A0108C6
:10A50C00620A0108730A0108760A0108700A010838
:10A51C006D0A01081B0E01084B100108790A01088D
:10A52C007C0A0108FF1201087F0A0108820A01084F
:10A53C00850A0108000C00501713010807130108C5
:08A54C000F130108210E0108A4
:10A5540070B59CB012901298ED490968401AED4903
:10A564000968884200D8AFE31298E9490860E949CC
:10A5740087200860E848C08813901399E748484347
:10A58400001313901399E6484843E64903F03EF854
:10A594001390E548CC21425AE4480168891A0160C5
:10A5A4000068002802D5E14900200860139ADF48BA
:10A5B4000168891801600068C117490F4018C20872
:10A5C400D949CC200A52085AD022895A884205DD3A
:10A5D400D549CC20085AD02288520BE0D249CC204D
:10A5E400085ACE22895A884204DACF49CC20085A24
:10A5F400CE228852C848408814901499C7484843CA
:10A60400001314901499C6484843C64902F0FEFF4B
:10A614001490C548D221425AC5480168891A01607C
:10A624000068002802D5C24900200860149AC04876
:10A634000168891801600068C117C90E40184209F1
:10A64400B948D2214252405ABA49884214DCBA4825
:10A65400006800280FD1B84901200860B24AF623E7
:10A66400D15A08242143D15283214B00D15A491C89
:10A67400D152B24908600EE0AB48D221405AB049E9
:10A68400884208DBAC4900200860A749F622885AB2
:10A69400082398438852A449D220085AD622895ABA
:10A6A400884205DDA049D220085AD62288520BE000
:10A6B4009D49D220085AD422895A884204DA9A49F8
:10A6C400D220085AD4228852934801889D4848438E
:10A6D4009D4940189D4902F099FF9D4940181190E9
:10A6E4009149E2200C5E9B4A13681B1B1360119C6A
:10A6F40013681B1913601268D317DB0ED2185209A2
:10A704000A52085EE622895E884205DD8649E22017
:10A71400085AE62288520BE08349E220085EE422CC
:10A72400895E884204DA8049E220085AE422885289
:10A734007D49E220085E098D884213DB8648006863
:10A7440000280ED1844901200860774AF623D15AA3
:10A754000143D15281214B00D15A491CD15277492E
:10A7640008601AE07048E221415E0A91018D4B2095
:10A774004843642102F072FF01460A9888420CDAC9
:10A7840076480068002808D07349002008606649AC
:10A79400F622885A01239843885271480068012898
:10A7A40006D16149F622885A02231843885205E0EB
:10A7B4005D49F622885A0223984388526948006802
:10A7C400012806D15849F622885A0423184388528E
:10A7D40005E05549F622885A042398438852624872
:10A7E4000068012806D15049F622885A20231843CC
:10A7F400885205E04C49F622885A2023984388520F
:10A804004948D821405E00281DD54749D820085E14
:10A814004042E022895A884206DD4349D820085A3A
:10A824004042E02288520DE03F49D820085E404271
:10A83400DE22895A884205DA3B49D820085A404228
:10A84400DE22885218E03849D820085EDC22895A72
:10A85400884205DD3449D820085ADC2288520BE0AE
:10A864003149D820085EDA22895A884204DA2E490E
:10A87400D820085ADA2288523C4B18682A49F82210
:10A8840088523B4C2068FA22885210201090394894
:10A894000668394A1568AD1B15601D6813685B1995
:10A8A40013601268D3171B0FD21812110260334BB6
:10A8B4001E68334A1568AD1B156025681468641951
:10A8C40014601268D417240F121912111A60006848
:10A8D4004C22895A884207DB26480068FD494C22ED
:10A8E400895A401A099001E00020099009980F90B4
:10A8F400F9480068F7494E22895A884242DBF648F3
:10A904000068F4494E22895A401A08903CE0C04637
:10A914006414002098060020DE150020B80B000007
:10A92400A086010010270000C81400209C140020F9
:10A934009C0600201F4E0000D8130020B4130020F2
:10A94400C15D0000140500000CE3F7FFEF060000F2
:10A95400D4FEFFFF58140020FC0700200C14002034
:10A96400C8130020C4130020CC130020BC13002003
:10A97400C0130020501400205C1400205414002044
:10A98400601400200020089008980E900F980E99EB
:10A99400401A0D900D99CE484843D04902F036FE36
:10A9A400CC490791FC2288520D9A5F2080005043C5
:10A9B400C98F02F02BFE01460798EC228152EA214E
:10A9C400405A002808D1C6480068C649884203D0C6
:10A9D400C349C448086015E0BE48EA21405A01282A
:10A9E40008D1BF480068C049884203D0BC49BE486A
:10A9F400086007E0BA480068BC49884202D0B849F8
:10AA0400BA480860BA480690402104F0C5FA0146E5
:10AA140006980CAA1170802104F0BEFA0BA90870E4
:10AA2400B448007800281AD10BA80078012804D172
:10AA3400A849C8220020885203E0A649C822012060
:10AA440088520CA80078012804D1A249CA22002007
:10AA5400885203E09F49CA220120885219E00BA8BA
:10AA64000078002804D19B49C8220020885203E0C2
:10AA74009849C822012088520CA80078002804D1E3
:10AA84009449CA220020885203E09249CA22012034
:10AA940088529048EA21405A012809D08D48EA2179
:10AAA400405A022804D08B48EA21405A032825D171
:10AAB4008848D821405E032809DB8F4802210122FF
:10AAC40005F0D0FB8D497D208000086015E08148A9
:10AAD400D821405E002810DC88480068012803DB88
:10AAE40086490868401E086084480068002804D12C
:10AAF40081480221002205F0B5FB04E07E480221D2
:10AB0400002205F0AFFB7E48008872494422895A2E
:10AB1400884225D06F494420085A898F88421FDD16
:10AB24006C484421405A6A49884203DB69494422FB
:10AB340067488852674805904421425A704B1A80EE
:10AB4400415A66484843624902F088FD0246059826
:10AB540046214252415A4A22805A48436949086070
:10AB6400694800885B494822895A88421ED059485E
:10AB74004821405A1E2803DC564948221F20885287
:10AB8400544804904821425A5F4B1A80415A5F4806
:10AB940048435F4902F03AFD014604984A22815233
:10ABA4004621415A805A4843564908600520000707
:10ABB4000121090204F0F0F9012804D14549FE22DB
:10ABC4000120885203E04349FE22002088520120DC
:10ABD4001B9000214F48405E3E494222895A8842D8
:10ABE40072D04D4805F0F2F93A494220085A898F4B
:10ABF400884203DA3749888F4222885235484221F5
:10AC0400405A4649884203DB32494222304888523E
:10AC140030484221425A3F4B1A80002203921A9232
:10AC2400199218921792169215923D4A1592032280
:10AC3400920516923B4A17921B9A531E9A4115ABE2
:10AC440002931A73415A25484843214902F006FDEC
:10AC540002990246039819921A902F48F9F712F9AB
:10AC6400002801D000F08AF92F48159003208005B0
:10AC740016902E4817901B98411E884115A90191E2
:10AC8400087314484221415A14484843104902F0B9
:10AC9400E5FC0199199000201A901F48F9F7F2F881
:10ACA400002801D000F06AF91B4808490622F8F789
:10ACB4003FFE002803D01E481E49FEF711F81E4926
:10ACC40008680422904308601CB070BDDE150020A3
:10ACD400B80B0000C814002054140020FF0F00001B
:10ACE4004414002055B2000875B20008D9B1000818
:10ACF400000800503B030020000C005068140020A2
:10AD0400F015002064060020F215002000E2040083
:10AD140040420F00EE15002098070020B90B0000F8
:10AD2400FFFF170004000008FFFF27004000001881
:0CAD3400AF0E0108750C01080800024079
:10AD400000B583B00290192001900298204909684B
:10AD5000401A0199884238D902981D490860192083
:10AD600001901C4908784000087005200007012167
:10AD7000C90304F013F9002820D1164801780122F4
:10AD8000114301700078002817D01348006800288C
:10AD900013D011490020086010480068002806D030
:10ADA0000F49114808600D490020086005E00C4972
:10ADB0000C48086009490120086006E00548007851
:10ADC000002802D104490120086003B000BDC0463C
:10ADD0002014002043070020780600207C06002075
:0CADE00048140020599E000895AF0008A0
:10ADEC0000B587B00122029206926846059004A82D
:10ADFC000090C821018003A90191064B0B8000F043
:10AE0C0029F900980199029A00F006F905988546EF
:08AE1C0007B000BDC4090000ED
:10AE240000B587B00222029206926846059004A8F3
:10AE34000090C823038003A901910B804380064B33
:10AE44004B8000F00BF900980199029A00F0E8F8A1
:0CAE54000598854607B000BDC409000049
:10AE600000B58BB003200A90684609900020089036
:10AE7000089801280CD80898420006A9C8208852D2
:10AE800008994A0004A988520898401C0890EFE7E6
:10AE900006A80190C821818004A90291074A8A80EE
:10AEA0000322039200F0DCF801980299039A00F063
:10AEB000B9F8099885460BB000BDC046C40900002A
:10AEC00000B58BB004200A906846099000200890D5
:10AED000089802280CD80898420006A9C820885271
:10AEE00008994A0004A988520898401C0890EFE786
:10AEF00006A80190C821C18004A90291074ACA800E
:10AF00000422039200F0ACF801980299039A00F031
:10AF100089F8099885460BB000BDC046C4090000F9
:10AF200000B58DB005200C9068460B9000200A906B
:10AF30000A9803280CD80A98420007A9C82088520A
:10AF40000A994A0004A988520A98401C0A90EFE71F
:10AF500007A80190C821018104A90291074A0A812A
:10AF60000522039200F07CF801980299039A00F000
:10AF700059F80B9885460DB000BDC046C4090000C5
:10AF800080B502480249FDF7ADFE80BDAF0E010855
:04AF9000CA0A0108E0
:10AF940080B504480122114605F064F902490348CA
:10AFA400086080BD000400504814002039030020CC
:10AFB40004490A6800209060096848610249EA224D
:0CAFC4008852704740130020C814002081
:10AFD00000B581B011485421405A1149098888426E
:10AFE0000CD10E4800900021FDF7FEFA0099562082
:10AFF0000A5A0B4802800088542288520848008868
:10B00000002804D0054950220120885203E003495A
:10B0100050220020885201B000BDC046C814002054
:04B02000EA1500200D
:10B0240000B587B0069005910492049B0698059993
:10B0340002220392054A02920191009004480549B4
:10B04400054A04F0B4FC07B000BDC046000400503B
:0CB054001C14002018140020141400200C
:10B0600000B587B0069005910492049B0698059957
:10B0700008220392054A0292019100900448054972
:10B08000054A04F096FC07B000BDC046000400501D
:0CB09000801400207C14002078140020A4
:10B09C0010B58AB00422039209926846089006A85B
:10B0AC000190C823038004A902910B8043807D2367
:10B0BC009C004C80AF239B0083808C80C380064B0C
:10B0CC00CB80FFF7C7FF01980299039AFFF7A4FF03
:0CB0DC00089885460AB010BDC4090000A9
:10B0E80000B583B00848019008210022029205F0BB
:10B0F800B7F80198029A022105F0B2F8034904480A
:10B10800086003B000BDC04600040050741400205D
:04B1180039030020D7
:10B11C0000B583B0F8F774F902901848006800285D
:10B12C0013D1029816490968401A164988420CD363
:10B13C00154810210122019205F090F801980F4951
:10B14C00086002980E49086015E00C480068002859
:10B15C0011D002980A490968401AC9280BD30A4829
:10B16C0010210022009205F079F80098034908603C
:10B17C0002980349086003B000BDC0468C1400203F
:0CB18C0088140020210300000004005083
:10B1980080B504481021002205F062F802490348EE
:10B1A800086080BD0004005084140020390300208A
:10B1B80080B504481021012205F052F802490348DD
:10B1C800086080BD0004005084140020390300206A
:10B1D80000B583B0F8F716F90290184800680028FF
:10B1E80013D1029816490968401A164988420CD3A7
:10B1F800154804210122019205F032F801980F49FF
:10B20800086002980E49086015E00C48006800289C
:10B2180011D002980A490968401A33280BD30A4802
:10B2280004210022009205F01BF8009803490860E9
:10B2380002980349086003B000BDC046701400209E
:0CB248006C140020B7030000000400504C
:10B2540080B504480421002205F004F8024903489B
:10B26400086080BD0004005044140020390300200D
:10B2740080B504480421012204F0F4FF0249034884
:10B28400086080BD000400504414002039030020ED
:10B2940000B585B0049003910398002803D0284991
:10B2A4000220086041E0049821490968401A2149B4
:10B2B4000968884239D904981D4908601E488021CC
:10B2C40003F06AFE02A908701C480078002804D123
:10B2D40002A9087842425041087002A800780190FF
:10B2E40001981749096888420CD0019882001848CF
:10B2F40080581449885001988100164840580D49D7
:10B3040008600AE0019882000E490F4888500198AD
:10B3140081000E4840580749086001988100094897
:10B324004058804701980649086005B000BDC046F2
:10B33400B4140020B4060020000800503B03002091
:10B34400B0060020AC130020390300202CE90008CB
:08B354007413002024E9000835
:10B35C0000B581B00920009003F021FD0098074A48
:10B36C0007491160074AEA230121D15203F00CFD71
:10B37C0005490648086001B000BDC0462C140020E9
:10B38C00C9000020C8140020841400201DB100083E
:10B39C0000B583B00920019003F001FD01980C4A1F
:10B3AC000C4911600C4A0292EA230021D15203F09D
:10B3BC00EBFC0299094A0A4810602120C200885A05
:10B3CC00401C885207490120086003B000BDC046EC
:10B3DC002C14002011010020C8140020841400201B
:08B3EC001DB10008B41300209C
:10B3F40000B585B0049003910398002804D028492F
:10B404000020C043086041E0049821490968401ABB
:10B4140020490968884239D904981D4908601E48A2
:10B42400802103F0B9FD02A908701C4800780028A7
:10B4340004D102A9087842425041087002A8007859
:10B44400019001981649096888420CDD0198820030
:10B45400174880581349885001988100154840586E
:10B464000C4908600AE0019882000E490E48885091
:10B47400019881000D4840580649086001988100F0
:10B4840008484058804701980549086005B000BD48
:10B494003814002094060020000800503B030020CC
:10B4A400900600209C130020390300201CE90008AA
:08B4B4007413002014E90008E4
:10B4BC0000B585B00920019003F071FC0198134A86
:10B4CC0013491160134A0392EA2300210291D152CD
:10B4DC0003F05AFC0299039881850F4A0F481060BB
:10B4EC000F48036801220492D2431A610268516228
:10B4FC00FAF72AFF039A04982121CB00D15A491C50
:10B50C00D1520849086005B000BDC0462C1400207B
:10B51C0001000020C81400208414002099B10008F8
:08B52C00B4120020B41300204A
:10B5340000B585B0049003910398002803D02849EE
:10B544000220086041E0049821490968401A214911
:10B554000968884239D904981D4908601E48402169
:10B5640003F01AFD02A908701C480078002804D1D1
:10B5740002A9087842425041087002A8007801905C
:10B5840001981749096888420CD00198820018482C
:10B5940080581449885001988100164840580D4934
:10B5A40008600AE0019882000E490F48885001980B
:10B5B40081000E48405807490860019881000948F5
:10B5C4004058804701980649086005B000BDC04650
:10B5D400A8140020A4060020000800503B0300200B
:10B5E400A0060020A4130020390300200CE9000861
:08B5F4007413002004E90008B3
:10B5FC0000B581B00920009003F0D1FB0098074AF8
:10B60C0007491160074AEA230121D15203F0BCFB20
:10B61C0005490648086001B000BDC0462C14002046
:10B62C0041000020C8140020841400201DB1000823
:10B63C0000B583B00920019003F0B1FB01980C4ACE
:10B64C000C4911600C4A0292EA230021D15203F0FA
:10B65C009BFB0299094A0A48106085204200885ACF
:10B66C00401C885207490120086003B000BDC04649
:10B67C002C14002089000020C81400208414002001
:08B68C001DB10008B4130020F9
:10B6940000B585B0049003910398002804D028498C
:10B6A4000020C043086041E0049821490968401A19
:10B6B40020490968884239D904981D4908601E4800
:10B6C400402103F069FC02A908701C480078002896
:10B6D40004D102A9087842425041087002A80078B7
:10B6E400019001981649096888420CDD019882008E
:10B6F40017488058134988500198810015484058CC
:10B704000C4908600AE0019882000E490E488850EE
:10B71400019881000D48405806490860019881004D
:10B7240008484058804701980549086005B000BDA5
:10B734002814002084060020000800503B03002049
:10B74400800600209413002039030020FCE8000840
:08B7540074130020F4E8000862
:10B75C0000B585B00920019003F021FB0198134A34
:10B76C0013491160134A0392EA2300210291D1522A
:10B77C0003F00AFB0299039881850F4A0F48106069
:10B78C000F48036801220492D2431A610268516285
:10B79C00FAF7DAFD039A049885214B00D15A491C1B
:10B7AC00D1520849086005B000BDC0462C140020D9
:10B7BC0001000020C81400208414002099B1000856
:08B7CC00B4120020B4130020A8
:10B7D40000B587B0069005910598002803D030493C
:10B7E4000420086052E0069829490968401A29494A
:10B7F400096888424AD90698254908602648019074
:10B80400402103F0C9FB0146019804AA117080216C
:10B8140003F0C2FB03A9087020480078002809D16E
:10B8240004A9087842425041087003A908784242AA
:10B834005041087004A80078400003A9097808431F
:10B84400029002981649096888420CD00298820036
:10B854001748805813498850029881001548405869
:10B864000C4908600AE0029882000E490E4888508C
:10B87400029881000D4840580649086002988100EA
:10B8840008484058804702980549086007B000BD41
:10B89400B0140020AC060020000800503B03002038
:10B8A400A8060020841300203903002064E900085E
:08B8B4007413002054E90008A0
:10B8BC0000B581B00920009003F071FA0098084A95
:10B8CC000849116003F060FA0749EA220120885206
:10B8DC00064907480860FFF701FC01B000BDC046EF
:10B8EC002C14002099040020C8140020841400207B
:04B8FC001DB1000872
:10B9000000B583B00920019003F04FFA01980D4A69
:10B910000D4911600D4A0292EA230321D15203F02E
:10B9200039FA0B490B480860FFF7DEFB029921202A
:10B93000C200885A401C885207490120086003B0A1
:10B9400000BDC0462C14002051010020C814002066
:0CB95000841400201DB10008B413002076
:10B95C0000B583B00920019003F021FA01980D4A3B
:10B96C000D4911600D4A0292EA230221D15203F0D3
:10B97C000BFA0B490B480860FFF7B0FB02998520C6
:10B98C004200885A401C885207490120086003B0C5
:10B99C0000BDC0462C140020DD010020C81400207E
:0CB9AC00841400201DB10008B41300201A
:10B9B80000B583B00920019003F0F3F90198104A0B
:10B9C80010491160104A0292EA230021D15203F073
:10B9D800DDF902990D4A0E4810600E4A0E481060B3
:10B9E8002120C200885A401C885285204200885A6B
:10B9F800401C885209490120086003B000BDC046B8
:10BA08002C14002069020020C8140020841400208F
:10BA180099B10008741400209DB00008B4130020E8
:10BA280000B587B0069005910598002806D03A4AD7
:10BA38000020C14311603C49086062E00698324921
:10BA48000968401A3149096888425AD906982E4926
:10BA580008602F480190402103F09CFA01460198A4
:10BA680004AA1170802103F095FA03A908702948E7
:10BA78000078002809D104A908784242504108708A
:10BA880003A9087842425041087004A80078400091
:10BA980003A909780843029002981F490968884257
:10BAA80016D021480068002811D10298012802DB2D
:10BAB8001D4901200860029882001C4880581749D7
:10BAC8008850029881001A484058104908600AE0D6
:10BAD8000298820011491248885002988100114842
:10BAE80040580A490860029881000C4840580028CC
:10BAF80004D00298810009484058804702980649B6
:10BB0800086007B000BDC046341400208C06002031
:10BB1800000800503B030020880600206413002022
:10BB28003903002044E90008301400207413002071
:04BB380034E90008E4
:10BB3C0000B583B0F7F764FC02901C48808D022896
:10BB4C0032D01A48808D01282ED0029818490968E5
:10BB5C00401A1849884227D3029817490968401A95
:10BB6C001649884220D3029815490968401A13498E
:10BB7C00884219D31348FAF73BFC02980C49086029
:10BB8C001148026801210191C94311610268002129
:10BB9C005162FAF7D9FB0198044A43218B00D15A20
:10BBAC00491CD1520949086003B000BDC8140020DB
:10BBBC00EC130020E90300005C06002011270000B4
:10BBCC00600600201C120020EC100020B413002092
:10BBDC0081B001466846017000214056002807D408
:10BBEC00684601781F200140012088400149086007
:08BBFC0001B0704780E200E097
:10BC040000B583B01948808D01282DD01748808D48
:10BC1400022829D016480068002825D0F7F7F4FB3D
:10BC2400144908601448026801210291C943009133
:10BC340011610268002101915162FAF789FB009AAF
:10BC440001990E4803681A6102685162FAF780FB91
:10BC54000298064A43218B00D15A491CD152084903
:10BC640008600C2003F09FF803B000BDC814002046
:10BC7400D0130020EC130020381100201C120020E7
:04BC8400B4130020D5
:10BC880000B589B00020089007901D4906910590DD
:10BC980005981C49884215D81F490A6808988018D1
:10BCA80008901E480368079AD2180792059A0B68ED
:10BCB800006800901A49002003F0F1FD0598401C27
:10BCC8000590E5E708980E49029101F0C5FC029934
:10BCD8000D4A04924C230393D052079801F0BCFC00
:10BCE800039A034604984E214352825A435A0749FD
:10BCF800002003F0D4FD06490648086009B000BDDD
:10BD080050C300004FC30000C8140020851001086C
:10BD18009814002039030020BC130020C013002011
:04BD280058100108A6
:10BD2C0000B585B0049003910398C72807DC0499EB
:10BD3C006E204843642101F065FC04901EE00398DA
:10BD4C00C82816DB03980F49884212DC049802902D
:10BD5C000398002100914B21CA00C8210A2303F04B
:10BD6C0085FE029964304843642101F04BFC049039
:10BD7C0004E003984B21C9008842FFDB049805B00E
:08BD8C0000BDC0465702000093
:10BD940000B585B02C482D49FCF75EFFF7F734FB5E
:10BDA40004900020039002900190F7F72DFB049972
:10BDB400401A2749884217D802990398401A0390D9
:10BDC4002A4801680398401803900398C117090F83
:10BDD400401800110290029A2549002003F061FDE9
:10BDE4000120F7F717FBE0E71A4900914E200A5AA1
:10BDF4000298801A02900298E222895EFFF794FF6B
:10BE04000290029914484843144901F0FFFB01468B
:10BE140000980191019981870299C187C18F6E2091
:10BE24004843642101F01AFC0146009840228152E3
:10BE3400C28F838F0A49002003F033FD09490A4861
:10BE4400086005B000BDC046AF0E0108880A0108AD
:10BE54005FEA0000C8140020B80B0000FF0F0000C8
:10BE64003F1301089814002039030020C013002058
:04BE74001F1301088F
:10BE780000B583B000200290144901910090009809
:10BE8800134988420ED81848026802998918029105
:10BE9800009A03681549002003F001FD0098401C32
:10BEA8000090ECE70298094901F0D6FB01460948E1
:10BEB800411A094841873A21425E0849002003F0A7
:10BEC800EEFC07490748086003B000BD50C30000F6
:10BED8004FC30000FF070000C8140020AA10010883
:10BEE8009814002039030020B8130020AF0A010875
:10BEF800BFF34F8F034904480860BFF34F8F00BF5B
:0CBF0800FDE7C0460CED00E00400FA0567
:10BF140010B588B00B9C0A9C079006910592049377
:10BF240006980799086007980168454808600798CB
:10BF340001684B2000024860079802680121080349
:10BF44009060079802680020D060079A12688902FE
:10BF5400116107990A680C21516107990968886180
:10BF640007990968C8610799096808620799096807
:10BF740048620799096888620598079909684860C2
:10BF84000498002809D107980268012081021161F0
:10BF9400079909680003886014E0049801280AD10D
:10BFA400079801680320400208610798016801208E
:10BFB4000003886006E0079801680020086107997B
:10BFC400096888600A98012804D10798016800204C
:10BFD400C86004E00798016801204003C86007981E
:10BFE400006803900B9801F0E9F900220292154BC6
:10BFF40003F00BFE01F09AF9029B014603980091AD
:10C0040019461A4600F024F8002801D0FEF7B6FFBE
:10C014000798006804F028FA002801D0FEF7AEFF64
:10C0240007990868273101221202FBF781F80028DA
:10C0340004D005480549FCF753FEFEE708B010BDDF
:10C044000038014000000C40CB130108D010010857
:10C0540010B586B0089C0490039102920193049851
:10C06400002803D105A90120087069E004988421FF
:10C074004058002806D1049980220020885404984E
:10C0840000F052FF04998422242088500498016807
:10C0940008680122904308600498FAF731FC0128EB
:10C0A40003D105A9012008704AE00498806A002899
:10C0B40002D0049802F0F1FF049801688868012214
:10C0C400930318438860049800688068D103884308
:10C0D4000399084304990968886002984005009010
:10C0E40001980104009808430090049800680068CF
:10C0F40015490840009908430499096808600498A0
:10C1040001684868D30518434860049801680868C2
:10C11400930618430860049800684069FF210906E3
:10C12400084008990843049909684861049801681B
:10C134000868104308600498FAF742FE05A90870DD
:0CC1440005A8007806B010BDFFFF00FC4D
:10C1500010B588B0079007980068C06906900798E6
:10C160000068006805900798006880680490069849
:10C170000F2108400390039800285BD004988F4952
:10C18000084205D105A8008809214901084251D07B
:10C1900006A80078C00700280DD005A84078C00781
:10C1A000002808D0079800680123036207998C22B1
:10C1B00088581843885006A80078800700280ED5B4
:10C1C00004A80078C007002809D007980168022059
:10C1D000086207998C22885804231843885006A8BF
:10C1E0000078400700280ED504A80078C007002872
:10C1F00009D0079801680420086207998C228858A2
:10C2000002231843885006A800780007002811D59B
:10C2100005A800788006002803D4049867490842DE
:10C2200008D0079800680823036207998C22885871
:10C230001843885006A840780007002819D505A89B
:10C24000C0784007002804D404A88078000600289D
:10C250000FD5079802680120C1021162079A88234E
:10C260002021D150079A8423D15055490875554A49
:10C27000885406A80078800600282BD505A80078E9
:10C280008006002804D404A8C078C006002821D560
:10C29000079888214058222816D149484521C900CD
:10C2A0004058FF2810D807980068406A4449452242
:10C2B000D2008B58CB18272418558858401C88501A
:10C2C000404A0120885405E00798016888690822DF
:10C2D0001043886106A800780006002813D505A839
:10C2E00000780006002804D404A8807800060028FE
:10C2F00009D533480290006804F068F902992320B8
:10C3000002010120885406A80078400600280FD5B5
:10C3100005A80078400600280AD5294926220020D1
:10C320008854079803F0C1FB07998822222088507F
:10C3300007988C21405800283DD007998822222058
:10C34000885006A800788006002814D505A8007833
:10C350008006002804D404A8C078C00600280AD5A6
:10C3600007980168886908221043886107998C2220
:10C37000002088501FE006A80078000600281AD583
:10C3800005A800780006002804D404A880780006D8
:10C39000002810D50A4901912622002088540798C8
:10C3A00003F083FB0199079A88232220D050232091
:10C3B00002010120885408B010BDC04601000010E1
:08C3C000C00C00203102000056
:10C3C80085B00490039102A91848088000200190C4
:10C3D80001980399884225D204980199415C0298F2
:10C3E800484002A90880082000900098002815D02D
:10C3F80002A80088C007002808D002A908884008B9
:10C40800088002980A4A5040088003E002A9088878
:10C41800400808800098401E0090E6E70198401CFC
:10C428000190D5E702A8008805B07047FFFF00001B
:04C4380001A000005F
:10C43C0000B585B0039003982730019003984521EF
:10C44C00C900405802900198007800900298042886
:10C45C0005D8039803F054FB002004901FE00198CA
:10C46C00029904F0E3F8401C002805D1039803F06E
:10C47C0047FB0020049012E00098002802D1022013
:10C48C0004900CE000980749C98B884202D1022025
:10C49C00049004E0039803F033FB0020049004980C
:08C4AC0005B000BDC81400201A
:10C4B40010B588B006900591049203A80370007823
:10C4C4003549C98B88420BD003A80078002807D0CF
:10C4D4000698049B06210B2203F060FB079058E0AA
:10C4E400059988780002C97840180290059908795E
:10C4F40000024979401800900098002802D0009862
:10C504007E2807D30698049B0322114603F046FBBA
:10C5140007903EE0029800994018401E8B2807D3EC
:10C524000698049B0321022203F038FB079030E0B5
:10C534000699049A032088540498401C0490009897
:10C5440040000699049A88540498401C0490029868
:10C55400019001980299009A8918884217D201988B
:10C5640041000D4841184978069A049BD154049916
:10C57400491C049101994900405C0699049A885425
:10C584000498401C04900198401C0190E1E7049831
:0CC594000790079808B010BDC8140020E4
:10C5A00010B586B0089C0490039102920193019803
:10C5B0003E49C98B88420AD00198002807D00498C8
:10C5C000029B06210B2203F0EBFA05906BE0039926
:10C5D00088780002C9784018009000988B2807D30B
:10C5E0000498029B0621022203F0DAFA05905AE031
:10C5F00008988D21890040580099405C002807D197
:10C600000498029B0621022203F0CAFA05904AE030
:10C6100008988D21890040580099405C02280ED16D
:10C6200008984721C90040580088002807D104987D
:10C63000029B0621022203F0B3FA059033E003982F
:10C64000007900994A0019498A1850700398407976
:10C65000009A520088540499029A0620885402983D
:10C66000401C02900098000A0499029A885402988B
:10C67000401C029000980499029A88540298401C29
:10C680000290039800790499029A88540298401CF9
:10C690000290039840790499029A88540298401CA9
:10C6A000029002980590059806B010BDC8140020AD
:10C6B00010B58AB00C9C08900791069205930598D6
:10C6C0004F49C98B88420AD00598002807D008989E
:10C6D000069B06210B2203F063FA09908DE007996F
:10C6E00088780002C97840180490079908790002F8
:10C6F000497940180390072001900398002802D040
:10C7000003987C2807D30898069B1021032203F086
:10C7100047FA099071E0049803994018401E8B284D
:10C7200007D30898069B1021022203F039FA0990DA
:10C7300063E00498029002980499039A8918884249
:10C7400034D20C988D21890040580299405C002811
:10C7500003D10198801C019024E00C988D21890060
:10C7600040580299405C02280AD10C984721C90020
:10C7700040580088002803D10198801C019011E0E6
:10C7800007980199405C02994A001D498A18507027
:10C79000079A019880184078029A520088540198AC
:10C7A000801C01900298401C0290C4E70899069AE8
:10C7B000102088540698401C06900498000A089996
:10C7C000069A88540698401C069004980899069A80
:10C7D00088540698401C06900398000A0899069A07
:10C7E00088540698401C069003980899069A885425
:10C7F0000698401C06900698099009980AB010BD4A
:04C80000C814002038
:10C8040000B583B00E48026801210A430260006843
:10C814000840029002980B480268012109070A4364
:10C8240002600068084001900198F6F71FFE02209C
:10C83400F6F70EFE03204002F6F720FE03B000BD1B
:08C84400401002403C100240CC
:10C84C0080B5F9F72FFB0448022103F01BFD0349C7
:10C85C00002002F019F8F6E700040050450E01081C
:10C86C0000B581B006490020009002F00DF8009848
:10C87C00044902F009F80448022103F003FDFAE729
:0CC88C00CF130108D7130108000400506E
:10C8980080B50248F9F7D4FD80BDC04638110020A4
:10C8A80080B50248F9F7CCFD80BDC046EC100020E9
:10C8B80080B50248F9F7C4FD80BDC046B412002017
:10C8C80080B50248F9F7BCFD80BDC046681200205B
:10C8D80080B50248F9F7B4FD80BDC0461C1200209F
:10C8E80080B50248F9F7ACFD80BDC046D0110020E4
:10C8F80000B583B002900298F9F77CFD02980068B1
:10C908002A4988420BD13049012088852F4B344A67
:10C918001A60EA2288522F493248086043E0029898
:10C92800006823490968884208D127490220888578
:10C938002A48026800200121904734E002980068E4
:10C948001C490968884200D12DE0029800681A49FC
:10C95800884200D127E002980068184988421AD115
:10C968001949002000908885184B194A1A60EA2254
:10C9780088521849184808600E480190F9F73AFD9E
:10C988000099019803680122D2431A610268516232
:10C99800F9F7DCFC07E0029800680949884202D1EF
:10C9A80008490120086003B000BDC04600100040DF
:10C9B800EC100020B4120020004001400044014067
:10C9C80000480140FC130020C81400202C1400204B
:10C9D800010000208414002099B10008AC14002044
:08C9E800A9020020B9B100080A
:10C9F00030B581B01F4801681F4A1268514000914C
:10CA00001E4A1168009B1940C943116013681C49F4
:10CA10000C68009D2C4063400B60126809680A4056
:10CA2000009911400091009A01685140016003682B
:10CA300000990B40134A11681943116000780007F0
:10CA4000800F002803D110494B20400108600E4997
:10CA50000868401E086000280AD10B49642008605D
:10CA6000044802680C200240084908681043086026
:10CA700001B030BDF0130020100C0050081400204D
:10CA800004140020F813002000140020F4130020E8
:10CA900081B0009005490A68009810400090009A03
:10CAA000086850400860009801B07047F8130020F3
:10CAB00081B0009005490A68009810400090009AE3
:10CAC000086850400860009801B07047F4130020D7
:10CAD00000B581B000900448016800988843FFF7D2
:0CCAE000D7FF01B000BDC046F0130020DD
:10CAEC0000B589B00021019108910791069105913B
:10CAFC000491039102911448012292070260416053
:10CB0C008160CA43C2600161816102F05AFA002857
:10CB1C0001D0FEF72FFA0120000305900A4805A961
:10CB2C00F9F7B2FD002801D0FEF724FA002002909C
:10CB3C000490054802A9F9F76FFE002801D0FEF712
:0CCB4C0019FA09B000BDC0468411002099
:10CB580000B583B000210291019100910D480E4A61
:10CB68000260F922426081600C4AC260816102F071
:10CB78002AFA002801D0FEF7FFF900200090029061
:10CB880004486946F9F74AFE002801D0FEF7F4F98F
:10CB980003B000BD3811002000100040FFF900006C
:10CBA80000B583B000210291019100910D480E4A11
:10CBB8000260F922426081600C4AC260816102F021
:10CBC80002FA002801D0FEF7D7F900200090029061
:10CBD80004486946F9F722FE002801D0FEF7CCF98F
:10CBE80003B000BDEC10002000140040FFF9000065
:10CBF80080B50948094901606321416000218160CD
:10CC0800074AC2600161816102F0DDF9002801D0A4
:10CC1800FEF7B2F980BDC046B412002000200040E3
:04CC2800FFF9000010
:10CC2C0000B589B0002100910891079106910591FA
:10CC3C0004910391029114480190144A02604160DE
:10CC4C008160134AC26001614161816102F0B9F9EE
:10CC5C00002801D0FEF78EF90120000305900A4848
:10CC6C0005A9F9F711FD002801D0FEF783F9002082
:10CC7C0002900490044802A9F9F7CEFD002801D0D7
:10CC8C00FEF778F909B000BD6812002000400140A1
:04CC9C00FFFF000096
:10CCA00000B581B00A4800900A4901600A49416014
:10CCB00000218160094AC26001614161816102F025
:10CCC00086F9002801D0FEF75BF901B000BDC0462F
:10CCD0001C120020004401405FEA0000FFF9000040
:10CCE00000B581B00A4800900A4901600A494160D4
:10CCF00000218160094AC26001614161816102F0E5
:10CD000066F9002801D0FEF73BF901B000BDC0462E
:10CD1000D011002000480140FFF900000F2700005B
:10CD200000B59BB01A900DA8342100F049FD1A9867
:10CD3000006801218907884209D15C480268012105
:10CD40000A430260006808400C900C989EE01A9814
:10CD500000684F49884212D15448026810210A43A2
:10CD60000260006808400B900B9811200590032189
:10CD7000002203F0F9F9059802F00CF886E01A9801
:10CD800000684449884212D14848026820210A4379
:10CD90000260006808400A900A981220049003215B
:10CDA000002203F0E1F9049801F0F4FF6EE01A9814
:10CDB00000683949884213D13B4802680121C90300
:10CDC0000A43026000680840099009981320039004
:10CDD0000321002203F0C8F9039801F0DBFF55E0BE
:10CDE0001A9800682D4988421FD1012080050D90B6
:10CDF000002018900DA8F9F77BF8002801D0FEF765
:10CE0000BFF829480268012109040A43026000684A
:10CE1000084008900898142002900022114603F060
:10CE2000A3F9029801F0B6FF30E01A9800681C4997
:10CE3000884213D11C480268012149040A43026058
:10CE400000680840079007981520019003210022F0
:10CE500003F08AF9019801F09DFF17E01A98006825
:10CE60001049884212D110480268012189040A43FE
:10CE70000260006808400690069816200090032182
:10CE8000002203F071F9009801F084FF1BB000BD8F
:10CE9000001000400014004000200040004001400D
:10CEA0000044014000480140401002403C10024054
:10CEB00000B583B01B4801901B490160E121490284
:10CEC000416001210A03826000230293C36089024A
:10CED00001610C2141618361C3610362436283622A
:10CEE00019461A46FAF712FD002801D0FEF748F855
:10CEF0000C48002102F08EFB002801D0FEF740F81C
:10CF00000848002102F0C7FB002801D0FEF738F8DE
:10CF1000044803F0ABFA002801D0FEF731F803B063
:0CCF200000BDC046A40F002000380140F6
:10CF2C0030B59BB01A90002019901890179016905D
:10CF3C00159008A8342100F03DFC1A98006825498A
:10CF4C00884245D1012008900220099008A8F8F7E2
:10CF5C00C9FF002801D0FEF70DF81F480268012117
:10CF6C0089030A43026000680840079007981B4831
:10CF7C00026801210A430260006808400690069886
:10CF8C00092040021590022416940020049017905A
:10CF9C00189001200190199005200007029015A906
:10CFAC000391F8F791F8019A02980399049B950262
:10CFBC0015951694179218931992F8F785F8049A08
:10CFCC001B200590032103F0C9F8059801F0DCFE45
:10CFDC001BB030BD003801404010024034100240FC
:10CFEC000122D20703004B403AD430B4431A01D289
:10CFFC00C01AC9184B004400240EFF2C29D0002C59
:10D00C0024D01B0E20D0E31A182B1DDC090211436F
:10D01C00C40D000210435D4219350A00AA40D20922
:10D02C00D940451801D36D080234013CE405280AA7
:10D03C000121C9072D062A438A4160414100090E8E
:10D04C00FF2901D3C00DC00530BC7047C00FC0070D
:10D05C00FAE74202F8D07F2000010C300005F3E71C
:10D06C00A4465140431A02D25340C01AC9184B006F
:10D07C00090211431B0E4400240EFF2C41D0002B3F
:10D08C0010D05B421B19012B10D322D1C30D4002CF
:10D09C00401A10D3DB050100400AC90591415841E3
:10D0AC00644670472442FBD10020F9E7C30D4002CF
:10D0BC004900401AF4D0002101314000FCD38C42CD
:10D0CC0004D95B1ADB05400AC018E9E7180AC00747
:10D0DC00E6E7192BE4D801330C00D940DC414C4075
:10D0EC00012C4941C30D00021043441A01D4A40081
:10D0FC006408013BDB05200A240694415841644630
:10D10C007047FF2B01D04102CAD07F2000010C30A8
:04D11C000005C5E75E
:10D120000122D2075140014B18470000F1CF0008FF
:10D1300030B405004D400124E407254042004B0077
:10D14000120E32D01B0E3CD0FF2A33D0FF2B3FD023
:10D15000D21800022043000A09022143090AC4B27E
:10D160004C43000AC3B24B43000A4843210A5B18F0
:10D17000190A091801D44900013A080A7F3A2ADB42
:10D18000FE2A0FD2D2051C43240601D001242143DC
:10D19000C9B280295041802901D14008400028436C
:10D1A00030BC7047FF20C005F9E71B0EFF2B0AD0EB
:10D1B0002800F5E7400206D1FF2BF3D1490202D146
:10D1C000F0E7FF2AF4D17F2000010C300005E7E7EB
:10D1D0004902F8D1E6E743020132E9D15B1202339A
:08D1E000E6D9D805E4E7C046DA
:10D1E80030B405004D400124E407254042004B00BF
:10D1F800120E26D01B0E34D0FF2A2DD0FF2B35D08F
:10D20800D21A000220430902214343084908A00D0D
:10D218005B1A02D2013A5B005B185B008B4200D3B9
:10D228005B1A4041F9D37F3222DDFF2A06D2D205AC
:10D23800C91A8B425041284330BC7047FF20C005B3
:10D24800F9E71B0E03D0FF2B12D1490210D07F2023
:10D2580000010C300005EFE74002F8D1FF2BEDD1BB
:10D26800F5E7FF2AEAD14002F1D1E7E74902EED11A
:04D278002800E1E7C2
:10D27C0002000A43520008D0884204D14000012128
:10D28C000906C84201D90020704701207047C046EA
:10D29C00012212064300DA4211D84B00DA420ED8B2
:10D2AC0002000A43520008D003D288428041013068
:10D2BC007047814280410130704701207047002047
:04D2CC007047C046A1
:10D2D000012212064300DA420FD84B00DA420CD882
:10D2E00002000A43520008D003D2814280414042EA
:10D2F0007047884280414042704700207047C046D6
:10D30000012212064300DA420FD84B00DA420CD851
:10D3100002000A43520008D003D2884280414042B2
:10D320007047814280414042704700207047C046AC
:10D330004A0010D2520D03231B02FF33D21A0AD423
:10D3400052421F3209D4400DC90208430123DB07B2
:10D350001843D040704700207047D0177047C04630
:10D36000420017D2120E7F3A14D480231B06202AC3
:10D3700006DA52421F3200021843D04000217047A3
:10D3800052423F3209DB010219430800D041D1402B
:10D3900048407047002001007047D01701007047D7
:10D3A0009D2201000AD002D4013A4900FCD5D205E1
:10D3B000080A0906494100D3012950417047C04677
:10D3C00042221201033A010007D002D4013A0018A8
:0CD3D000FCD51205C30A400599187047EF
:10D3DC00BD22094210D003D4013A00184941FBD5B3
:10D3EC00D2050128804101300143080A0906494150
:10D3FC0000D301295041704700490847A1D30008C8
:10D40C004B1801225205DA4217D25B0D0722D201CA
:10D41C009B1A0FD9FF2B13D2DB05CA0FD20713436C
:10D42C000903020D1143490AC200524100D90131CE
:10D43C00C8187047C80FC007704706D1002804D120
:10D44C00C80F0002FF30C00570470123DB070A003C
:10D45C00C900400F084398431A4010435B0A184315
:04D46C007047C046FF
:10D47000F0B581B00A464149C30D5C1EFD2C59D858
:10D48000FD24E443D50DFF3DA54253D306460E408F
:10D49000491C0140964261D90091DCB20123DD05AF
:10D4A000002C03D0691E0840284309E0AE4206D292
:10D4B0009F05641E7000BE420646FAD300E0304667
:10D4C000D10DCEB2002E03D0691E0A402A4309E0D6
:10D4D000AA4207D29F051146761E4A00B94211465C
:10D4E000FAD3FFE7B4420ADD811A02D4904201D197
:10D4F00009E00146641E4800B442F5DC3446861A51
:10D5000003D4904202D1009A11E00646AE4206D200
:10D510009905641E70008E420646FAD300E030463C
:10D52000002C1FDD611E009A8018C90542181046A4
:10D5300001B0F0BD4500124CA5421BD25500AC42D3
:10D54000F5D906460E40FF24E5050E4CAE4213D039
:10D55000002E0BD10A420246E9D10DE000D001466F
:10D560000A46E4E7191BC8400021DCE70A4003D063
:10D57000AA428DD10246DAE72246D8E7FFFFFF7FB5
:08D58000010000FF0000C07F64
:10D58800C10DC9B24A1EFE2A19D27E2903D8002825
:10D5980013DA104870479529FCD87F390C4A0A419C
:10D5A8000240134603D5094B5B1CCB40D318884077
:10D5B800400200D01A4610467047002070470029E4
:10D5C800E8D10121C90708407047C046FFFF7F0026
:08D5D800000080FF000080BF8D
:10D5E00030B5514343435C18010C130C0D005D43EF
:10D5F000641992B2514380B242430D0C090452188F
:10D6000065415843010C00048018694130BDC04693
:10D61000CA1751408B1A17D0C1174A409446484048
:10D62000411A48081A0000E052008242FCD900204A
:10D6300000E05208914200D3891A40419A42F8D141
:10D6400062465040801A704710B500F07DF810BD5A
:10D6500007B5FFF7DDFF0EBC4243891A00BDC04687
:10D660000A0015D00300400800E052008242FCD9B5
:10D67000002000E052089B1A06D340418A42F9D1AB
:10D68000704752089B18F8D200188A42F9D17047A7
:08D6900010B500F059F810BDBF
:10D6980038B504004D42FFF7DFFF4543611938BD37
:10D6A800002B09D1002907D110B51100FFF7F0FFB1
:10D6B8000A000021002310BD70B400240125ED07E5
:10D6C800002B07D1002905D0834203D21300002282
:10D6D8002C0000250026A419994200D1904212D9A5
:10D6E80092185B4103D2EE076D086408F3E7DE0782
:10D6F8005B08520892190126F6079B1903E0DE071A
:10D708005B0852089219801A994103D364416D410C
:10D71800F5D30FE024196D410AD2DE075B085208E1
:10D72800921980185941F5D364416D41E7D301E05E
:10D738008018594102000B002000290070BC704776
:08D74800002000217047C046DB
:10D7500003490868002800D07047024808607047F5
:08D76000E81300204006002040
:10D768007F2805D8034A125C0348405C1040704784
:0CD7780000207047EB1301083E1101086F
:10D784007F2805D8034A125C0348405C1040704768
:0CD7940000207047EB1301083E11010853
:10D7A000411C02780130002AFBD1401A7047C04664
:10D7B000002A03D0013A8B5C8354FBD17047C046EA
:10D7C00000220B0011001A00002A02D0013A8154F5
:04D7D000FCD17047D1
:10D7D400F0B581B00022002933D00378002B30D07B
:10D7E400032302469A4316680024E5438707FF0E85
:10D7F400BD40ED43354306461E407118042900938D
:10D804000AD3124EAF19104BAB433B4204D1091F4C
:10D814005568121D0329F5D82B060DD02B041B0EB9
:10D8240007D02B021B0E06D02B0E009C04D0042420
:10D8340002E0012400E002248C4200D30C46101ABA
:10D844000219104601B0F0BD80808080FFFEFEFE0C
:10D85400F0B581B004467F20C605002C00960FD099
:10D86400E11722464A40571AC6050A4DF80704D064
:10D8740029683046FFF75AFC06462D1D7F08F5D16E
:10D8840000983146FFF7AEFC002C00D4304601B0BE
:08D89400F0BDC046F8E90008F0
:10D89C00F0B503AF93B06E46F51D2135F41D393448
:10D8AC0074613362F261F160306100F003FFB060CB
:10D8BC00C21D07218A436946B1616946881A7060A6
:10D8CC008546F41D1D34002124222046FFF776FFE7
:10D8DC000B487169F2680A6048600A482860306930
:10D8EC002862B06868617068E8602046F169326A45
:10D8FC0000F01EF8B1698D46FC1F053CA546F0BD35
:08D90C0071080108FFFFFF7F15
:10D9140083B010B581B0044603A80EC00548006862
:10D9240003AA0092214602F086FA01B010BC02BCA0
:08D9340003B00847680600205B
:10D93C00F0B59FB014460F460021159001600120F0
:10D94C0002020C92460282020392C202029203224B
:10D95C000A929202059202031792420307928203E3
:10D96C0004920090C00316900891C84301900F9642
:10D97C003978252908D0002901D100F067FE7F1CD9
:10D98C00159802F0F7F9F3E7FF1C089BB81E057811
:10D99C002A46203A102A2BD880219200184602A33E
:10D9AC009A5803469746C046F9D9000819DA000878
:10D9BC0019DA000813DA000819DA000819DA000875
:10D9CC0019DA000805DA000819DA000819DA000873
:10D9DC0043DA000809DA000819DA00080DDA000841
:10D9EC0019DA000819DA000811DA000840210AE0F7
:10D9FC005E2D179907D009E0169904E0202102E06A
:10DA0C00102100E031460B437F1CBFE77F1E2946E7
:10DA1C003039C9B20929139419D800240A21614359
:10DA2C006C18303C791C3D782A46303AD2B20A2A1E
:10DA3C000F46F3D30CE001CC0028139401D5102130
:10DA4C000B43C1174840441A781E057800E00024A7
:10DA5C0000202E2D08D13D782A2D07D17D78BF1CB2
:10DA6C00139901C9139113E00E9018E07F1C2946FD
:10DA7C003039C9B209290FD80A2141436818303806
:10DA8C00791C3D782A46303AD2B20A2A0F46F3D393
:10DA9C0000280E9001D502E00E900C980343184616
:10DAAC00E1172A46683AD301D2B252089A18D2B278
:10DABC00092A2BD8920002A39A5803469746C046CF
:10DACC00F5DA0008FFDA000809DB000829DB00089A
:10DADC0029DB000829DB000803DB000829DB000830
:10DAEC0029DB000803DB00083D78682D10D10820E5
:10DAFC0008E0022003433D787F1C0FE03D786C2D3D
:10DB0C0009D1022003437D78BF1C07E0034605E0E2
:10DB1C007F1C042201E07F1C012213438C43462D01
:10DB2C000B941BDD2946633915292BD8139CC04651
:10DB3C007944097949008F44460B421CC30A0B0AED
:10DB4C000A0A0A5966730A0A810A830A0A2E0FE71F
:10DB5C00049803430021099119467AE0442D159845
:10DB6C00139C08DD452D28D0462D00D000E70798E2
:10DB7C000343029824E0252D00D081E2252102F0F8
:10DB8C00F9F8F5E6472D139C00D197E0582D00D0FD
:10DB9C00EEE607980343CE4A782D00D120321906C1
:10DBAC00C81709900C98034201D0CA480340194683
:10DBBC000498099B134009934BE00798034303987F
:10DBCC000343059A7EE0264624780B98421E159D49
:10DBDC00284619461292149302F01EF92846214643
:10DBEC0034460F9E02F0C6F8241DDFE0180700D55E
:10DBFC004AE29807159801682068016000D447E252
:10DC0C000021416044E20C980342194601D0B1480E
:10DC1C0001401A06D217302010400990049818E0E1
:10DC2C00069718060C990B43C01723210140099144
:10DC3C0004CC1394002708200E90B3E101CC8DE0A6
:10DC4C000C98034201D0A3480340194604980022C3
:10DC5C00099202220A400142069706D1002A09D1F4
:10DC6C00231D002722461C460AE0002A12D104CCB0
:10DC7C00D01715E0E21D07239A4357681446083461
:10DC8C0013684A0714D408220A4000D0DBB2002AD9
:10DC9C000FD1FCE0E41D072294432268606808342D
:10DCAC004B0708D40B0700D5DDE013460746DDE033
:10DCBC009BB20027EBE013B21204D6E007980343A3
:10DCCC00059A13430C98034201D00E9800E00620ED
:10DCDC0014931340991A4A424A410E92002800D0DC
:10DCEC000E90E41D0720844303CC083CFFF788FB0F
:10DCFC002546044602F037F80835139500282046CF
:10DD0C000ED00021FFF7F6FA149B1A4607990A4029
:10DD1C00002813D0002A704800D07048139C1BE0D8
:10DD2C0002F018F8002846D00798149B03426C4860
:10DD3C0000D06C486C490B40139C0FE0002A6B49D7
:10DD4C0000D06B49002A01D0694800E06748139C59
:10DD5C00401C9A0600D5084663490B400028654EC6
:10DD6C0000D0064619465B48014014910C980342BA
:10DD7C001394304602D1FFF70DFD02E00E99FFF728
:10DD8C0023FD05460B98441B15981499224602F066
:10DD9C0043F8002D129407D0159C3178204601F0E1
:10DDAC00E9FF761C6D1EF8D1139C0F9E1498C006CB
:10DDBC0000D4DDE55EE10126204602F0DBFC0546E1
:10DDCC00002801D0F007444012961EA9204602F00C
:10DDDC00EFFC1E980A9948430A21FFF713FC0646EC
:10DDEC001E90002D03D0602014990143149100253E
:10DDFC0020462946FFF73CFA002818D1701CFFF783
:10DE0C0023FD01462046FFF75DFA00281E9806D038
:10DE1C00411C1E91801CF2E71E98401E1E90FFF7BD
:10DE2C0013FD01462046FFF765FA0028F4D1149A39
:10DE3C0016460598064012998B029E4200D129E1A4
:10DE4C00864209D11E980E99814200DC23E10421FF
:10DE5C00C943884200DC1EE112930398024200D0B1
:10DE6C0021E10E9D0AE253B21206D717002F05D4FA
:10DE7C008A060AD44A060AD5202007E000225B4213
:10DE8C00BA412D200990174601E02B2009901A4623
:10DE9C000C98014201D00F4801400B460C980142EE
:10DEAC00139401D00E9800E0012000246E2D0E90EA
:10DEBC0039DD6F3D092D00D995E0C0467D442D79A3
:10DECC006D00AF44196F909090903690906FC04653
:10DEDC0058300000FFFDFFFF501101084B110108E5
:10DEEC008F1401088B140108FFFEFFFF5A11010863
:10DEFC00551101088C0B01081046384373D0D0081B
:10DF0C0079074018014607201040303018AA1055E8
:10DF1C00C808FF087A0780180A463A43641C002A8E
:10DF2C000A46EFD15FE0582D3CD0642D01D0692D0D
:10DF3C0059D11046384356D01946169801400D91C8
:10DF4C000021149314463B460D9800280F4608D028
:10DF5C0008460A990840032803D118A82C21C1555A
:10DF6C007F1C0A26002520461946324612932B4662
:10DF7C00FFF794FB10940446119132462B46FFF7A1
:10DF8C0029FB109A101A3021014318A8C155791C8D
:10DF9C000920801A12988541119F0F9E149BD2D391
:10DFAC000C4620E0104638431CD007981D4603420F
:10DFBC00F94800D0F948134611093A07891800248A
:10DFCC000A460F211940415C18AB195511093F093C
:10DFDC003B07C91813463B43641C002B1346EFD177
:10DFEC002B4600E00024099A511E104688410B99DB
:10DFFC00091BFF2A00D9491E069F081A0E990D1BF2
:10E00C00E9178D43421B3342149305D115981946D9
:10E01C0001F002FF149B0022099E310A129204D0D7
:10E02C00159801F0A7FE129A149B002E3146159EEE
:10E03C0004D0304601F09EFE129A149B30461946CD
:10E04C0001F0EAFE302130462A4602F0FDFB012C9D
:10E05C000ADB641C18A80019801E0178304601F0F8
:10E06C0089FE641E012CF5D81498C006139C0F9ED3
:10E07C0000D47DE420211598129A02F0E5FB77E498
:10E08C00002D00D074E4F1E2206815990968017044
:10E09C00241D6DE41E98119626282FD12046CE49BA
:10E0AC00FFF79CF830E01E980E2800DDE6E0C04338
:10E0BC000E990E18102E00DB10261498000600D5B1
:10E0CC00DBE0002E354600D1D8E03046FFF7BCFB34
:10E0DC002146FFF727F83F210906FEF781FFFFF7DE
:10E0EC004DFABE49FFF7BEF900252946FFF7C0F8E7
:10E0FC00002800D1C1E0761EE7D1BFE04042FFF717
:10E10C00A3FB2146FFF70EF8064600252946FFF72C
:10E11C00AFF80028139C15D1304601F024FE0028DE
:10E12C00304611D00021FFF7E5F8149B1A460799E9
:10E13C000A40002800D198E0002AA94800D10BE63B
:10E14C00A84809E6099527E00995A44C2146FFF754
:10E15C009FF81E9D00280BD030462146FFF73EF855
:10E16C0006462146FFF794F86D1C0028F4D11E9545
:10E17C007F20C40530462146FFF7BCF800280BD0A1
:10E18C0030469649FEF7CEFF06462146FFF7B2F819
:10E19C006D1E0028F4D11E950598119981420E9898
:10E1AC0001D0054600E0451E8C4C0028294600D1C4
:10E1BC00014611914842FFF747FB019902F0DCFA46
:10E1CC003146FEF70DFF06462146FFF761F80028A1
:10E1DC0007D01E98401C1E9030462146FEF7FEFFCD
:10E1EC000646149A11980D9600283BD01195029969
:10E1FC000B46803313408B4200D0AEE0102800DB7E
:10E20C0010200546FFF720FB0D99FEF78BFFFFF75B
:10E21C00A1F8109008430998119000D19DE00A22B2
:10E22C00002310980E46FFF739FA002D00D193E029
:10E23C001A4300D090E0119531460A25002610981B
:10E24C002A463346FFF72AFA10900C462A463346E4
:10E25C00FFF724FA1198401E11907ED01A432146E4
:10E26C00EBD07AE00998119077E0002A5E4900D053
:10E27C005E49002A6ED05D486AE535461E98103816
:10E28C006942884200DC0846FFF7DEFA019902F089
:10E29C0073FA2146FEF7A4FE04461E98401CFFF7B5
:10E2AC00D3FA01462046FFF70DF81E99002800D03E
:10E2BC00491C14980029119511D4112914D308461E
:10E2CC0010381E901020401AFFF7BEFA2146FEF7B8
:10E2DC0029FFFFF73FF806460C46002012E00D948C
:10E2EC0000261E9634460FE000201E902046FFF7B5
:10E2FC0031F8254606460C46FFF76AF801462846D3
:10E30C00FEF708FF0D90149812998843DC490831E8
:10E31C0000250A4608326D1C0B684968F31A23461F
:10E32C008B411146F6D21095119B002B0099149A33
:10E33C0001D1D1B2C9095206920F01D1494200E074
:10E34C00C9431E9A891A0B9AD21A5118109A891A13
:10E35C00024675E0C748FBE41195119D002D00980D
:10E36C00149A01D1D0B2C0090B99491B081A411F4C
:10E37C001E9C17980242129E01D110963EE00E91FF
:10E38C00032120461091FFF75DF9881C042820D842
:10E39C0003A1085C400087447B1401086B1401083E
:10E3AC0006122B061200641E1E940D98B249FEF73D
:10E3BC00B9FE0D900E99491E022010901BE0A41E70
:10E3CC001E940D98AD49FEF7ADFE0D900E99891E69
:10E3DC0011E000200DE0C0469976967E00002041A9
:10E3EC00501101084B1101085A110108551101086F
:10E3FC00012010900E99149AE81785435006800F4F
:10E40C00119500D0491E0E91F502204602F0E2F95A
:10E41C00632802DD0E98401E0E9014980D9CA843A4
:10E42C0014902046FEF796FF254606460C46FEF74E
:10E43C00CFFF01462846FEF76DFE149A0D900E99FB
:10E44C00C8170D4685430F9810300242149209D11B
:10E45C00012907DB2021159801F08CFC6D1EF9D1E8
:10E46C000025149A40201040910603D400280AD0AD
:10E47C00202104E0002801D02D2100E02B2115984B
:10E48C0001F078FC149AD0060AD4002D08D0302163
:10E49C00159801F06FFC6D1EF9D100200E9000E074
:10E4AC000E951099491E0D46C800754A11184968F9
:10E4BC001258B01A2046884101D2302007E0302093
:10E4CC00B61A8C41401CB31A23468B41F8D2C1B208
:10E4DC00159801F04FFC2946002D1498E2D1014605
:10E4EC00029801401291159E0BD01E98012808DB52
:10E4FC00401E1E903021304601F03CFC1E98002836
:10E50C00F6DC802014990840119C20430E9D4BD0C2
:10E51C002E21304601F02EFC102C264600DB102656
:10E52C00F017344684431298002801D1204601E0AC
:10E53C001E98201AFFF788F9014611981094001BB9
:10E54C000B90012E23DB0D98FEF7ECFDFEF702FF7E
:10E55C0004460E46109B5B1ED800494A11184968A8
:10E56C001258A01A30468841129301D2302007E08D
:10E57C003020A41A8E41401CA31A33468B41F8D28A
:10E58C00C1B2159801F0F6FB129B002BE3D10B984E
:10E59C000028159E119807D010990C1A302130467E
:10E5AC0001F0E8FB641CF9D30398149901423DD0A7
:10E5BC000798014201D0452100E06521159C2046B9
:10E5CC0001F0D8FB1E980028204604D42B2101F022
:10E5DC00D1FB1E9805E02D2101F0CCFB1E9840428A
:10E5EC001E90642810DB64242146FFF733F80146A3
:10E5FC003031159E304601F0BDFB1E982146FFF7C9
:10E60C0021F808461E9100E0159E0A242146FEF7CB
:10E61C00F9FF01463031304601F0ACFB1E98214623
:10E62C00FFF710F83031304601F0A4FB002D139C9D
:10E63C000F9E01D1FFF79CF9159C2021204601F07B
:10E64C0099FB6D1EF9D1139CFFF792F9159CE068AC
:10E65C00002805D006CC083C914201D2089A4254BD
:10E66C00204601F0CCFB20681FB0F0BD01F0C7FBC9
:10E67C000198F9E75A110108000020410000C84236
:04E68C00C030000892
:10E69000084B1B6883420AD0074B1B68834206D095
:10E6A000064B1B68181A431E9841404270470020D1
:10E6B000FCE7C0466C0600206806002070060020BB
:04E6C000402070473F
:0CE6C40010B5006800F0CAF810BDC04698
:10E6D00003231048104A03614361104B8261C361F8
:10E6E0008023DB000362002383624362C36202660D
:10E6F0000B4A53214266102282660367094AC366A9
:10E70000436700E0D17BC1540133013A102BF9D1AA
:10E710007047C046FC0E00203CEB0008C0080020FB
:08E720005413002048EB00082F
:10E72800F8B54746CE46C5688368040040689946F0
:10E738005B1B80B50E00170098464019934207D915
:10E74800FFF732F8ED19E560C0BCB946B046F8BD30
:10E758001A00FFF729F84B463100ED19ED1A2A0087
:0CE7680060684144FFF720F8EDE7C04670
:10E77400F8B54746CE46002380B588460700160004
:10E784009946C56884681BE0013B5B1B641BB4426B
:10E7940000D934009C4200D91C007868220041460C
:10E7A4004019FFF703F82D19A144A044361BBC6897
:10E7B400631B5A1E93415B421D40FD60002E06D030
:10E7C4003B699D42E0D3013B1B195B1BDEE74846D6
:08E7D400C0BCB946B046F8BD17
:10E7DC0070B50600431C5C00E418E00074001C4B90
:10E7EC00A419E400C0181B19DC6A1500012C06D012
:10E7FC00022C1FD0002C10D00024200070BD9A6A6F
:10E80C005C6AA2421FD9013A121B2C00954200D916
:10E81C0014002200FFF782FFEFE79A6A5E6AB242A9
:10E82C000CD9013A961BB542E7D82A00FFF776FFC0
:10E83C002C00E2E7FFF798FF0400DEE71B6AD21812
:10E84C00013A961BEFE71B6AD218013A121BDCE760
:04E85C00FC0E00208E
:10E86000F8B50B4B04001B780D001600002B0CD0E4
:10E87000EFF31087012181F3108832002900200076
:10E88000FFF7ACFF87F31088F8BDFFF721FFEFE734
:04E89000FC0E00205A
:10E89400F8B5050008000C00FEF780FF0A4B0600DF
:10E8A4001B78002B0CD0EFF31087012181F3108823
:10E8B400320021002800FFF78FFF87F31088F8BD8E
:0CE8C400FFF704FFEFE7C046FC0E002049
:10E8D000004B0000650001000100E803000000009B
:10E8E000000038004C00E902AE014A023F02B800C5
:04E8F0000000000024
:08E8F4000A000000B80B00004F
:08E8FC000100000064000000AF
:08E904000A000000B80B00003E
:08E90C0001000000640000009E
:08E914000A000000B80B00002E
:08E91C0001000000640000008E
:08E924000A000000B80B00001E
:08E92C0001000000640000007E
:10E934000A000000B80B0000B80B0000B80B000080
:10E944000100000064000000640000006400000096
:10E954000A000000B80B0000B80B0000B80B000060
:10E964000100000064000000640000006400000076
:0CE97400710E0108A0E9000880E900080D
:10E9800069D70008250801083108010885D7000863
:10E990003D0801084908010815080108E9070108B0
:10E9A000730E01082B1101082B1101082B1101080E
:10E9B0002B1101082B1101082B1101082B11010843
:10E9C0002B1101082B110108FFFFFFFFFFFFFFFFC5
:10E9D000FFFFFFFFFFFF0000750E0108DD100108BB
:10E9E0001F0B0108FA100108760B01082C11010811
:08E9F000351101087D0B01083F
:10E9F800000020410000C84200401C4620BCBE4C1C
:08EA0800CA1B0E5AAEC59D7435
:10EA1000034C206804348047FBE7FAF785F9FEE7EA
:04EA20009414010841
:04EA24007131000844
:10EA280087B006900591049203A9002008701F2062
:10EA380002900299481E029000200029019009D0F6
:10EA4800059802991F221140C840012108404142FF
:10EA5800484101900198C007002800D0E9E70498D0
:10EA6800009018284CD80098810001A0405887468B
:10EA780007EB000809EB000809EB000809EB0008A0
:10EA880009EB000809EB000809EB000809EB00088E
:10EA9800F9EA000809EB000809EB000809EB00088F
:10EAA80009EB000809EB000809EB000809EB00086E
:10EAB800EBEA000809EB000809EB000809EB00087D
:10EAC80009EB000809EB000809EB000809EB00084E
:10EAD800DDEA00080298072802D303A9012008707C
:10EAE80011E00298082802D303A9012008700AE05F
:10EAF8000298102802D303A90120087003E002E05D
:10EB080003A90120087003A8007800280DD10598F2
:10EB18000699096848610698006880681821884342
:10EB28000499084306990968886003A8007807B023
:02EB3800704724
:02EB3A00FEE7F4
:09EB3C005465726D696E616C0094
:03EB45003A200073
:10EB480000000000000054545220524547474553E6
:01EB580000BC
:10EB59004465766963652049443A20756E6B6E6F2A
:03EB6900776E00C4
:02EB6C00FEE7C2
:02EB6E00FEE7C0
:02EB7000FEE7BE
:02EB7200FEE7BC
:02EB7400FEE7BA
:02EB7600FEE7B8
:02EB7800FEE7B6
:02EB7A00FEE7B4
:02EB7C00FEE7B2
:02EB7E00FEE7B0
:02EB8000FEE7AE
:02EB8200FEE7AC
:02EB8400FEE7AA
:02EB8600FEE7A8
:02EB8800FEE7A6
:02EB8A00FEE7A4
:02EB8C00FEE7A2
:02EB8E00FEE7A0
:02EB9000FEE79E
:02EB9200FEE79C
:02EB9400FEE79A
:02EB9600FEE798
:06EB9800F4F7E2FA38E791
:10EB9E0081B000900098806804210840800801B080
:02EBAE007047AE
:10EBB00083B002900191009202984069019A042169
:10EBC0000A400721914088430099914008430299E7
:06EBD000486103B070472C
:10EBD60000B583B0019001980068FFF7DDFF0028BB
:10EBE6002CD00198006800F0C9F8002803D10198DC
:10EBF6000068F5F746FCF4F706FC009001980068FB
:10EC060080684007002819D5F4F7FDFB0099401AE3
:10EC1600032812D3019800688068400700280CD5A5
:10EC26000199886D102210438865019AD16D0120E3
:10EC36000143D16502A9087003E0DFE702A90020BD
:0AEC4600087002A8007803B000BDBA
:10EC500000B583B0019001985421405C012803D194
:10EC600002A90220087024E001995422012088544E
:10EC70000198FFF7B0FF0146684601700078002850
:10EC800010D1019801F0F8F801466846017000784B
:10EC9000002807D10198806D0121084309028843AB
:10ECA000019988650199542200208854009802A98E
:0AECB000087002A8007803B000BD50
:10ECBA0081B000900098C06803218902084041424F
:06ECCA00484101B0704753
:10ECD00000B583B002900298806A0190019801F01B
:06ECE000DDF903B000BDE8
:10ECE60000B583B002900298806A01900199886D00
:10ECF6004022104388650199C86D04221043C865F7
:0AED0600019801F0C4F903B000BD4C
:10ED100083B00290019100920298806A019A1F21AB
:10ED20000A400F2319469140884300999B061940D9
:0EED3000890E914008430299886203B0704733
:10ED3E0081B000900098006807218905084001B055
:02ED4E0070470C
:0EED500081B0009000998020086001B07047EB
:10ED5E0081B000900099486880221043486001B04D
:02ED6E007047EC
:10ED700081B000900099486880229043486001B0BB
:02ED80007047DA
:10ED820081B000900098806802210840400801B0DC
:02ED92007047C8
:10ED940000B581B001466846017000214056F5F780
:06EDA40043FC01B000BDBC
:10EDAA0000B581B001466846017000214056F5F76A
:06EDBA004CFC01B000BD9D
:10EDC00000B583B001900198002803D102A9012069
:10EDD000087014E001980079002805D101990020FD
:10EDE00048710198F9F720FA0199022008710199F8
:10EDF00000200861019A0121117102A9087002A87E
:06EE0000007803B000BD24
:10EE060082B00190009101980068806B00991022F1
:0EEE160011401F228A401040C84002B07047D1
:10EE240000B587B0059004910392029301A90020D4
:10EE3400087005982421405C012803D106A902200A
:10EE4400087030E005992422012088540598252172
:10EE5400405C01281AD1059925220220885405997D
:10EE64000020C86305980168086801220092904355
:10EE7400086005980499039A029BF5F751FE009ADD
:10EE84000598016808681043086009E00599802026
:10EE9400C863059924220020885401A90120087020
:0EEEA400019806A9087006A8007807B000BD06
:10EEB20000B587B0059004910392029301A9002046
:10EEC200087005982421405C012803D106A902207C
:10EED20008705EE0059924220120885405982521B6
:10EEE200405C012848D105992522022088540599C1
:10EEF2000020C863059801680868012290430860F1
:10EF020005980499039A029BF5F70BFE0598006B8E
:10EF1200002806D00598016808680E221043086090
:10EF22000BE0059801680868042290430860059880
:10EF3200016808680A22104308600598406C00685E
:10EF4200C003002806D50598416C08680122120208
:10EF5200104308600598006D002806D00598016DE1
:10EF620008680122120210430860059801680868C7
:10EF720001221043086009E005998020C8630599C1
:10EF820024220020885401A901200870019806A9B2
:0AEF9200087006A8007807B000BD63
:10EF9C0084B0009101460098039102A9088003985F
:10EFAC0000690988084203D001A90120087002E019
:0EEFBC0001A90020087001A8007804B0704779
:02EFCA0070478E
:02EFCC0070478C
:10EFCE0000B583B001900198002803D102A9012059
:10EFDE0008703EE001983D21405C002806D1019961
:10EFEE003C22002088540198FDF793FE01993D22A2
:10EFFE0002208854019901C9F7F7DDF801994822DA
:10F00E000120885401993E220120885401993F2203
:10F01E0088540199402288540199412288540199BB
:10F02E004222885401994322885401994422012096
:10F03E008854019945228854019946228854019991
:10F04E004722885401993D220120885402A90020AC
:0AF05E00087002A8007803B000BD9E
:10F0680085B00490039102920193049880680090FF
:10F078000098FF2109028843009003990298019A99
:10F088001202104301430098084300900098049925
:06F09800886005B070471E
:10F09E0081B0009000982821405CC00700280AD05B
:10F0AE000098006840680121490488430099CA6AA3
:10F0BE0010430968486000982821405C80070028AA
:10F0CE000AD5009800684068012109048843009918
:10F0DE000A6B10430968486000982821405C40077D
:10F0EE0000280AD5009800684068012189048843E9
:10F0FE0000994A6B10430968486000982821405CCB
:10F10E00000700280AD50098006840680121C9034D
:10F11E00884300998A6B104309684860009828213B
:10F12E00405CC00600280AD500980068806801215E
:10F13E00090388430099CA6B1043096888600098D8
:10F14E002821405C800600280AD500980068806857
:10F15E0001214903884300990A6C104309688860AD
:10F16E0000982821405C4006002819D500980068B8
:10F17E004068012109058843009A536C18431268B0
:10F18E0050600098406C88420AD100980068406830
:10F19E0003214905884300998A6C10430968486029
:10F1AE0000982821405C000600280AD500980068C7
:10F1BE0040680121C90488430099CA6C104309684C
:06F1CE00486001B070472B
:10F1D40010B596B0189C0890079106A80270059384
:10F1E40008980068C06907990840401A414248419C
:10F1F40006A90978884200D098E01898401C002895
:10F2040000D192E0F4F700F90599401A1899884260
:10F2140002D81898002838D1EFF310800D900D987B
:10F22400049001201590159880F3108808980168BF
:10F2340008680D22520190430860049814901498B1
:10F2440080F31088EFF310800C900C980390012247
:10F254001392139880F31088089801688868904383
:10F26400886003981290129880F310880899842279
:10F2740020208850089988228850089980220020EC
:10F28400885409A90320087053E0089800680068AE
:10F294004007002849D508980068C0690121C902BF
:10F2A4000840C00A012840D1089801680120C00222
:10F2B4000862EFF310800B900B98029001201190DC
:10F2C400119880F310880898016808680D2252018B
:10F2D4009043086002981090109880F31088EFF320
:10F2E40010800A900A98019001220F920F9880F3DF
:10F2F40010880898016888689043886001980E9087
:10F304000E9880F310880899842220208850089948
:10F314008822885008998C228850089980220020DD
:10F32400885409A90320087003E059E709A90020BB
:0AF33400087009A8007816B010BD9B
:10F33E0089B0029002988421405821283DD102982C
:10F34E005621405A00282AD1EFF3108004900498D9
:10F35E00019001200890089880F3108802980168A7
:10F36E00086880229043086001980790079880F300
:10F37E001088EFF310800390039800900120069000
:10F38E00069880F31088029801680868402210439E
:10F39E00086000980590059880F310880DE002999A
:10F3AE00086D0078096888620299086D401C08652E
:0EF3BE0002995622885A401E885209B07047A4
:10F3CC0000B591B0079007986021405A05A90880B4
:10F3DC00079888214058222800D07CE007980068C4
:10F3EC00406A04A908800798806D069004980599D6
:10F3FC000840069908800799886D801C8865079AD3
:10F40C005E21505A401E50520798405A002861D134
:10F41C00EFF310800A900A98039001201090109836
:10F42C0080F31088079801680868092252019043FC
:10F43C00086003980F900F9880F31088EFF31080FA
:10F44C0009900998029001220E920E9880F3108870
:10F45C000798016888689043886002980D900D9811
:10F46C0080F3108807998822202088500799002063
:10F47C0008670798C06E012829D107990020C86633
:10F48C00EFF3108008900898019001200C900C98D4
:10F49C0080F3108807980168086810229043086070
:10F4AC0001980B900B9880F3108807980068C0693E
:10F4BC00102108400009012803D107980168102089
:10F4CC00086207985C21415A00F0BCFF02E00798E3
:10F4DC0000F0C2FF05E00798016888690822104314
:06F4EC00886111B000BDB3
:10F4F20000B58FB0059005986021405A04A9088094
:10F50200059888214058222800D07AE005980068A2
:10F51200406A03A908800398049908400599896DF7
:10F5220008700599886D401C8865059A5E21505ABD
:10F53200401E50520598405A002861D1EFF31080C6
:10F5420008900898029001200E900E9880F310887F
:10F5520005980168086809225201904308600298E0
:10F562000D900D9880F31088EFF3108007900798A4
:10F57200019001220C920C9880F310880598016882
:10F5820088689043886001980B900B9880F31088EC
:10F59200059988222020885005990020086705983F
:10F5A200C06E012829D105990020C866EFF31080AA
:10F5B20006900698009001200A900A9880F310881D
:10F5C2000598016808681022904308600098099025
:10F5D200099880F3108805980068C06910210840D6
:10F5E2000009012803D105980168102008620598D6
:10F5F2005C21415A00F02BFF02E0059800F031FF38
:10F6020005E00598016888690822104388610FB0F7
:02F6120000BD39
:10F6140000B585B00390029103988021405C0128D5
:10F6240003D104A9022008702FE00399802201204D
:10F6340088540399842200922420885003980068F7
:10F6440000680190039801680868012290430860EB
:10F654000398006880680721490788430299084392
:10F664000399096888600398F8F7B4F9009A019837
:10F67400039909680860039920208850039980221F
:10F684000020885404A90020087004A8007805B05C
:02F6940000BDB7
:10F6960000B585B00390029103988021405C012853
:10F6A60003D104A9022008702FE0039980220120CB
:10F6B6008854039984220092242088500398006875
:10F6C6000068019003980168086801229043086069
:10F6D6000398006880680721490688430299084311
:10F6E6000399096888600398F8F773F9009A0198F6
:10F6F600039909680860039920208850039980229D
:10F706000020885404A90020087004A8007805B0D9
:02F7160000BD34
:10F7180030B58FB0139C129C0E900D910C920B93E8
:10F728000D98002803D50D984042089001E00D98E7
:10F7380008900898099001200A9009980C99884225
:10F7480008DB09980C99FDF75FFF09900A98401C9F
:10F758000A90F2E70B980A99884201D90B980A9007
:10F76800129800280AD00D98002804D413A800780D
:10F778004007002802D51298401E129013A800785E
:10F788008007002802D50B98002829D013A80078F4
:10F79800C007002824D11298002821D012990020EF
:10F7A800002907900BD00A99129A0120002305938B
:10F7B8009142069001D305980690069807900798FD
:10F7C800C00700280CD01298401E12900E982021D5
:10F7D80000F07EFE0E98C068002800D500E0DDE746
:10F7E8000E98C068002858D40D98002807D50D98A1
:10F7F80040420D900E982D2100F06AFE09E013A8F2
:10F8080000784007002804D50E982B2100F060FEF0
:10F81800FFE70E98C06800283FD413A80078800737
:10F8280000282CD513A80078C007002827D10B98EA
:10F83800002824D11298002821D0129900200029EC
:10F8480004900BD00A99129A012000230293914246
:10F85800039001D302980390039804900498C0077A
:10F8680000280CD01298401E12900E98302100F0FB
:10F878002FFE0E98C068002800D500E0DDE70E983E
:10F88800C068002809D40E980D990C9A0B9B129CFD
:0EF89800139D01950094F8F7A1FA0FB030BD52
:10F8A60082B000B585B0079306920490039106A82E
:10F8B60001900498039901AAF8F7D3F802900298E8
:0AF8C60005B002BC02B08E46704788
:06F8D000F920C0007047A2
:10F8D60010B596B008A803903821FDF76EFF0020FA
:10F8E6000190079006900590049001200290400236
:10F8F600F5F7F3FD019A029903980B2308930B047D
:10F9060009930B020B930323DC020C9440240D9401
:10F916000E9102240F9410931192102212924A040F
:10F9260013924A06149249071591F5F710FE00281E
:10F9360001D0FBF722FB072004900221059100204D
:10F946000690079004A8F6F7F6F8002801D0FBF712
:0AF9560014FBF6F7A0FA16B010BD7E
:10F9600000B587B006AB1880059104A8028000207E
:10F970000390039806A90988884218DA059804A913
:10F9800001910988012200F06FFCFF204E300290A7
:10F99000F3F742FD019905980988002200F064FC04
:10F9A0000298F3F739FD0398401C0390E1E707B094
:02F9B00000BD98
:10F9B20030B587B004460D980C9D0B9D0A9D0694A8
:10F9C20005910492039302A90880F3F71EFD0190AA
:10F9D200059800680399884248D20498006800900C
:10F9E200002806D00098012811D00098022827D0BC
:10F9F2003BE00C9802A90988012200F034FC01982E
:10FA02000699086004990868401C08602DE0019876
:10FA120006990968401A0A99059A12685200895A89
:10FA220088420CD90C9802A90988002200F01BFC1C
:10FA320001980699086004990868401C086014E05F
:10FA4200019806990968401A0B99059A12685200A2
:10FA5200895A884209D901980699086004990020B8
:10FA6200086005990868401C086002E005990020BA
:06FA7200086007B030BD82
:10FA780010B586B0089C05900491039202930898EB
:10FA880002990091411A0598049A801A48430399EB
:10FA9800891AFDF7B9FD009940180190019806B040
:02FAA80010BD8F
:10FAAA0000B581B000900098016808684022904330
:10FABA000860009984222020885000990020486715
:0AFACA00009800F0C6FC01B000BD7A
:10FAD40000B581B00090009926220C208854009A29
:10FAE4001068FF21283151188B239B00D25AF7F755
:06FAF400B3F901B000BDF2
:10FAFA0081B0009000998B2082000020885001B0CC
:02FB0A00704742
:10FB0C0081B0009000994520C200002088500099D7
:06FB1C00087501B07047FE
:10FB220010B588B00A9C07900691059204A803704C
:10FB320006984078039003980190032806D0019814
:10FB420006280CD00198102814D01EE007980699B8
:10FB5200059A04AB1B78FCF7ACFC02901CE00798FA
:10FB62000699059A04AB1B780A9C0094FCF717FDD2
:10FB7200029011E007980699059A04AB1B780A9C3B
:10FB82000094FCF794FD029006E007980399059B08
:0EFB9200012200F004F80290029808B010BDA5
:10FBA00084B00390029101920093029880300290F9
:10FBB00002980399009A88540098401C009001987C
:10FBC0000399009A88540098401C0090009804B053
:02FBD00070477C
:02FBD20070477A
:02FBD400704778
:10FBD60008D1002806D1F54204D801D3002A01D164
:10FBE6006D0D09D10020C143090DC904F0BDF9D13D
:10FBF6001242F7D1640DF5D00020C14349054908EA
:10FC0600A6E000206146F0BDF0B50127FF070E0013
:10FC16005E403E40B446BE0A4C18DD18F442D7D2C8
:10FC2600F542E4D2640DECD06D0DEAD06419C90238
:10FC36003943460DC0023143DB023B43DB0A10B4B5
:10FC46008E4685B297B26F43140C6C433E0CA419D2
:10FC5600260C2404BFB227439CB26C43A419190C8A
:10FC66006943250CA4B249190D04090C6419000C4A
:10FC760095B245433E0C76193743BFB2360C150C88
:10FC86004543AD19A6B2240CAD192E0437432E0CEC
:10FC960036199DB24543AD19ACB22E0C89191D0C0F
:10FCA60045436D182E04290C3443704680B295B234
:10FCB60045433E0C76193743BFB2360C150C454307
:10FCC600AD19A6B2AD19240C2E0437432E0C3619E5
:10FCD6009DB24543AD19ACB22E0C89191D0C454396
:10FCE6006D182E043443290C75462D0C90B26843CA
:10FCF6003E0C80190604BFB23E43070CA0B23F1863
:10FD0600120C6A43D019020C80B2240CA4189AB2C1
:10FD16006A43121914042043120C89181B0C6B43F6
:10FD2600C91810BC01273D05294203D1B619404127
:10FD36004941013CFF077D0D013D641B0BDB6D0056
:10FD4600AC4209DA240500254208BE4168416141FA
:0AFD560066463143F0BD54E74EE766
:10FD6000FF2109064000884201D800207047012089
:02FD70007047DA
:0EFD72000121090640004118484248417047EF
:10FD800030B581B0044668460170206900280FD064
:10FD90000CCC083C9A4233D26269531C6361815493
:10FDA000A069616981422BD1204600F02EF827E03E
:10FDB000E068002809D00CCC083C9A4220D2551C9F
:10FDC0009D4200D1002181541AE0A068002808D08B
:10FDD0000CCC083C9A4213D2551C9D420DD0C9B29E
:10FDE0000CE0236A002B0BD003CC083C884207D2DE
:10FDF000694601222046984702E000219200815086
:0AFE00002068401C206001B030BDF6
:10FE0A0010B54269002A07D00446036A002B01D0C4
:0AFE1A00216998470020606110BDC7
:10FE240080B5CB0606D4890501D5302100E0202118
:06FE340000F00EFD80BD90
:10FE3A0070B514460D460646FDF785FC0146304668
:0AFE4A002A462346FDF725FD70BD92
:10FE540081B0009000988068012109070840000FD4
:04FE640001B0704732
:10FE680081B00090009880680121084001B0704777
:10FE780000B585B0039003980068FEF77EFF0190F7
:10FE880003980068FFF7ECFF002842D0019800288B
:10FE98003FD103980068806805210840012808D1EF
:10FEA80003980068F3F7C0FD039801680320086011
:10FEB8000CE00399886D102210438865039AD16D70
:10FEC80001200143D16504A9087025E0F3F79AFAE7
:10FED8000290039800688068C007002819D0F3F7DB
:10FEE80091FA0299401A032812D30398006880688F
:10FEF800C00700280CD00399886D1022104388652C
:10FF0800039AD16D01200143D16504A9087003E06B
:10FF1800DFE704A90020087004A8007805B000BD38
:10FF280000B583B002900298806A01900198806DB4
:10FF38005021084238D10199886D0122520210439C
:10FF4800886501980068FEF7B4FE002828D001985B
:10FF5800807E002824D101980068006800070028E6
:10FF68001ED501980068FEF716FE00280ED10198EC
:10FF7800016848680C22904348600198806D01210F
:10FF88000843090288430199886509E00199886D49
:10FF98002022104388650199C86D01221043C86565
:10FFA800019800F06FF80DE00198806DC0060028F8
:10FFB80003D5019800F06AF804E00198006D416BE0
:08FFC8000298884703B000BD58
:10FFD00000B583B0019001985421405C012803D101
:10FFE00002A9022008704DE0019954220120885492
:10FFF0000198FEF7F0FD0146684601700078002880
:020000040801F1
:1000000039D10198006D2521405C02280ED101985C
:10001000006DF4F7BFFD01466846017000780028C6
:1000200004D00199886D40221043886501980168C9
:10003000486810229043486068460078002805D13F
:100040000198FFF719FF6946087002E00198FFF771
:1000500013FF68460078002807D10198806D0121C0
:100060000843090288430199886501980168C868B6
:1000700001229043C86001995422002088540098BE
:0C00800002A9087002A8007803B000BDBF
:08008C0081B0009001B0704743
:0800940081B0009001B070473B
:08009C0081B0009001B0704733
:1000A40082B0019000910198006807218905884376
:0C00B400009908430199086002B07047F1
:1000C00081B00090009901200002086001B07047E3
:1000D00081B00090009948680122120210434860E4
:0400E00001B07047B4
:1000E40081B0009000994868012212029043486050
:0400F40001B07047A0
:1000F80081B00090009901204002086001B070476B
:1001080081B000900099486801225202104348606B
:0401180001B070477B
:10011C0081B00090009948680122520290434860D7
:04012C0001B0704767
:1001300081B00090009880680121084001B07047AC
:1001400081B0009000988068C00F401E4142484135
:0401500001B0704743
:1001540081B0009000980068B42140587F21084085
:0401640001B070472F
:1001680000B583B0034602A80370019100920021F4
:0C01780040560199F4F716FA03B000BDE0
:04018400F4F77EFA14
:1001880000B581B000900098F4F786FA01B000BD80
:1001980083B00190009101984079012803D102A908
:1001A800022008703AE00199012048710199022063
:1001B80008710098102108400122824001980168C6
:1001C800086810430860009800280DD1019800685D
:1001D80000683E210840022805D101980168486856
:1001E80001221043486010E00198006800681F2150
:1001F80049040840009A02219140884205D101989B
:10020800016848680222104348600199012008717A
:1002180001990020487102A90020087002A80078FE
:0402280003B0704768
:10022C0085B00490039102920193002000900498F1
:10023C00006800900398002805D102980099401896
:10024C000830009004E00298009940181430009097
:0C025C00019800990860002005B0704770
:1002680083B0029001A801806846027000780028D7
:1002780004D001A800880299886103E001A80088D9
:080288000299886203B070477F
:1002900083B0029001A80180029949690091009AF7
:1002A0000188104608400004914340180299886173
:0402B00003B07047E0
:0802B40081B0009001B0704719
:0802BC0081B0009001B0704711
:0802C40081B0009001B0704709
:0802CC0081B0009001B0704701
:1002D40085B00490039102920498006A00900499F6
:1002E400086A012290430862049880690190019889
:1002F400F02188430190029801010198084301907C
:1003040000980A21884300900399009808430090BC
:1003140001980499886100980499086205B07047AF
:1003240085B00490039102920499086A10229043C4
:1003340008620498806901900498006A009001980A
:100344000F2109038843019002980103019808438F
:1003540001900098A021884300900398010100981F
:1003640008430090019804998861009804990862F0
:0403740005B0704719
:0803780081B0009001B0704754
:0803800081B0009001B070474C
:0803880081B0009001B0704744
:100390008AB00390039884214058212852D10398B1
:1003A0006A21405A02A9088002A80088002849D082
:1003B00003985621405A00282AD1EFF31080059067
:1003C0000598019001220992099880F310880398FA
:1003D00001688868D2059043886001980890089861
:1003E00080F31088EFF310800490049800900120AF
:1003F0000790079880F310880398016808684022E6
:100400001043086000980690069880F3108819E061
:1004100003980068C069000600280ED50399086D8E
:100420000078096888620399086D401C0865039983
:100430005622885A401E8852FFE70298401E02A9A1
:080440000880B1E70AB0704723
:0804480081B0009001B0704783
:0C04500082B001906846018002B0704745
:08045C0081B0009001B070476F
:0804640081B0009001B0704767
:10046C0083B0019001988021405C012803D102A93E
:10047C000220087026E001998022012088540199FD
:10048C00842224208850019800680068009001980C
:10049C00036818680121884318600098490788434D
:1004AC00009001990020486600980199096808603D
:1004BC00019920208850019980220020885402A99B
:0C04CC000020087002A8007803B0704700
:1004D80000B583B0029001A801700298806800906E
:1004E8000098401C0299496888420CD801980299E2
:1004F8000968009A88540098401C029988600299FB
:10050800C868401CC860029988684968884211D147
:10051800029A106911689268FEF79EF90299896833
:10052800884204D002990020C043C86002E00299C2
:080538000020886003B000BD43
:1005400030B589B00D9C0C9C0890079106920593DC
:100550000698002802D00698012802D101200390B5
:1005600001E00220039003980930049006980028C7
:1005700002D00698012802D10498401C04900898E3
:100580000599079A069B039C049D01950094FBF72F
:10059000C1FC089900204877089988840899088444
:1005A000089926228854089908770899C8830899D9
:1005B000222288540C9808998D22920088500D9818
:0C05C00008994722D200885009B030BDD5
:1005CC0081B00090009884214058212820D10098B7
:1005DC005621405A00280CD10098016808688022E6
:1005EC009043086000980168086840221043086036
:1005FC000DE00099086D0078096888620099086D13
:10060C00401C086500995622885A401E88520BE0FF
:10061C00009801680868802290430860009801687F
:0C062C00086840221043086001B07047CD
:1006380000B585B00490039104980399891EFBF7CF
:10064800BFFE014601A80180049A03998A18511E29
:1006580009780902921E12788A1869460A80008869
:100668000988884202D10398029002E00020C04322
:080678000290029805B000BDDC
:1006800000B585B00490039104980399FBF79CFE94
:10069000014602A80180029901AA117040786946BA
:1006A000087001980499039A88540398401C039099
:1006B00000980499039A88540398401C0390039867
:0406C00005B000BDC4
:1006C40081B000900098007D0121084001B070477E
:1006D40010B586B00590002004900598273003904B
:1006E4000598FFF708FA03980178059AFF20283047
:1006F400029011540499491C0491059C20180399F3
:10070400049A0B780094FFF70AFA0299049005986A
:1007140040180499FFF7B2FF0490049805998B22BE
:10072400920088500598FFF7D3F90598FFF7ECF984
:0407340006B010BD3E
:1007380000B581B000900098FCF7B6F9FCF7A4F971
:0407480001B000BD3F
:10074C00F0B581B01E4615460C4607461846FDF717
:10075C0099FF0146002000290AD46543A54207D31E
:10076C00304639462A46FDF7A7FF2146FCF772FFB3
:04077C0001B0F0BD1B
:04078000C00F7047EF
:1007840010B5FD22D343C20DD2B21446FF3C9C42A5
:1007940008D351184A1EFD2A05D8FF22D2059043DA
:1007A400C905084310BD0122D20710400129F9DB15
:0807B400FF21C905401810BD2A
:1007BC00C20DD2B2FF2A01D0002A02D100220A6057
:1007CC0070477E3A0A60FF21C90588433F2109061C
:0407DC00401870470A
:0807E000C1174840401A7047A0
:1007E80010B5002A0DD00446097848B200280AD46A
:1007F800002C00D02160002119605960411E8841F9
:0C08080010BD002010BD0120C04310BD39
:10081400024601207F2901D9C043704711707047F7
:0C082400014661391A2900D220387047C3
:0C083000014641391A2900D220307047DF
:0C083C00014661391A2900D220387047AB
:0C084800014641391A2900D220307047C7
:1008540070B5012A09DB0C460546561C284621467C
:0C086400FFF78CFA761E012EF8D870BD4C
:1008700010B50C46436A01212046FFF767FF10BD03
:10088000010002000400060008000A000C0010002D
:0808900020004000800000017F
:10089800547279696E6720746F207265737461721F
:0308A800742E00AB
:1008AB0043616E6E6F742072656164207374617442
:1008BB0069737463616C20646174612066726F6D1F
:0F08CB0020464C415348206D656D6F72792100B6
:1008DA004144432063616C6962726174696F6E207E
:0708EA006572726F722100BC
:1008F1005374617274696E6720566563746F7220F8
:100901005461626C6520636F7079696E67206672ED
:100911006F6D20464C41534820746F2052414D2E3B
:030921002E2E0077
:100924004D6F646520302069732073656C65637452
:1009340065642E204175746F2D7265636F6E6E65EC
:0B0944006374206973204F46462E00AC
:10094F004D6F646520312069732073656C65637426
:10095F0065642E204175746F2D7265636F6E6E65C1
:0B096F006374206973204F46462E0081
:10097A004D6F646520322069732073656C656374FA
:10098A0065642E204175746F2D7265636F6E6E6596
:0B099A006374206973204F46462E0056
:1009A5004D6F646520332069732073656C656374CE
:1009B50065642E204175746F2D7265636F6E6E656B
:0B09C5006374206973204F46462E002B
:1009D0004D6F646520342069732073656C656374A2
:1009E00065642E204175746F2D7265636F6E6E6540
:0B09F0006374206973204F46462E0000
:1009FB004D6F646520352069732073656C65637476
:100A0B0065642E204175746F2D7265636F6E6E6514
:0B0A1B006374206973204F46462E00D4
:100A2600555020627574746F6E206973206C6F6EFA
:0B0A3600672D707265737365642E00FD
:0B0A410056613A20253664206D5600F7
:0B0A4C0056623A20253664206D5600EB
:0B0A57004441435F413A202534640015
:0B0A62004441435F423A202534640009
:030A6D004F5000E7
:030A7000434C00F4
:030A7300424100FD
:030A7600414200FA
:030A7900257300E2
:030A7C004F5400D4
:030A7F004F4300E2
:030A82004F4C00D6
:030A85004C4200E0
:100A880043757272656E742063616C6C6962726121
:100A980074696F6E2073657175656E636520737414
:070AA80061727465642E0009
:100AAF00095B2534645D2053616D706C656420763D
:0B0ABF00616C75653A202534640A0064
:0B0ACA0048414C206572726F722100E1
:100AD50053415645204C4F434B2D4B455920434FD1
:070AE5004D4D414E442E006F
:100AEC0043616E6E6F7420726573746F72652064EF
:100AFC00656661756C742073657474696E677320B8
:100B0C0066726F6D20464C415348206D656D6F7257
:030B1C007921003C
:100B1F004A616E75617279004665627275617279AC
:100B2F00004D6172636800417072696C004D6179AC
:100B3F00004A756E65004A756C790041756775736B
:100B4F00740053657074656D626572004F63746FE6
:100B5F00626572004E6F76656D6265720044656303
:070B6F00656D626572000074
:070B7600414D00504D00004D
:0F0B7D002561202562202565202554202559005B
:070B8C00286E756C6C290056
:020B93000A0056
:100B95004465766963652049443A2053544D3332A0
:100BA50047304231206F722053544D333247304322
:020BB50031000D
:100BB7004465766963652049443A2053544D33327E
:100BC70047303731206F722053544D333247303816
:020BD7003100EB
:100BD9004465766963652049443A2053544D33325C
:100BE90047303531206F722053544D3332473036F8
:020BF9003100C9
:100BFB004465766963652049443A2053544D33323A
:100C0B0047303331206F722053544D3332473034D9
:020C1B003100A6
:100C1D004672656520737061636520666F7220632F
:100C2D006F66696775726174696F6E20696E206693
:100C3D00616B6520454550524F4D3A202575206218
:060C4D00797465730A00D2
:100C53004D41585F504F535349424C455F444946B9
:100C6300465F544F5F4D4541535552453A202575D4
:020C73000A0075
:100C750043616E6E6F7420737461727420414443D6
:0E0C850020696E20444D41206D6F6465210092
:100C930043616E6E6F7420636F7079205665637461
:100CA3006F72205461626C652066726F6D20464CD2
:100CB30041534820746F2052414D2120444D41201F
:0E0CC3006973206E6F74207265616479210080
:100CD10043616E6E6F742066696E69736820636F1D
:100CE1007079696E6720566563746F722054616212
:100CF1006C652066726F6D20464C41534820746FBD
:060D01002052414D2100CB
:100D07004D6F646520302069732073656C6563746B
:100D170065642E204175746F2D7265636F6E6E6505
:0A0D27006374206973204F4E2E0004
:100D31004D6F646520312069732073656C65637440
:100D410065642E204175746F2D7265636F6E6E65DB
:0A0D51006374206973204F4E2E00DA
:100D5B004D6F646520322069732073656C65637415
:100D6B0065642E204175746F2D7265636F6E6E65B1
:0A0D7B006374206973204F4E2E00B0
:100D85004D6F646520332069732073656C656374EA
:100D950065642E204175746F2D7265636F6E6E6587
:0A0DA5006374206973204F4E2E0086
:100DAF004D6F646520342069732073656C656374BF
:100DBF0065642E204175746F2D7265636F6E6E655D
:0A0DCF006374206973204F4E2E005C
:100DD9004D6F646520352069732073656C65637494
:100DE90065642E204175746F2D7265636F6E6E6533
:0A0DF9006374206973204F4E2E0032
:100E0300555020627574746F6E206973207072651B
:060E1300737365642E00FC
:020E19004E0089
:060E1B00523A202573008D
:020E21000A00C5
:100E230043616E6E6F7420736176652064617461D3
:100E330020696E20464C415348206D656D6F727971
:020E430021008C
:0E0E45004E4D49204552524F522121210A00A4
:0A0E530053746167652023300A0024
:0A0E5D0053746167652023310A0019
:0A0E670053746167652023320A000E
:020E710043003C
:020E73002E004F
:100E750053756E646179004D6F6E646179005475C8
:100E85006573646179005765646E657364617900A3
:100E9500546875727364617900467269646179009A
:0A0EA50053617475726461790000F6
:050EAF004D41494E0019
:100EB40043616E6E6F742073746172742054494D73
:050EC40045523221003F
:050EC9001B5B324A0032
:100ECE0050726F6772616D20737461727465642EF7
:010EDE000013
:100EDF0043505520467265713A20257520487A0A8D
:010EEF000002
:100EF00043616E6E6F74207265616420636F6E660D
:100F0000696775726174696F6E2066726F6D2046D5
:0D0F10004C415348206D656D6F72792100D2
:100F1D00257325733A204144432043616C69627205
:100F2D006174696F6E2076616C75653A2025750A5E
:010F3D0000B3
:100F3E0043616E6E6F742073746F70204144432151
:010F4E0000A2
:100F4F0025733A204441432043616C696272617496
:100F5F00696F6E2076616C756520666F72206368AD
:0D0F6F00616E6E656C20313A2025750A0018
:100F7C0025733A204441432043616C696272617469
:100F8C00696F6E2076616C756520666F7220636880
:0D0F9C00616E6E656C20323A2025750A00EA
:100FA90049742069732074696D6520746F207361B9
:100FB900766520737461746973746963616C206404
:100FC90061746120696E20466C617368206D656D7E
:050FD9006F72792E008B
:100FDE00496C6C6567616C204D6F64652069732088
:100FEE0073656C65637465642E2044656661756C0B
:100FFE0074204D6F646520342069732073656C65B1
:10100E00637465642E204175746F2D7265636F6E07
:0D101E006E656374206973204F46462E00F6
:05102B00257325730090
:09103000493A20253564204100F5
:091039004F56503A202531730096
:091042004C56503A202531730090
:0D104B00543A202532642E256420B0430065
:10105800095B2534645D2053616D706C656420768E
:10106800616C7565733A20492B203D202536752023
:0D107800202020492D203D202536750A003E
:1010850009094F66667365742076616C7565733AF8
:1010950020492B203D20257520202020492D203D4D
:0510A5002025750A0082
:1010AA0009094F66667365742076616C75653A2026
:0510BA002534640A006A
:1010BF00556E6B6E6F776E20636F6D6D616E642111
:0110CF000020
:0D10D0005553415254206572726F72210019
:1010DD0053756E004D6F6E00547565005765640055
:0D10ED00546875004672690053617400007C
:1010FA004A616E00466562004D617200417072007D
:10110A004D6179004A756E004A756C004175670039
:10111A00536570004F6374004E6F76004465630038
:01112A0000C4
:01112B0000C3
:09112C00256D2F25642F257900A3
:0911350025483A254D3A255300E6
:0D113E00000703200417020108571040802D
:05114B002D494E460095
:051150002D696E660030
:051155002B494E46008D
:05115A002B696E660028
:08115F0001010103070100007A
:08116700080402040801010163
:10116F0030313233343536373839414243444546CE
:08117F001B5B323B33326D00B3
:081187001B5B323B33336D00AA
:08118F001B5B323B33316D00A4
:1011970025733A205265766973696F6E206E756D97
:0C11A7006265723A2030782534580A0046
:1011B3004672656520737061636520666F72207384
:1011C30074617469737469637320696E2066616BFB
:1011D3006520454550524F4D3A202575206279745C
:0411E30065730A0026
:1011E700435055207370656564206973206E6F7472
:0811F7002036344D487A210036
:1011FF004669727374207374617274212057726917
:10120F0074696E672064656661756C7420636F6EB8
:0C121F0066696775726174696F6E21006A
:08122B001B5B313B33326D0007
:10123300566563746F72205461626C6520686173D4
:10124300206265656E20636F706965642066726FE6
:101253006D20464C41534820746F2052414D2E005F
:10126300496C6C6567616C204D6F64652069732000
:1012730073656C65637465642E2044656661756C83
:1012830074204D6F646520342069732073656C6529
:10129300637465642E204175746F2D7265636F6E80
:0C12A3006E656374206973204F4E2E00AE
:1012AF00444F574E20627574746F6E2069732070AF
:0812BF007265737365642E0073
:0812C7001B5B323B33306D006C
:0812CF002573207C202573002B
:0C12D7005661623A20253464206D5600F8
:0C12E3005662623A20253564206D5600EA
:1012EF001B5B323B33316D591B5B313B33326D002E
:0812FF001B5B313B33316D0034
:081307001B5B313B33366D0026
:08130F00434847202D20310066
:08131700434847202D2030005F
:10131F000909566F6C746167652D64726F70204197
:10132F0044432076616C75653A202535642E0A009A
:10133F0009090946696E616C20766F6C7461676587
:10134F002D64726F70204144432076616C75653A4D
:10135F00202534752E2046696E616C20766F6C7473
:10136F006167652D64726F702076616C75653A20C8
:08137F00253375206D560A00AC
:1013870043616E6E6F742073617665206E6577209A
:10139700534E20696E20464C415348206D656D6F52
:0413A7007279210036
:1013AB0043616E6E6F742073746172742054494D77
:1013BB00313720696E20495352206D6F64652100CF
:0413CB004D4F44003E
:0813CF001B5B313B33316D0063
:1013D700486172646661756C74204552524F5221A0
:0413E70021210A00B6
:1013EB00202020202020202020682828282820208A
:1013FB0020202020202020202020202020202020E2
:10140B004810101010101010101010101010101099
:10141B008484848484848484848410101010101039
:10142B001081818181818101010101010101010192
:10143B000101010101010101010101101010101046
:10144B001082828282828202020202020202020263
:10145B00020202020202020202020210101010200B
:10146B0030313233343536373839414243444546CF
:10147B0030313233343536373839616263646566FF
:04148B004E414E0080
:04148F006E616E001C
:01149300FF59
:10149400093C010843070020B10E00001B3C010871
:1014A40000000020C4140108430700001B3C01088D
:1014B40000600020071C0108002000001BEA00084F
:1014C40082B00E480168C96A01910068006B0090FF
:1014D40001980F2802D301980F38019000980F2823
:1014E40002D300980F380090019804490A6890606C
:1014F40000980968486102B07047C0464013002054
:1015040082B010480168C96A01910068006B0090BC
:101514000198FF210901884202D801980F300190F7
:101524000098FF210901884202D800980F300090EA
:10153400019804490A68906000980968486102B0FB
:101544007047C0464013002082B00E480168C96A43
:1015540001910068006B009001980F2802D3019854
:101564000F38019000980F2802D300980F3800908C
:10157400019804490A68906000980968486102B0BB
:101584007047C0464013002082B010480168C96A01
:1015940001910068006B00900198FF2109018842C5
:1015A40002D801980F3001900098FF210901884268
:1015B40002D800980F300090019804490A6890609E
:1015C40000980968486102B07047C0464013002083
:1015D40082B00E480168C96A01910068006B0090EE
:1015E40001980F2802D301980F38019000980F2812
:1015F40002D300980F380090019804490A6890605B
:1016040000980968486102B07047C0464013002042
:1016140082B01D480068C06A01901C4800681C49DB
:101624003A22895E40181B49884206DC01980F283B
:1016340002D301980F38019010E01448006814494F
:101644003A22895E40181449884207DB0198FF2139
:101654000901884202D801980F30019001990A4883
:10166400026891600068006B00900098FF210901F6
:10167400884202D800980F30009000980249096807
:10168400486102B07047C04640130020B8130020E0
:10169400C8140020970900009909000082B01D4871
:1016A4000068006B01901C4800681C493A22895E5E
:1016B40040181B49884208DC0198FF21090188422F
:1016C40002D801980F3001900EE0134800681349C6
:1016D4003A22895E40181349884205DB01980F2895
:1016E40002D301980F38019001990A4802685161A8
:1016F4000068C06A00900098FF210901884202D85E
:1017040000980F300090009802490968886002B080
:101714007047C04640130020B8130020C8140020AE
:10172400650600006706000082B00E480168C96AB9
:1017340001910068006B009001980F2802D3019872
:101744000F38019000980F2802D300980F380090AA
:10175400019804490A68906000980968486102B0D9
:101764007047C0464013002082B010480168C96A1F
:1017740001910068006B00900198FF2109018842E3
:1017840002D801980F3001900098FF210901884286
:1017940002D800980F300090019804490A689060BC
:1017A40000980968486102B07047C04640130020A1
:1017B40082B010480168C96A01910068006B00900A
:1017C4000198FF210901884202D801980F30019045
:1017D4000098FF210901884202D800980F30009038
:1017E400019804490A68906000980968486102B049
:1017F4007047C046401300207047010180B500F0D7
:101804008BF880BD10B584B01E48029000891E4933
:1018140008801E480068804702998A881C48026034
:101824004A891C490A601C4B1A68022422431A6024
:1018340000680968884203DB15480068019002E0EB
:1018440014480068019001980390039813494022BA
:10185400895E884210D3039A11480168891801608F
:10186400006810490968884205D90F480068804714
:101874000B490020086002E009490020086004B018
:1018840010BDC046DE150020B81300202C14002023
:10189400BC130020C013002004000240C814002020
:1018A40090140020640600204C14002080B500F041
:1018B4003BF80C2000F040F80B490C4808600C4839
:1018C400006800280ED10B49012008600A49096804
:1018D4000A4A11600A4A41218B00D15A491CD1524B
:1018E4000849086080BDC0462C140020390300203C
:1018F400C4130020C8130020440700206006002001
:10190400C8140020B413002080B5024800F01CF86D
:1019140080BDC046A40F002008B4024B9C4608BCFE
:101924006047C046F533000808B4024B9C4608BC27
:101934006047C046B5AF000808B4024B9C4608BCDB
:101944006047C046ABED000808B4024B9C4608BC97
:101954006047C04651C1000800B589B064200890B2
:101964000A20079020200690032005900020049070
:1019740003900290314800680190002806D0019835
:1019840001281CD00198022832D055E0324800F0DA
:1019940065F800200490039004982A490A6890602E
:1019A4000398096848610298411C0291202805DBCC
:1019B4000020029021490868401C08603CE024484B
:1019C40000F04CF823480490039004981D490A68D9
:1019D40090600398096848610298411C02910328A9
:1019E40005DB0020029015490868401C086023E0CC
:1019F400134800F033F80020049003900498114930
:101A04000A6890600398096848610298411C029131
:101A1400202811DB0020029008490860092000F00A
:101A240025F809480068002803D0074800680749DA
:101A34000860092000F022F809B000BD2414002039
:101A4400670E010840130020101400202C140020FD
:101A54005D0E0108FF0F0000530E010808B4024B8D
:101A64009C4608BC6047C04615D9000808B4024B20
:101A74009C4608BC6047C046ABED000808B4024B66
:101A84009C4608BC6047C04695ED000888B00590A8
:101A9400049103A90020087005980290049801900D
:101AA400154908680122920410430860EFF310807E
:101AB40006900698009072B603A800783F280ED8C6
:101AC40001980068029908600198001D019002982D
:101AD400001D02900398401C03A90870ECE7074816
:101AE4000068C003002800D5F9E70098079007981C
:101AF40080F3108808B07047142002401020024080
:101B040074E9000874E9000874E9000874E900083D
:101B140074E9000804000000FFFFFFFFC0E0FFFFBE
:101B2400C0E0FFFFFFFFFFFFDC130020E0130020F5
:101B3400E41300200024F400010000000100000070
:101B4400FFFFFFFF01000000FFFFFFFF0100000097
:101B5400FFFFFFFF01000000B80B000000B80B00FE
:101B64000200000001000000040000000100000069
:101B7400020000000100000000000000020200005A
:101B84000000000202020202010000000000000046
:101B94000000000000010101000101000100020237
:101BA400010100000000000000000000000000002F
:101BB4000000000000000000000000000000000021
:101BC4000000000000000000000000000000000011
:101BD4000000000000000000000000000000000001
:101BE40000000000000101010100010100000001EA
:101BF40001010100000000000000000000000000DE
:101C0400000000CDCDCDCDCDCDCDCDCDCDCDCDCD67
:101C1400CDCDCDCDCDCDCDCDCDCDCDCDCDCDCDCDF0
:101C2400CDCDCDCDCDCDCDCDCDCDCDCDCDCDCDCDE0
:101C3400CDCDCDCDCDCDCDCDCDCDCDCDCDCDCDCDD0
:101C4400CDCDCDCDCDCDCDCDCDCDCDCDCDCDCDCDC0
:043C0400CDCDCD0055
:103C0800206861680834002200E042540139FCD57C
:023C18007047F3
:103C1A0020686168A2680C3401E08B5C8354013A25
:043C2A00FBD570470F
:103C2E00FFFFFFFFFFFFFFFFFFFFFFFFFFFFFFFF96
:103C3E00FFFFFFFFFFFFFFFFFFFFFFFFFFFFFFFF86
:103C4E00FFFFFFFFFFFFFFFFFFFFFFFFFFFFFFFF76
:103C5E00FFFFFFFFFFFFFFFFFFFFFFFFFFFFFFFF66
:04EFFC00AE7A8CB9A4
:040000050800EB996B
:00000001FF
